:020000040800F2
:1000000000A000203D34010811E30008712401081C
:100010000FE300080DE300080BE3000800000000F8
:1000200000000000000000000000000009E30008DC
:1000300007E300080000000005E300081DC20008F7
:10004000A5340108A5340108A5340108A534010828
:10005000A5340108A5340108A5340108A534010818
:10006000A5340108A5340108A5340108A534010808
:10007000A5340108294800084BDE0008A534010812
:10008000A5340108A5340108A5340108A5340108E8
:1000900071E30008A5340108A5340108A53401085E
:1000A000D1080108FD080108C10801080D0901086F
:1000B000F1080108E1080108A5340108A534010888
:1000C000A5340108A5340108A5340108A5340108A8
:1000D000A5340108C90A0108BD0A0108B10A0108CE
:1000E0002DC20008A53401086D040108A5340108DB
:1000F000A5340108A5340108A5340108A534010878
:10010000000000000000000000000000A53401080D
:10011000A5340108A5340108A5340108A534010857
:10012000A5340108A5340108A5340108A534010847
:10013000A5340108A53401080000000000000000FB
:10014000A5340108A5340108A53401080000000009
:10015000000000000000000000000000000000009F
:100160000000000000000000A5340108A5340108CB
:10017000A53401080000000000000000000000009D
:0801800000000000A534010895
:100188002DE9F04F2DED028B6F4E704B3360AFB001
:100198000023736010F048FF18B910F067FF09F0EA
:1001A800ADFA09F065FB6A4B6A4C1A7842F0010215
:1001B8001A70694A4FF47001C2F888100022099237
:1001C8000A92226842F4803222600493236803F47E
:1001D80000330A93099B013309930A9B1BB9099BB6
:1001E800B3F5A04FF2D1236813F4003318BF0123ED
:1001F8000A930A9B012B70D0574F584BFB60636AD8
:10020800B360636ADFF884A1DFF88481DFF8849142
:1002180043F080736362636943F4FC032EAD63614A
:1002280003238DF86A3041F6FF7325F8503D4FF0EF
:100238009040294604F0EAFB4FF6FF7350462946E2
:10024800ADF8683004F0E2FB4548294604F0DEFBCF
:100258004448294604F0DAFB4348294604F0D6FB13
:100268002946424804F0D2FB284607F005FE1A9BAF
:100278003F4AB3FBF2F33F4A3F4913603F4B00222A
:100288001A603F4B5960F02187F823109A603D4F60
:1002980007221A60BB68C8F8003099E80F0085E8A3
:1002A8000F0063691A9843F480236361636943F418
:1002B800802363614FF0200B1023CAF818301BA964
:1002C800CAF818B004F0A2FB1DA91C9804F09EFB04
:1002D800D8F80030190729D464E02B4B12221A6091
:1002E8006368636063686360636843F48063636042
:1002F800636823F47C136360636843F4E813636002
:10030800236843F0807323602268124B9201FBD567
:100318005A6822F003025A605A6842F002025A6090
:10032800636803F00C03082BFAD165E797F892315C
:10033800012B37D8044B97F893219B6813F080530F
:1003480000F0A7842EE000BF800100207F8F000806
:10035800A42F00200010024000ED00E00005FA057F
:1003680000080048000C004800100048001400482D
:1003780040420F00B41800203F190100F018002077
:1003880010E000E0A0240020002002400004004803
:1003980040240020987D0108B54B002283F8932162
:1003A80009F002FC64200BF0BEFDC822B148002110
:1003B80015F029FBE369B04A43F00303E361A3693D
:1003C80043F4A123A361636943F4C023636102F189
:1003D800B00C937B506892F80FE003F00701DB083C
:1003E80000EB83038900186A4FF00F0A0EFA01FE2A
:1003F8000AFA01F120EA01011962196A10324EEA7B
:10040800010162451962E4D10023DFF894A20AF1E0
:100418000C020021995401330B2BF6D1FF23974A84
:100428008AF817308AF818308AF819308AF81A309A
:100438008AF81B30924BDFF86CB21360914A039331
:10044800042010705846302215F0DDFA14220221DB
:100458008BF800208BF8241001228B49039B8BF822
:10046800182097F805B081F800B0A3F5EA71CAF82A
:100478001C108649D8F80080A3F58A730B60844B5A
:1004880003EBCB0318F0200F5B78CAF8203018BFB5
:10049800CAF8202000237F4A40F2DC5122F81310CA
:1004A8000133082BF7D113A800211C2215F0ABFA51
:1004B800BBF10E0F03D00BF0EF03082B02D1012381
:1004C8008DF85C3002200BF0BBFB18B1408800307F
:1004D80018BF0120C8F340038DF85230C8F38013C9
:1004E8008DF85430C8F340338DF84C30C8F3C0331E
:1004F80000F001008DF84F3018F400638DF85100BA
:1005080007D097F8863103F1FF3EDEF1000343EB95
:100518000E038DF85030C8F300438DF85530336A18
:10052800B7F84801ADF86000003318BF01238DF813
:100538005630C8F300538DF85730B7F84A31ADF844
:100548005A3018F4805FB7F8563118BF4848ADF8EC
:100558005830C8F380438DF85330B7F854311CBF76
:10056800B0F85001ADF86000B3F5FA7FADF85E3031
:1005780084BF0023ADF86030474897F8CE3186F83D
:100588002430002386F8253043709DF85C3008F04D
:100598000101002BC8F3C0028DF84D108DF84E20D4
:1005A8000CBF0023022301B902B1013309EB83090F
:1005B8004FF0000AD9F810309A1E143303920593AD
:1005C800039A32F8023F03924FF6FF72934200F00B
:1005D80089819DF85100190ADAB2CBB280B1264F51
:1005E800DFF8C4E007EB02177868704508D138894E
:1005F800B0F5806F00F07181B0F5006F00F06D818B
:100608009DF8550090B11001DFF86CE00EEB000783
:100618005EF800E02148864500F05F817868B0F117
:10062800904F03D1B87B062800F057819DF85200FF
:1006380050B1114F07EB02177868B0F1904F03D112
:100648003889102800F049819DF8500050B10A4FB0
:1006580007EB02177868B0F1904F03D138898028EA
:1006680000F03B81022921D19DF84C1022E000BF07
:10067800A02400202819002028A00108FC2200201E
:10068800882600209D1200209C0A00206C1A002059
:10069800DCAB01080C120020A50100200044014039
:1006A800800100200023002000040048012904D113
:1006B8009DF84D10002900F010819DF85600BF49A3
:1006C8004FEA021850B19DF85C0038B9012A05D8E4
:1006D80051F80800BA4FB84208BF04239DF85700E4
:1006E80001EB080730B19DF85C0018B9043A032AF9
:1006F80040F2DC80012B53D19DF85330DFF8D092C3
:100708003BB151F80830B3F1804F04BF032389F897
:100718002730AA4AC9F87C7002EB0801FF2391F838
:100728000DE089F86C3089F86D3048688DF86AE01A
:1007380001F108030989ADF868104FF0000B022198
:100748008DF86B1089F870B01AA90792069389F88A
:1007580028B0C9F82CB0C9F830B0C9F834B0C9F815
:1007680068B089F86EB089F86FB004F04FF9069B4D
:10077800079A997852F808005A4603F09BFF3846C2
:1007880010F0C2F98F4B9049C9F880308F4BC9F8E7
:100798008430C9F888B038460A1D10F02BF99CE05F
:1007A800022B49D15FFA8AF21C2101FB02FC884A1C
:1007B800CDF81CC002EB0C09804A89F871A0012110
:1007C80089F8701002EB08014FF0000B91F80DE06A
:1007D800486889F872B001F108020989ADF8681013
:1007E80089F87AB01AA9C9F87C708DF86AE006927F
:1007F8008DF86B3004F00AF9704B069A53F808002C
:1008080091785A4603F056FF384610F07DF9704B40
:10081800DDF81CC06F4AC9F8802003EB0C016E4A52
:10082800C9F884208031C9F888B038460A1D10F00C
:10083800E1F80AF1010A50E0032B35D19DF8533055
:10084800DFF88C81DFF8C4913BB198F826B03846C0
:1008580008214FF6FF7200231AE0BDF85E2098F8D1
:1008680026B0BDF86030B2F5FA7F0BD95B49B1FB11
:10087800F2F23846082192B204F0F1F8584B49F8E0
:100888002B000AE05749B1FBF2F23846012192B237
:1008980004F0E5F8544B49F82B00C36098F826306B
:1008A800013388F8263018E0042B16D196F82580F5
:1008B800BDF858204B4B93FBF2F23846BDF85A303E
:1008C800012192B204F0CBF896F8253006EB88089F
:1008D8000133C8F8500186F82530039B059A9342E6
:1008E8007FF46EAE96F8252086F870213F4A404B7B
:1008F80092F800E0AEF117020027022A1F709C460A
:100908001AD8F3693B44D3ED007AF5EE407AF1EE5C
:1009180010FA02D1336A63BB26E0364A07EB0208B5
:100928000FCB88E80F009CF8003010370133C02F38
:100938008CF80030E5D1EDE72F4B13F83E908CF89A
:10094800009003EBCE03D3F804A0BAF1000FE1D076
:100958004F45DFDA274A3B0103EB020853440FCB2C
:10096800013788E80F00F3E7244F3B68DE0451D4D1
:100978001DE0234B234A13F83E00107003EBCE030F
:100988005E68002EF0D000238342EDDAC3EBC3018A
:100998007218DFF87C80D2F8009041F8089001EBDB
:1009A80008079188B9809279BA710133ECE70EF0A3
:1009B800EF03082B144B4DD14FE000BF28A00108CE
:1009C800004001404544000800020020314500086D
:1009D80080010020B94700081D44000800127A0071
:1009E8005145000840420F00414500089C0A00207C
:1009F80024190020D8090020DCAB0108402400207D
:100A080088830108F819002070140020F4180020C9
:100A1800F91900209CF80020012AC8D9B94B03EB2A
:100A28000212103210339342C1D053ED047AB6EE5D
:100A3800007A67EE877A43ED047A53ED057A67EE1C
:100A4800877A43ED057A53ED037A67EE877A43EDAB
:100A5800037AE7E7BEF10E0F09D11A7842F01002C7
:100A68001A70BEF1180F09D10BF092FD06E01A7842
:100A780022F010021A70BEF1190FF4E70BF06CFDAA
:100A88003B68A14E58035EBFA04B01221A70049B1D
:100A9800049A1B7843F0040313709D4B1E6063692E
:100AA80043F400336361E36943F48003E361236B38
:100AB80023F020032363236B43F080534FF09048C7
:100AC80043F020032363D8F8243023F0F003C8F858
:100AD8002430D8F8243043F04003C8F82430D8F83C
:100AE800243023F47063C8F82430D8F8243043F451
:100AF8008063C8F824304FF0000902234FF40072D5
:100B080029464FF0030B40468DF86C3004931A9237
:100B18008DF86E908DF86F908DF86DB007F01AFB18
:100B28004FF48062294640461A9207F013FB326858
:100B380022F0010232603168764A0A403260764A11
:100B48003261326842F001023260C6F80890C6F895
:100B58000C90C6F80890B26842F40042B26032685D
:100B68003260726822F0784222F400427260326881
:100B780042F0010232603D68684E4FF0100A05F4F9
:100B88000063524630464946039314F03CFF4FF643
:100B9800FF72049B0E9215F002058DF83D308DF81A
:100BA8003E908DF83F908DF83CB00CD02EA9404671
:100BB80041F880AD07F0CEFA01250723357086F895
:100BC8000190F370B570039B83B12EA9802341F87F
:100BD800803D4FF0904007F0BDFA0423337307239C
:100BE800F373012375731D44B373EDB2E36A4C4884
:100BF80023F4F873E362E36A43F4D873E362636946
:100C080043F0805343F00203636107F06AF81AA8BF
:100C180007F03CF8434B1A93434B1B93022D4FF0BC
:100C2800000314BF1A4680221F924FF480723C4C76
:100C380020924FF4806221922022204622921AA903
:100C48004FF400521C931E9323922493ADF87450D2
:100C580007F029F8236843F001032360334CA368A5
:100C680023F04053A360A36843F08053A3600A2095
:100C78000BF059F9A36823F08043A360A368A3602D
:100C8800A36843F00043A360A368284A002B51DA05
:100C9800FAE7013A092A3FF685ABD9F8240003930D
:100CA8002946AAF828B028604FF0904003F0AEFE1D
:100CB8004FF09042082191613C200BF034F9039BDE
:100CC800CAF818B09A4697F893319A45BFF664ABBC
:100CD800174A4FF0904B1021082391617820069114
:100CE8000592ABF8283003930BF012F9059A069990
:100CF800039B11857820CBF818300BF009F90AF11D
:100D0800010AE0E7E009002000580040080F002031
:100D1800D8110020FFE0CF007A25E0007C160020E3
:100D280008040240400100508C16002000010050C9
:100D3800000400489368AC4923F0405393609368DB
:100D480043F0005393608868A84B034043F468332A
:100D58008B60D168A64B0B4043F40053D360136BF0
:100D6800013D23F00F031D431563002401233219AD
:100D78009178002972D05D1C042B16F804E0D07815
:100D8800DFF870C2EDB20ED803EB43035A00DCF86B
:100D980030101F23934021EA03010EFA02F30B439C
:100DA800CCF8303031E0092B0ED8053B06225A43E7
:100DB800DCF834101F23934021EA03010EFA02F3F2
:100DC8000B43CCF8343020E00E2B4FF006010ED840
:100DD800A3F10A024A43DCF838801F23934028EA2B
:100DE80003010EFA02F30B43CCF838300DE00F3B49
:100DF80001FB03F2DCF83C801F23934028EA03013F
:100E08000EFA02F30B43CCF83C30BEF1090F794AD5
:100E180011D993699169AEF10A0303EB43034FF0CB
:100E2800070E0EFA03FE21EA0E01916191699840BE
:100E38000843906111E0536951690EF1FF3303EBE8
:100E480043034FF0380E0EFA03FE21EA0E015161FA
:100E5800516903339840084350612B460434102CE1
:100E680085D1644B9A6842F001029A601A4611686B
:100E7800604BC907FBD5DA685F4C22F00202DA60E2
:100E8800DA6842F00202DA60DA6842F00102DA60F7
:100E98009A6842F004029A60B4F85C31002B40F082
:100EA8009087B4F95E21002A40F08B87B4F960215D
:100EB800002A40F086873B689B0320D5C8200BF0AA
:100EC80032F8AE200FF063FC08B10FF065FC4B4D13
:100ED80085F87101C8200BF026F8494BC5F8743124
:100EE800484D00210C22284614F08DFD0223EB709A
:100EF80009F083FB0AF0F2FF434B0344AB6094F81C
:100F08006B310393414B42481B68B4F86461B3F8F2
:100F18005630049300210C2294F863B194F86C5174
:100F2800B4F80C9094F80FA014F06DFD394B0693AB
:100F380018460021142214F066FD374A002111706A
:100F48002E4A0592C2F878110FF0E3FB059A804605
:100F5800002833D0069B314919603149596031491D
:100F6800D960B6F5807F30491961304B01D1002135
:100F780016E0BB2E01D9012112E0612E01D9022110
:100F88000EE0292E01D903210AE0132E01D90421EC
:100F980006E0092E01D9052102E0002EE7D006213E
:100FA80019701D4B04211970214B02211970214918
:100FB8000B6843F001030B6059460FE003200BF068
:100FC800F7F835E24FF0010B0BFA01F040F2B233BB
:100FD80003409BB3012940F28D800021164800236D
:100FE80009290370F9D8EDE700030050E010FCFF71
:100FF80007C0FFFD00010050A02400208001002050
:101008002A260020801A0020404B4C001C12002089
:10101800D0210020902C00208A0F0020FD05010817
:10102800310501081105010890C1793D0000002033
:10103800080100206C140020CC2F002010F04D0F68
:10104800C8D00691C2F8783105920FF062FB059A74
:1010580006990028BED0062168200A460DEB000339
:1010680003F0EAFD9DF86D1001EA0B029DF86B1084
:1010780001EA0B0101FA0BF343EA82019DF86920AA
:1010880002EA0B030B430BD05BB25B4501D1002294
:1010980002E0022B0FD10122AF4B83F87C2111E033
:1010A8000EAB68200C215A4603F0C6FD9DF8383077
:1010B80013F00F0303D105200BF07AF802E0042B9C
:1010C800E9D1E4E7A54BA64A1A60A64A5A60A24AA3
:1010D80092F87C21002A0CBF6F226E221A72A24B52
:1010E80004221A70A14B03225A70A14A136843F0D4
:1010F80002031360042D00F2A380DFE805F003BEAD
:101108006B036B000A200AF00EFF7720A021012252
:101118000EAB03F091FD00285CD01E210122772040
:1011280003F006FE4FF42F600AF0F2FE4FF0000BBA
:10113800ABF160010025C9B202221AAB77208DF805
:1011480068508DF8695003F077FD9DF869309DF877
:10115800682043EA0222804B03F5BF712BF8012077
:101168000BF1020BBBF1100FE2D1B3F88C2102F0A6
:101178000F0E02F47F42A3F88C2101202B4629464A
:10118800DFF8D4C121F001056544B5F87E51002D82
:1011980018BF002011F0010F03D0EDB26B400825F5
:1011A80002E083EA1523FAE713F4004F18BF83F42B
:1011B800C053013D4FEA4303F6D101311029DFD175
:1011C800654942EA0E02A1F88C2118B9C3F303332A
:1011D8009E4538D0604D95F88EB1BBF1000F40F0B8
:1011E800E68514200AF09FFE05F28F137620D021A1
:1011F800012203F021FD95F88F31582B3DD105F5DB
:10120800C87388211822762003F016FD3122762033
:10121800F42103F08DFD012385F88E31554B564A94
:101228009A60564A5A6045F6D8125A80544ADA608B
:10123800544A1A61544AA3F800B05A6100F0B7BD85
:10124800012D13D119E04B4B42F210721A805A80CB
:101258004E4A5A604E4A9A604E4ADA604E4A1A61BD
:101268004E4A5A61B8F1000FB4D003253F4B404AAB
:101278009D70136843F0040313603D4D2B689A0773
:1012880002D5364B1B6898473349454ABAF1000FD7
:1012980025D016F0FF0F0AD12B6813F0020F4FF07C
:1012A8007D0040F2712308BF4FF4FA7302E04FF457
:1012B8007A731846994505DBB9F57A6FA8BF4FF4DC
:1012C8007A6900E09946431E4B44B3FBF0F3013BB7
:1012D800DBB203FB000081F8AC31106003E081F859
:1012E800ACA1C2F800902F4B1B689847DDF80CA002
:1012F8002D4E00233370BAF1000F04D0AAF1020278
:10130800012A00F257852EAB4FF0000903F8509DD3
:101318000C204946012203F08FFC002800F0798553
:101328009DF86830482B13D1204B214A1A60214A76
:101338005A604046B8F1000F00F06B850523337002
:101348000A4B0322DA702B6843F008032B6033E062
:10135800484600F05EBD00BF80010020D02100207B
:101368006D06010871050108CC2F00200801002036
:101378006C140020F40600204D5F00084F5F000841
:10138800DD61000873620008515D0008BF040108B0
:1013980001050108B5040108F1040108515F0008BE
:1013A800D42C0020902C0020CD2F0020D006002027
:1013B800BD620008E7610008174B93F858210AB18D
:1013C80016490A7093F859210AB115490A7093F819
:1013D8005A3103B133702B68124913F0080F25D026
:1013E800BDF91000DFED106A642290FBF2F302FBF6
:1013F800130212B207EE902AB8EEE77A07EE903A97
:10140800F8EEE77AE7EE267AB2EE047A67EE877AA4
:10141800C1ED007A0CE000BFA02400208A0F002054
:10142800CC2F0020781A00208988883C00230B6084
:10143800AC4B1A7842F002021A70AB4A202111858F
:10144800102191610A259846A74EB38A9BB283F072
:101458002003B382B38A9BB283F01003B3821920AE
:101468000AF061FD013D19200AF05DFD15F0FF0548
:10147800EAD110234FF020099C4DB361C6F81890AB
:101488002B681B0709D59A4BA6F828901B68984724
:10149800984BC6F8189001221A70974B9FED978ABF
:1014A8001B68974E1B7B00EE103AB8EEC00A20EE80
:1014B800080A08F02DF8338807EE903AF8EEE77A34
:1014C80027EE800A14F0AEFC8E4B9FED8F7A1880C1
:1014D80033888E4E07EE903AF8EEE77A8C4BC7EEDB
:1014E800277A3046FF211A229FED8A7AC7EE877A3B
:1014F8009FED897AC3ED007A884BD3ED047A884B47
:1015080067EE887A67EE877AC3ED007A14F07BFA83
:10151800002232702A68834B012112F0020F1970E1
:101528001FBF717003211970022118BFB1703046B6
:10153800560741BF19784D1C1D70032548BF4554F7
:1015480012F00A0F0CD01A7804218154511CC9B228
:1015580005254554D11C0232D2B219700621815496
:1015680039688D0641BF1A78551C1D70072548BF7C
:1015780085540A0608D51A7809258554951C013220
:10158800D2B21D700A258554674F7D79082D01D088
:101598000E2D04D11A78561C1E700B2686541A7804
:1015A80011F4803F4FF00C0E00F802E002F1010642
:1015B8001CBFDFF870E10232F6B21E701FBF8EF852
:1015C8000020524A4FF00E0E02F806E04A0741BFCB
:1015D8001A78561C1E70102648BF86541A78561C56
:1015E800F6B24FF0120E11F4806F1E7000F802E090
:1015F8000ED097F80CE2BEF1000F09D0DFF824E115
:1016080002328EF80020414A4FF0130E02F806E02D
:101618001A7811F4007F4FF0140E00F802E002F17E
:1016280001061CBFDFF8FCE00232F6B21E701FBFD5
:101638008EF80020354A4FF0150E02F806E0182DF6
:101648000DD11A7816268654561CF6B24FF0170E8E
:1016580000F806E0D61C0232D2B21E7085540A0386
:1016680041BF1A78511C1970192348BF83540021AF
:1016780098222E4814F0C7F90EF01FFE2C4B2D4A65
:101688002D491A6000234B800B712C490A60B7F86A
:10169800982190B22A4921F813000133122BF9D16D
:1016A800284B196811F0080F994600F0128197F835
:1016B8009231062B00F20781DFE803F004046B95F2
:1016C800ACC8C8002049214A0A60012B204D214896
:1016D800214943D103262E7007250B7005700C2372
:1016E80043E000BFA42F0020000400486C14002031
:1016F800D0060020E8060020DC08002035FA8E3CE1
:1017080016000020F80800200AE81C41E511002016
:101718001808002000401C46BD378635902C002054
:10172800D8080020E4110020A02400206022002016
:10173800EC0F00202A260020C82C0020E42E0020D0
:101748007C24002040240020B4060020382F0020EC
:10175800B0060020B80600207515002002232B7063
:101768000323037000230B70072313707F4B804AF9
:101778001A6040200AF09CFA002800F0A480012397
:101788004FF0000B90F900007A4A8DE808084021D4
:101798003DE007EE902ADFED786AB8EEE77ADFEDF4
:1017A800777AE7EE267A0023FCEEE77A744A17EE9A
:1017B800901A42F823100133122BF7D16B4A714962
:1017C8001160714A402013700AF072FA00287AD02A
:1017D80001234FF0070A90F900006C4A8DE80804CD
:1017E80040216B4B69E0614B6A4A1A60664B1022D4
:1017F80040201A700AF05CFA002864D001234FF0E8
:10180800000C90F90000644A8DE8081040214FF45C
:10181800E13352E0554B614A1A605B4B0822402085
:101828001A700AF045FA00284DD001234FF0000E37
:1018380090F900005A4A8DE8084040214FF4E133FE
:101848000AF07BFB574BC3F8B00138E04E49DFF88C
:1018580084C1DFF884E1544E544D55480C22062BC0
:101868000A700ED000238CF800308EF800303370E8
:101878001B232B704F4B027005221A704FF4E13571
:101888000BE000218CF800108EF800103170027007
:101898002121484A2970484D1370344B474A1A6031
:1018A80040200AF005FA70B101230026444A90F955
:1018B800000040218DE848002B460AF03EFB00302E
:1018C80018BF012028B9082007F0E6FE274B0022A0
:1018D8001A60D9F800302C4A13F4804F1FBF082132
:1018E80011702249374818BF086042F201011940B7
:1018F80003F0010003F4005541B11C49324E0E605B
:101908000DB10821117008B10C2111701178180659
:10191800A1F10401517040F19B802248DFF8BCA07E
:101928002A4EC0F8B46100252946152200F5DC705E
:10193800DFF8ACB08AF80150CAF80450CAF8085069
:10194800053E14F060F82846CBF8006004F0F0FF7C
:101958001F4B02201B68CAF80C300AF0A9F90028AE
:1019680040D1802007F098FE6AE000BF342F0020A5
:1019780085780008AD790008CDCCCC3F0000B0C414
:10198800842E002025210108382F00203522010847
:10199800A0860100C5780008C9210108AD780008B3
:1019A800F979000880010020101600201216002086
:1019B800731500201316002090D00300CD7700087F
:1019C800D9780008592101086521010888260020D6
:1019D8006424002074150020111600202C08002013
:1019E8004C08002045799AF80130C6490C2202FBC0
:1019F80003125278AA4204D00133DBB2042BF4D983
:101A080000238AF80130DBF800309AF801201B78AF
:101A180090F90000002B4FF00C0303FB021314BFD6
:101A28000325012500225B780095019202210AF026
:101A380084FAB54B1860002893D0012004F078FF91
:101A4800B24B1868B24B00F5C5721A6005F01EF863
:101A5800B04AB14B1360B14AB14E80331360D9F824
:101A680000300025D903357040F1AF800DF084F8BF
:101A7800DFF80CC3DFF80CB3CDF814C040F22A33FA
:101A88004FF0010A1A4660462946049386F800A0DA
:101A980013F0B9FFDBF81420A24E4FF0904042F447
:101AA8000032CBF81420026A22F070620262026AE5
:101AB80042F080720262032140220C928DF83510A8
:101AC80002220CA98DF8342003928DF836508DF837
:101AD80037A006F03FFBDBF81810039A41F40031F9
:101AE800CBF81810318821F440710904090C3180B1
:101AF8001D21F162304632850EA935866022C6F86E
:101B080014A00E92ADF83E501095ADF84450ADF8C3
:101B18004650ADF84850ADF84A50ADF83CA006F034
:101B28006DF9B26942F00802B261726C42F4004287
:101B38007264DBF8142042EA0A02CBF81420ABF5F1
:101B48007D6B584606F0CDF81AA806F09FF8049B5E
:101B5800ADF874308023744A1F934FF48073DDF816
:101B680014C01A921AA91022209358464FF4005311
:101B7800CDF86CC01C9223931E952195229524952F
:101B880006F091F8F36843F40073F360DBF8003073
:101B980043F00203CBF800300BA80D238DF82C304E
:101BA8008DF82DA08DF82E508DF82FA00EF08EFFF9
:101BB80029465E4B1A685E4B43F8212001312029E3
:101BC800F7D102F045FE02F043FED9F800305A057D
:101BD80055D5584D584BD5F8F8A4C3F800A00420A3
:101BE8000AF066F80421C5F8FC040AF03DF8534BE6
:101BF80085F800050820C3F800A00AF059F8082164
:101C0800C5F804050AF030F84D4E85F8080500219E
:101C180030462C2213F0F7FE8E227C2372704FF090
:101C28007D0BE0223370F27086F82BB0454E03939B
:101C38002C220021304613F0E6FE039B33708A23E2
:101C480073701020A023F37086F82BB0C5F80CA58C
:101C58000AF02EF81021C5F810050AF005F885F8E5
:101C680014052020C5F818A50AF022F82021C5F887
:101C78001C0509F0F9FF85F8200508F095FBD9F84F
:101C88000030314A13F4002318BF012313700AF0FF
:101C980025F92E4B18607B79052B02BF2C4B4FF48E
:101CA800C8721A802B4B4FF47A721A802A4BC822BA
:101CB8001A802A4A137843F008031370284A1378C5
:101CC80023F002031370D9F8002040F602031340F2
:101CD8006BB1244B24491960244B03211970244B00
:101CE80001211970234900230B8023490B8093039A
:101CF80041BF224B04221A71DA7848BF42F0010230
:101D080042E000BFF47D01087C1A00201C1200206C
:101D180048100020C81A0020BC260020C01A002045
:101D2800090F00200044014034440140B87D0108F7
:101D38000A0F00208001002060140020B814002041
:101D480088140020BD140020D02C00201809002081
:101D5800FE0F0020C62F0020C42F00207014002082
:101D6800CF2F0020581400201C260020BC1400206F
:101D780001010020A80F0020AA0F0020801A0020CF
:101D88004D0300200010024048BFDA70A368C9F86C
:101D98000030244B01221A7098F8003063F07F035A
:101DA80088F800302FB0BDEC028BBDE8F08F042519
:101DB800FFF75CBABAF1010F7FF6FEAA9A46FFF761
:101DC80097BA1BB207EE903ADFED176AB4F95E31A5
:101DD800164AF8EEE77A07EE103A67EEA67AB4F9F3
:101DE8006031CDED1A7A07EE903AB8EEC77AF8EE80
:101DF800E77A002127EE267A67EEA67A11701AA8EC
:101E08000B498DED1B7ACDED1C7A07F089FBFFF7A6
:101E180052B8BAF1010F7FF6CFAA4FF0000A30701E
:101E2800FFF771BA080F002035FA8E3C4A000020EF
:101E3800581600202DE9F04FC14BB3F90610C14BDD
:101E48002DED028B1F687A8985B0914201930EDBD4
:101E5800B1F5FA6FFC79BDBF8B1A6343A2F5FA643A
:101E6800C4F16404BCBF93FBF4F4643400E064245C
:101E7800B54BB64AB3F898B193F962311268029239
:101E88009BB2154603930022AD4B33F912E0CBEB1E
:101E98000E0303F2F31640F2E63086424FEA420C94
:101EA80003D8002BB8BF5B4201E04FF4FA73022A53
:101EB8002ED0029E96F811611EB1B342CCBF9B1B77
:101EC8000023A34E6FF0630A642093FBF0F836F802
:101ED80018900AFB083A08F1010836F918600FFA59
:101EE80089F8C8EB060606FB0AF696FBF0F6994851
:101EF8004E4420F80C60BE18642036797343964E21
:101F080093FBF6F364339BB2634393FBF0F02DE04D
:101F1800029890F812611EB1B342CCBF9B1B0023FC
:101F2800DFF860926FF06308642093FBF0F008FB21
:101F3800003A39F910600130002B39F91000A0EB94
:101F4800060000FB0AFABDF80C009AFBF8FAC6EB8B
:101F58000A0A1AFB00FA7F48A0F804A0B879B8BFAB
:101F68005B4243437C4893FBF0F064306B787B4ED4
:101F78004FF06408434393FBF8F3B354784EEB7A7D
:101F8800434393FBF8F3B3546B7D724E5843754B40
:101F980090FBF8F0022A9854734B0ED1DE4583F873
:101FA80002800DDB684CB4F89A21914214DBB1F53C
:101FB800FA6FA8BF4FF4FA610FE0DE459C5404DACB
:101FC80036F80C305B4226F80C300132032A05F152
:101FD80001057FF459AFE5E71146DFF8BCE15D4D37
:101FE800891A4FF47A736FF063075943C2F5FA629E
:101FF8006423B1FBF2F191FBF3F23EF8120007FB08
:102008000211013207B23EF91220D21B514391FB53
:10201800F3F30344F380554B1B885F0635D5544BC7
:10202800544A1B881288DFED547A9B1A1BB208EEBB
:10203800103AB8EEC88A28EE278AB0EE480A07F0A8
:1020480067FAF0EE408AB0EE480A07F0FEF9B5F9F3
:10205800023006EE903AB5F90030F8EEE66A07EE7F
:10206800903A20EE667AF8EEE77AA7EEA87A67EE5D
:10207800807ABDEEC77AE6EEA87A17EE103AFDEE42
:10208800E77A2B8017EE903A6B803C4D2B689807C7
:1020980040F1A1803A4B3B4F1A687B6945F2072112
:1020A800D31A8B4240F397807A6106F069F9364B70
:1020B800DFF8E8901A78032A9846B9F8003022D158
:1020C8000A2B2AD90023282088F8003009F02BFF92
:1020D80006F056F92D4B188806F03CF92C4B1A6877
:1020E800D37890FBF3F0013008282A4BA8BF0820CA
:1020F8001870537980B213FB00F33B83137913FBF9
:1021080000F0788309E00A2B07D80323214A88F8CE
:102118000030002313703B837B8398F800301A4A01
:10212800012B3DD002D3022B4CD054E03A8BB9F8A6
:1021380000309A424FDD012388F8003040E000BFAC
:102148007C24002040120020A02400201C12002023
:1021580096180020501400200CFEFFFF28180020BD
:102168009E0F0020401800208C17002030150020FA
:10217800481400204210002035FA8E3C40240020EC
:10218800B02F0020900F0020BC14002094160020CF
:1021980058140020010100207E1800205C14002043
:1021A800B9F800107B8B8B4202DD022313700FE01D
:1021B8009C4B1B8B0133994202DD002313700AE00C
:1021C800082006E07B8BB9F8002001339A42B2DC84
:1021D800072009F049FE2D68290575D5924B914FC6
:1021E8001A68FB69C3EB020845F2072398456BDDC3
:1021F800B6F90630FA61A3F57A7B8C4BB4F8520134
:10220800D3F800908A4E99F80A30012B4FF47A716E
:1022180098FBF1F803D040D3022B1FD03FE0854B49
:10222800386A5A7B844B33F812204FF0080E92B26A
:1022380090FBFEF3C01A8318BA843B6240F6E4426E
:1022480093FBFEF39BB25343B9F80820C2EB133358
:102258004B43B9F9062093FBF2F31FE0774BB9F82B
:1022680008A01B78C6F800A05A0718D50EF0C3FEC0
:1022780020B915F0100F18BF4FF0000BB9F9062060
:102288000BFB0BF1322391FBF3F35B445A434FF4FE
:102298007A7392FBF3F3534400E000233360D7E9E9
:1022A8000A013368664A03FB08F84FF47A7398FB0F
:1022B800F3F810EB080041EBE8710023C7E90A01C5
:1022C80010F0ECF85F4B18605F4E3368DB0427D5DD
:1022D8002F0622D55D4B1B789D071ED55C4B1878C1
:1022E80004281AD900225B4BD7180521951C4FF0FA
:1022F8000A0E122AD154E9B287F801E004D0B0EBF3
:10230800510F2A46EFD800E014215A18322002F85B
:10231800010CFF225A540F2000E00A2009F0A4FD06
:102328004D4D2A68002A44D04C4B4D4F18683968E7
:10233800814298463DD84B4BDFF834911878516864
:10234800B0B901221A70B9F80030CB5CD3B1464B52
:102358001A7010F063F8B9F800309BB92B681B7835
:10236800053B012B0ED809F0B9FD404B186009E078
:1023780000221A70B9F80030CB5C1BB13A4B1A70C6
:1023880010F04CF82A68B9F8003052683848D25C26
:10239800FE2A01D100230BE0FF2A02D109F052FDE9
:1023A80007E0D8F800500A2111FB02523A600133C5
:1023B8000380224D2B78580703D52E4B10221A85FF
:1023C80070E03268D1075CBF43F001032B701F4BEC
:1023D8001B781F075EBF2B7823F001032B70D602F2
:1023E80048BF2B78204A44BF23F001032B70224BAF
:1023F8001B6813F0040F02D02049098851B92049FD
:10240800098809B1980705D41E4B1B88003318BFEB
:102418000123CBB3022313702B7823F001032B7015
:1024280037E000BF900F0020B02F00205814002084
:10243800641400207C1600208C160020CF2F00206A
:10244800407E050068140020E01100207014002070
:1024580076140020DC210020B0180020642400201D
:10246800A8180020A41800209E2F0020742E0020F9
:10247800AC180020000400486C140020C42F002071
:10248800FE0F0020C62F00202978C90758BF022355
:10249800137009F023FDAF4B1B68C01A002801DB3D
:1024A8000FF0BCFF07F080FFAB4B1E789846002E5C
:1024B80000F0A980A94E3368002B00F0D28630685E
:1024C80009F0C4FE002800F0CC86A44BA44C186880
:1024D80009F0B9FE092801D03F2850D14FF0000A71
:1024E800D4F800909F4D5746B9F1000F05D09E488B
:1024F80029684A4613F0D4FA10B9AA4607B92F46F4
:102508009A4B10359D42EFD3C7B1D7F800E0DAF8FF
:1025180000C023681EF803501CF80300A8420DD120
:102528005A1C914938B92D2B05D88D4D2A60202584
:10253800CD54885402E0CD542260EAE723680BB1F9
:10254800574511D08A480DF089FA574507D857F8EA
:10255800100B0DF083FA09200DF078FAF5E785489D
:102568000DF07CFA4FF0000923689945A7D27E4BFD
:1025780013F809000DF06AFA09F10109F4E7236874
:10258800002B40F05286042840F0948676480AF0E2
:1025980013FA00F066BED9F80000DFF8E8A109F0E8
:1025A80055FE30B3DAF8000009F04DFEDBF80030D4
:1025B80093F848100246002933D124286AD1012211
:1025C80083F84820DBF80030DFF8B4A193F84820FE
:1025D800062AE0D193F8490002F018FC8346002847
:1025E8007BD03B6898790DF082F93B68002283F82C
:1025F8004820614B93F83530002B40F004864C3668
:10260800982E00F02E865D4BF21892F84A10012998
:10261800F5D15B4FF3583A605A4ABB46136091466E
:10262800B9E7012904D14D2814BF00220222C7E7C7
:10263800022904D13C2814BF00220322C0E7032941
:102648000CD140284FF0000102D983F84810B9E7AF
:1026580058711971D97198710422B1E7042906D10A
:10266800997983F849004A409A710522A8E7052913
:10267800A8D1587919798842987906D95040987123
:10268800481C18710B441A729CE790420CBF062232
:10269800002295E72B78580794D4232ADAF80030DB
:1026A8000ED1012188F800102C4937480B603249B7
:1026B80002920B630DF0D2F92E480DF0CFF9029A71
:1026C800324B1B681B78934201BF314B314A1A6069
:1026D800314B04BF314ADA6074E7DAF8002092F827
:1026E80049304C2B00F0968400F28580332B00F0A3
:1026F800CC8421D8292B00F0598409D8252B00F047
:102708001384272B00F01784232B40F0CF8539E260
:102718002D2B00F05C8407D82B2B40F0C7850DF0DB
:10272800C9F8607100F06ABD2F2B00F01A85312BB3
:1027380000F02C8500F0BABD3E2B00F0198144D87A
:10274800372B00F0D6842BD8352B00F06F8200F0A1
:10275800ADBD00BFA02F0020D02F0020CC2100202D
:10276800BC1A0020808101088C1A002030830108DF
:10277800D7A10108DCA10108900F002060220020E9
:1027880010150020141500200CA20108FC220020BE
:10279800FC9F0020EFBEADDE00ED00E00400FA056E
:1027A800392B00F0D5833C2B40F08085DFF84C9422
:1027B800D9F800A00DF07EF88AF80000D9F80030AA
:1027C800187809F081FF00F019BD432B00F06E84E2
:1027D80006D8412B40F06A854FF0000900F05ABC3A
:1027E800442B00F007854A2B40F060850DF06CF80B
:1027F800A08100F003BDD02B00F00F8355D8CA2B61
:1028080000F0C08009D8C82B00F0858000F226832C
:102818004E2B00F00C8400F049BDCD2B00F008834E
:1028280004D8CC2B00F02A8200F040BDCE2B00F05B
:102838000883CF2B40F03A850DF046F86FF4AF626D
:1028480083189BB2C62B98BFA4F898010DF03CF8EA
:10285800A4F844010DF038F8A4F846010DF034F856
:10286800A4F848010DF030F8A4F8D2010DF022F8D0
:1028780084F8E3010DF01EF80DF01CF884F8E4016B
:102888000DF018F884F887010DF014F884F8940115
:102898000DF010F8D94BD3F800900DF015F800EBB7
:1028A80080004000A9F8560052E3D62B00F0398288
:1028B8000AD8D22B19D0C0F0F882D32B25D0D42B2C
:1028C80000F03B8200F0F2BCEF2B41D005D8D82BAA
:1028D80040F0EC844FF0000AE6E0F22B00F075823D
:1028E800FA2B00F0B78200F0E1BC2B78590700F111
:1028F80085840CF0DFFF022884F8A40740F2938255
:10290800BF4B002283F8A4278DE20CF0DDFFBD4BFE
:10291800188000F073BC92F805904FEA5909B9F194
:10292800120F03D90DF066FD00F068BC4FF0000AE5
:10293800CA4507D20CF0C8FFB34B23F81A000AF1B6
:10294800010AF5E7B14B012283F8342000F056BCA8
:10295800DFF8A892D9F800A00CF0B6FFAAF85A0040
:10296800D9F800900CF0B0FFA9F8580000F046BC68
:102978000CF0A0FF84F8D6010CF09CFF84F8D50178
:1029880000F03CBC9D4B1A681278022A8246994690
:102998006FD1D9F800B00CF08DFF07EE900AF8EE71
:1029A800677AB2EE048AC7EE887A0BEB8A0BCBED16
:1029B800087AD9F800B00CF07DFF07EE900A9FED79
:1029C800947AF8EE677A0BEB8A0BC7EE877ACBED31
:1029D8000B7AD9F800B00CF06DFF07EE900A9FED66
:1029E8008D7AF8EE677A0BEB8A0BC7EE877A0AF1D5
:1029F800010ABAF1030FCBED0E7ACAD1BAF1070F6B
:102A0800D9F800B01CD10CF055FF07EE900AF8EE8B
:102A1800677AC7EE887ACBED117AD9F800B00CF056
:102A280049FF07EE900AF8EE677AC7EE887ACBED91
:102A3800127AD9F800B00CF03DFF8BF84C0012E088
:102A48000CF038FFD3448BF80100D9F800B00CF033
:102A580031FFD3448BF80B00D9F800B00CF02AFFF3
:102A6800D3448BF815000AF1010ABAF10A0FC5D14F
:102A7800C4E3D9F800B00CF01DFFD3448BF8010073
:102A8800D9F800B00CF016FFD3448BF80B00D9F836
:102A980000B00CF00FFFD3440AF1010ABAF10A0F93
:102AA8008BF81500E5D1A9E3DFF850919FED598A1D
:102AB800D9F800B00CF008FF07EE900AF8EE677A34
:102AC8000BEB8A0BC7EE887ACBED087AD9F800B001
:102AD8000CF0FAFE07EE900AF8EE677A0BEB8A0B19
:102AE800C7EE887ACBED0B7AD9F800B00CF0ECFE83
:102AF80007EE900AF8EE677A0BEB8A0BC7EE887A36
:102B08000AF1010ABAF1030FCBED0E7ACCD1BAF172
:102B1800070FD9F800B01CD10CF0D6FE07EE900ACA
:102B2800F8EE677AC7EE887ACBED117AD9F800B05B
:102B38000CF0CAFE07EE900AF8EE677AC7EE887ABC
:102B4800CBED127AD9F800B00CF0BEFE8BF84C0031
:102B580012E00CF0B9FED3448BF80100D9F800B0AC
:102B68000CF0B2FED3448BF80B00D9F800B00CF08F
:102B7800ABFED3448BF815000AF1010ABAF10A0F2B
:102B8800C5D13BE30CF096FE132883463FF6CAAE48
:102B9800DFF868A0DAF800900CF08CFE00231E4ADB
:102BA8000C2101FB0322117A814222D10FFA8BFBFF
:102BB80009EB8B09137889F879300CF07BFE89F8DA
:102BC8007A000CF077FE89F87B000CF073FE134B4B
:102BD800134A1A6089F87C00124BDAF80000186072
:102BE8000021793009F0F4F80F4B80F001001870DB
:102BF80004E301331B2BD2D194E600BF1C12002042
:102C0800A0240020401000207C240020900F0020E9
:102C18000000C84200007A44A47F01083810002050
:102C2800E42500203C100020140000200CF042FE97
:102C38000B2882463FF676AECE4BD3F800900CF0C8
:102C480039FE03283FF66EAE062303FB0A9989F87E
:102C5800CE000CF02FFE89F8C9000CF02BFE89F885
:102C6800CA000CF027FE89F8CB000CF023FE89F887
:102C7800CC000CF01FFE89F8CD00BFE25379092B78
:102C88007FF650AE019BD3F800900CF013FE019B29
:102C980089F80000D3F800900CF00CFE89F80100C8
:102CA8000CF008FE019B64281B68A8BF64201871FB
:102CB8000CF000FE019B64281B68A8BF64205871B3
:102CC8000CF0F8FD019BFF281B68A8BFFF20987136
:102CD8000CF0F0FD019B6428D3F8009028BF642015
:102CE80089F807000CF0E6FD019B89F80200D3F88B
:102CF80000900CF0DFFD019B89F80300D3F80090E9
:102D08000CF0E2FD3B68A9F80A005B790A2B40F257
:102D18007582994BD3F800900CF0CCFD89F8080027
:102D28006CE282460CF0D0FD944B23F81A000AF1AD
:102D3800010ABAF1080FF5D160E253790F2B7FF43D
:102D4800F1AD0CF0B7FD072881463FF6EBADDFF893
:102D580024A2DAF800B00CF0B7FD0E2303FB09F942
:102D6800CB44ABF81901DAF800B00CF0ADFDCB4458
:102D7800ABF81B01DAF800B00CF0A6FDCB44ABF8B9
:102D88001D01DAF800B00CF095FDCB448BF81F015B
:102D9800DAF800B00CF08EFDCB448BF82001DAF89D
:102DA80000B00CF087FDCB448BF82101DAF800B0B5
:102DB8000CF080FDCB44DAF800A08BF822010CF06F
:102DC8008DFDD144C9F8230118E20CF073FD0F28DA
:102DD80081463FF6A7AD0CF06DFDC9EBC909A144CA
:102DE80089F8D4000CF066FD89F8D5000CF062FD76
:102DF80089F8D6000CF05EFD89F8D7000CF05AFD72
:102E080089F8D8000CF056FD89F8D9000CF052FD6D
:102E180089F8DA0009F0BCFBF0E12B785B0700F1D8
:102E2800ED810EF023F906F069FC06F021FDE5E1DD
:102E38002B78580700F1E281514B4FF4C8721A8081
:102E4800DCE12B78590700F1D9814E4A137843F019
:102E5800040328E02B785A07E5D527E20CF02AFD71
:102E6800484B1A7810B142F0020201E022F0020247
:102E78001A700CF01FFD444BDFF82C9118700CF001
:102E88002DFDC9F800000CF029FDC9F804000CF06C
:102E98001BFD3E4B18800CF017FD3D4B3D4A18803A
:102EA800137843F002031370A8E10CF003FD0290BD
:102EB8000CF014FD83460CF011FD82460CF00EFD5B
:102EC80081460CF001FD0CF0FFFC0CF0F3FC029BBA
:102ED800A3B9314B1020C3F800B0C3F804A006F022
:102EE800BAFB284A137843F001031370B9F1000FB5
:102EF80000F08481294BC3F800907FE1102B40F04B
:102F08007D81274BC3F800B0C3F804A0B9F1000FC6
:102F180002D0224BC3F800902148224B0222011D07
:102F28001A7003F069FD69E1A0600CF0D7FCA36892
:102F38001843A06062E10CF0C7FCA4F85C010CF037
:102F4800C3FCA4F85E010CF0BFFCA4F8600155E1D5
:102F58000CF0B0FC84F87C010CF0ACFC84F8800127
:102F68000CF0A8FC84F87F010CF0A4FC84F8810123
:102F780044E100BF1C12002040120020B2210020B2
:102F8800FE0F002070140020761400207414002016
:102F98007214002046120020481200205812002007
:102FA8005012002044100020781400200CF08CFCF3
:102FB800A4F882010CF088FCA4F884010CF07AFCD7
:102FC80084F886010CF080FCA4F8880116E10CF066
:102FD80071FC84F892010CF077FCA4F89C010CF0C9
:102FE80073FCA4F898010CF06FFCA4F89A010CF09B
:102FF80061FCDAF8003084F893015B79082B40F221
:10300800FD800CF061FCA4F89E010CF05DFCA4F8B6
:10301800A001F3E00CF04EFC84F8D0010CF04AFC5F
:1030280084F8D1010CF050FCA4F8D201E6E092F843
:1030380005900323B9FBF3F9B9F10E0F3FF672AC13
:10304800DFF888A34FF0040BCB4580F0D7800CF055
:1030580031FC8AF8A2010CF037FC40F2ED239842CB
:1030680005DD40F6CA039842A8BF184601E040F2C1
:10307800EE20A0F2EE2019230BF1010B90FBF3F0E8
:103088000AF1020A8AF8A101DEE70CF013FC84F8C1
:103098009401B3E00CF00EFC04EB090309F10109FB
:1030A800B9F1080F83F88A01F4D1A7E00CF002FC0B
:1030B800C4F808B060710CF011FCA3681843A06054
:1030C8000CF0F8FB84F892010CF0FEFBA4F85C010C
:1030D8000CF0FAFBA4F85E010CF0F6FBA4F8600112
:1030E8000CF0F2FBA4F882010CF0EEFBA4F88401CA
:1030F80084E053794FF0070AB3FBFAF2C2EBC2023D
:103108009A1A12F0FF0F7FF40DACB3FBFAFA0AF12A
:10311800FF3A5FFA8AFABAF1FF0F6FD00CF0CAFBD8
:103128005FFA80FB4FFA8BF008F08AFD8146002891
:103138003FF4F8AB80F800B00CF0C6FBA9F8020029
:103148000CF0B8FB89F804000CF0B4FB89F8050012
:103158000CF0B0FB89F807000CF0ACFB89F806000E
:10316800D5E7DFF8689209F1400A0CF0ADFBA9F841
:103178009C020CF09FFB89F89E020CF09BFB09F166
:10318800040989F89B02D145EFD137E00CF092FB96
:103198001F2881463FF6C6AB3B685B79082B7FF456
:1031A800C1AB0CF091FB09F1860904EB890900F029
:1031B8003F00A9F806000CF087FBB9F8063080013B
:1031C80000F4FE501843A9F806000CF073FB000148
:1031D80089F804000CF06EFB99F8043000F00F0039
:1031E800184389F804000CF065FB89F805000BF01A
:1031F800C3FC03E0624B012283F8352000200CF069
:10320800A5FBFFF7EEB95F4B985909F016F818B906
:10321800322008F088FEF6E709F07AF906F044FA59
:10322800594B5A4ADA60FFF7EAB90C2844D00A2801
:103238004BD1574D57480CF011FC2846232112F06A
:1032480018FC08B1401B20602368002B60D150484F
:1032580023600021302212F0D6FB98F80030002BB2
:103268002DD14D4B1B689B0615D54C4B44491B680B
:103278008A6B9A1A002A0EDB494A1278042A0AD95C
:10328800484A03F5123303F5F8738B63938A9BB2AC
:1032980083F020039382444B9B68002B6BD04348F8
:1032A80005B0BDEC028BBDE8F04F18470DF0A2F851
:1032B800FFF797B90C2804D13D480CF0CFFB3D48E7
:1032C8000DE07F2812D1FFF7FAB80D28B1D07F287A
:1032D80009D1013B2E4A384823600021D1540CF013
:1032E800BDFBFFF7ECB82F2B3FF6E9A8A0F12002B1
:1032F800D2B25E2A3FF6E3A813B920283FF4DFA82C
:103308005A1C2260224AD0540CF0A0FBFFF7D7B811
:103318005A1EA95C202901D1134696E71C4A23604E
:103328000021D154254B264DD3F800A0D5F800B084
:10333800DFF85C90584612F0AAFB07463A46484622
:10334800594612F0ADFB1F4A28B919F80730534403
:103358005B785B0703D010359542E7D306E09542CA
:1033680004D2781CEB684844984702E016480CF0F1
:1033780075FB00236BE705B0BDEC028BBDE8F08F51
:10338800900F00206022002000ED00E00400FA0504
:103398008C1A002094B001086C140020B02F002073
:1033A8007614002000040048902C0020CC0F002048
:1033B800E1A10108DCA1010808A201081001002010
:1033C8008081010830830108ECA10108A0240020B5
:1033D8002DE9F04FAA4FAB4D3B68AB4CAB4E03F514
:1033E8009C4320332DED028B23602B8832680133F8
:1033F8002B8042F20103134087B01BB1A44A137813
:10340800013313700EF03AFF3368D80405D5A14B89
:103418001B68D90701D40EF04DFE9F4B3968186818
:10342800837AD3B1013B9D4F027B37F813301AB131
:10343800C3F53B6308339BB21BB2A3F57A73B3F5AC
:103448007A7FA8BF4FF47A7323EAE37307EE903AC2
:103458009FED937AF8EEE77A36E0326812043FD5AA
:103468006268DFF824E28A1A002A39DB01F59C42F7
:103478002032CEF804208B4AC07A57798A4A32F82B
:1034880017209EF80870013792B292FBF0F207F00D
:103498000F008EF80800704442721A468348185C80
:1034A80001330244102B92B2F8D112B292FBF3F31B
:1034B8001BB2642BA8BF642323EAE37307EE903A98
:1034C8009FED7B7AF8EEE77AC7EE877A794A9FED27
:1034D8007A7A67EE877AFCEEE77A17EE903A1380ED
:1034E8003368DF0540F19280744B994204D92B79F7
:1034F80013B9644B01221A71714AB5F900E01778C3
:10350800604BBEF1140FC7F38002CCBF4FF0000E22
:103518004FF0010E0192BEF1000F06D04FF00008E7
:1035280083F8068083F8058001E04FF003085B4AC2
:10353800A879D4F81CB0D4F820C0B5F900906979FE
:103548006B881288032856D8DFE800F0021222425E
:10355800BEF1000F03D051480280002236E00198E6
:10356800002840F0C0864D4802809DF804202DE0D8
:103578009CF8000000EB8000814503DC474802808E
:10358800012223E0019F0120002F34D000F017BF53
:10359800019850B14148BBF80E20428082803F4FCD
:1035A800BCF80200F8804FF002089CF800A09CF8D4
:1035B8000100504400EB8000814500F39786019894
:1035C800002800F09386354802800222AA7115E08F
:1035D80032486B80019B02800322AA7169717BB11A
:1035E800374A137843F002031370264B00225A71AE
:1035F8000EF060FD04E0294FA8713A8069716B8074
:10360800B8F1000F02D0404608F02EFC2D4FB7F855
:1036180052010DF0F0FC834668B90EF0A3FB2A4B6B
:10362800C3F800B0C3F804B0C3F808B0274B0022B1
:103638001A605A609A60224B1A7812F0040F984662
:1036480064D03368D80661D5214B1B78D9065DD480
:10365800204B1B78002B41D097F8D631BBF1000FD7
:1036680044D1002B3DD01C4B1A68636A9B1A002B6F
:1036780037DA0EF01FFD044B83F828B046E000BF90
:10368800B02F0020C82C0020D00F0020402400209C
:103698003B2F0020E0110020E42E00207C24002095
:1036A80000007A447C1600208C160020D90F0020D8
:1036B8000000C8423C12002000C07F44404B4C0030
:1036C800CF2F0020A0240020AC170020681800206D
:1036D800701400201400002064240020BBF1000FA7
:1036E8000CD1102008F0C0FB01230DE033B1914A42
:1036F80012684FF47A7101FB0323636294F828304F
:1037080023B108F09FFB002384F8283097F8D431C0
:10371800019397F8D511B7F89AE1B7F89CC100233F
:103728001846854A32F9132080087245C4BF60F0F4
:103738007F00C0B201336245B8BF40F04000042B9F
:10374800EFD194F829307D4A834205D192F82A3086
:10375800F92B04D8013300E0002382F82A30784B93
:1037680084F829001A78DFF8F0919A46EAB9D9F86E
:103778000030DA0709D5BBF1000F16D198F80030F0
:10378800DB0712D50EF00AFB0FE098F80030580757
:103798000BD56C4B1B7843B16B7933B911B10EF073
:1037A80089FC02E0BBF1000FF9D094F82A30634A93
:1037B800DFF8A8B1142B40F09080019B003318BFAC
:1037C800012301939AF8003073B392F829305F2BE4
:1037D80012D198F8003003F0040303F0FF0113B18D
:1037E8000EF068FC08E00B200391029208F03CFB05
:1037F800029A039982F82A10019BABB194F82930F8
:103808007D2B11D198F8003003F0040303F0FF0278
:1038180013B10EF04FFC07E00B20029208F024FBD6
:10382800464B029A83F82A2098F8003003F00403E4
:1038380003F0FF01002B50D194F829303F4A572B51
:1038480015D1414B4FF47A721A803368190601D5A5
:1038580003F07EF93D4B1B685A0742BF3C4A0A21D8
:10386800118013F0080338D13A4A138035E03068E4
:10387800400717D55A2B15D192F82B302BB10123BD
:1038880082F82B1082F82C3027E092F82D3083F044
:10389800010382F82D300BB10C2000E00D2008F058
:1038A800E3FA1AE05D2B00F024855B2B00F02385FA
:1038B8005E2B02D1032000F01FBD562B03D10293CB
:1038C80006F072F9029B9AF80020002A00F0288579
:1038D8006F2B40F020850EF061FA33685A074FD5F8
:1038E80094F82D30154A9BB198F800305B070FD536
:1038F800114BB3F90610B7F89A31994208DDD9F897
:10390800003013F0010302BF3221118682F82D30F6
:10391800D9F80030D80323D594F83220074B22B9C0
:1039280093F82B200AB932221A86012384F8323000
:1039380026E000BF642400207C240020D00F002053
:10394800140000203A2F0020C62F00206C140020FD
:10395800C42F002048140020E01100201C12002071
:1039680094F82B30B74A5BB198F8003003F00403A1
:1039780003F0FF0123B9012382F82B1082F82C30C1
:10398800DBF800800023C9F8003008F17B0708F154
:10399800CB0A3A787B7817F8010C9A420DD239464F
:1039A80008F0F0F948B117F8022C012303FA02F2E3
:1039B800D9F800301343C9F8003004375745E8D127
:1039C800A14B1B7853B1A14FDFF89C923B68DFF8FD
:1039D8009C8213F0020F40F03D8336E308F1CA07DA
:1039E80008F589783A787B7817F8010C9A4222D240
:1039F800394608F0C7F9F0B1BB7897F804E0944A63
:103A080097F803908F480C21013B01FB0E4103EB13
:103A1800430313448A6B9A420DD08B63002390F8BA
:103A28006420CB63012303FA0EF322EA030381F82F
:103A3800349080F8643006374745D3D1854BDFF89A
:103A480030A21F68844B1B680293844B1B78039336
:103A580000230193DAF80030002B00F0ED8293F890
:103A68000090B9F1000F00F0E782DAF8042002991B
:103A78008A1A002A0CDB01F5FA720199CAF80420A7
:103A880001228A4094F8641021EA020284F8642032
:103A9800039A002A00F0D0821AF8042C59780432CC
:103AA800D2B2002940F087826D4931F912106D4A6F
:103AB800B2F8982102F1C800814202DD93F802B001
:103AC80015E0C83A914203DA9978C1F1000B0EE08B
:103AD800019A0123934094F8642022EA030384F8AE
:103AE8006430029B03F5FA73CAF80430A4E294F830
:103AF8006430019A1341D90700F19E82BBF1000F8F
:103B0800CCBF0220012008F0D1F909F1FF33DFF81A
:103B18003481132B00F28882DFE813F014002500AB
:103B280037004B0064006B00F1005401BB01EB014E
:103B38001B0286024B005A006B00F1005401C100C1
:103B480026018B0197F80080D844B8F1FA0FA8BF76
:103B58004FF0FA0828EAE878384687F8008008F035
:103B6800F7F801200FE097F80180D844B8F1640F06
:103B7800A8BF4FF0640828EAE878384687F801803B
:103B880008F0E6F802204146E0E197F80390D944AE
:103B9800B9F1640FA8BF4FF0640929EAE97987F8F9
:103BA80003903846D8F8681008F088F8032049468A
:103BB800CCE1797959446429A8BF642121EAE171EB
:103BC80079710D2008F02AF9B9F10D0F00F02C8257
:103BD800397959446429A8BF642121EAE17139710E
:103BE8000E20B3E1B979594481F30801B971052070
:103BF800ACE1D8F86C301A78022A41D107EE90BAB5
:103C0800F8EEE77AB2EE040A87EE800AD3ED097A75
:103C180030EE270AB5EEC00AF1EE10FA09D4DFED4E
:103C2800167AB4EE670AF1EE10FAC8BFB0EE670A6A
:103C380001E09FED120A83ED090A0F2008F0D9F878
:103C480029E000BFD00F0020D02F0020E011002075
:103C5800387F010840120020642400203A2F0020F9
:103C68007C240020A02400206C14002030150020A3
:103C78000810002000007A440000C842000000003C
:103C880099785944C829A8BFC82121EAE1719970D7
:103C98000F2008F0C3F8B9F10F0F00F0C581D8F86C
:103CA8006C301A78022A20D107EE90BAB8EEE78A6B
:103CB800B2EE040A88EE008A93ED080A38EE000A8C
:103CC800B5EEC00AF1EE10FA09D45FED157AB4EE3C
:103CD800670AF1EE10FAC8BFB0EE670A01E01FEDFF
:103CE800190A83ED080A122058E159785944C8295D
:103CF800A8BFC82121EAE1715970122026E1D8F83D
:103D08006C301A78022A20D107EE90BAB8EEE70A8A
:103D18005FED277A93ED0C7A80EE270A30EE070ADA
:103D2800B5EEC00AF1EE10FA07D4B4EE670AF1EE68
:103D380010FAC8BFB0EE670A01E01FED300A83ED44
:103D48000C0A102008F055F80AE0197B5944C829D4
:103D5800A8BFC82121EAE1711973102008F05EF8A4
:103D6800B9F1100F00F06081D8F86C301A78022A87
:103D78001ED107EE90BAB8EEE78A5FED417A93ED6F
:103D88000B0A88EE278A38EE000AB5EEC00AF1EE73
:103D980010FA07D4B4EE670AF1EE10FAC8BFB0EE15
:103DA800670A01E01FED4B0A83ED0B0A1320F5E0CB
:103DB800D97A5944C829A8BFC82121EAE171D97222
:103DC8001320C3E0D8F86C301A78022A22D107EE03
:103DD80090BA1FED580AF8EEE77A87EE800AD3ED1D
:103DE8000F7A30EE270AB5EEC00AF1EE10FA09D4C0
:103DF8005FED5F7AB4EE670AF1EE10FAC8BFB0EE75
:103E0800670A01E01FED630A83ED0F0A112007F02E
:103E1800F0FF0AE0997D5944C829A8BFC82121EAC2
:103E2800E1719975112007F0F9FFB9F1110F00F050
:103E3800FB80D8F86C301A78022A20D107EE90BAA5
:103E48001FED740AB8EEE78A88EE008A93ED0E0A31
:103E580038EE000AB5EEC00AF1EE10FA09D45FEDAB
:103E68007A7AB4EE670AF1EE10FAC8BFB0EE670AC4
:103E780001E01FED7E0A83ED0E0A14208EE0597DC5
:103E88005944C829A8BFC82121EAE17159751420ED
:103E98005CE0D8F86C301A78022A20D107EE90BA84
:103EA800B8EEE78AB2EE040A88EE008A93ED0A0AB1
:103EB80038EE000AB5EEC00AF1EE10FA09D45FED4B
:103EC800927AB4EE670AF1EE10FAC8BFB0EE670A4C
:103ED80001E01FED960A83ED0A0A09205EE0D97811
:103EE8005944C829A8BFC82121EAE171D97009201D
:103EF8002CE0D8F86C301A78022A1ED107EE90BA56
:103F0800B8EEE78A5FEDA47A93ED0D0A88EE278A6A
:103F180038EE000AB5EEC00AF1EE10FA07D4B4EE96
:103F2800670AF1EE10FAC8BFB0EE670A01E01FEDAC
:103F3800AD0A83ED0D0A0A2030E0597B5944C8299F
:103F4800A8BFC82121EAE17159730A2007F066FF6A
:103F58006AE0D8F86C301A78022A22D107EE90BAB3
:103F68001FEDBC0AB8EEE78A88EE008A93ED100AC6
:103F780038EE000AB5EEC00AF1EE10FA09D45FED8A
:103F8800C27AB4EE670AF1EE10FAC8BFB0EE670A5B
:103F980001E01FEDC60A83ED100A0B2007F029FF88
:103FA80042E0D97D5944C829A8BFC82121EAE17156
:103FB800D9750B20CAE7012936D19878B44B33F963
:103FC8001230B3F5617F05DB40F633029342A8BF98
:103FD800134601E04FF46173B9F10C0F24D14FF48B
:103FE800966292FBF0F0AB4AA3F5617393FBF0F392
:103FF8005FFA83F81378434516D0B8F1040F34BF3D
:10400800434602231370A44A09FB0323A34A063339
:10401800136005F009FC4846414607F0FFFE08F129
:104028000100C0B207F042FF019A0123934094F8BF
:104038006420134384F86430019B0133042B0193FB
:104048000AF10C0A7FF406ADBDE43368DA0510D531
:104058006B7973B1D9F800309B070AD5B8F80030EE
:1040680013F001050AD10DF07DFE012005F004FBD7
:1040780004E0012005F0EFFA012300E000233A688C
:1040880055070DD563B1012005F0E5FAB8F8003001
:10409800980708D40DF066FE022005F0EDFA02E05C
:1040A800022005F0D8FAB8F800307D4A13F0030F63
:1040B8004FF020010CBF91611185D9F8002012F052
:1040C8000A0F24D03A68D10609D55A070AD4042021
:1040D80005F0D2FA734B1B88A4F8703002E0042074
:1040E80005F0B9FA3B689B0607D5B8F800305D06BD
:1040F80006D4402005F0C0FA02E0402005F0ABFAF3
:104108003B68580642BF674B1B88A4F87230D9F841
:104118000030990608D43B681A0540F18E804FF4A8
:10412800807005F0A9FA8CE05F4B1B789B0750D58F
:104138005E4B1B78042B4CD93B6813F400790FD0E5
:10414800B8F80030DD0638D4102005F095FA2020A4
:1041580005F081FA5648011D02F04EFC022328E0C2
:10416800B8F8005005F01005ADB22DB1102005F0DB
:1041780072FA012584F874903B68580511D5A36F2D
:104188004C495A89B1F90030002BB8BF5B429342C1
:1041980007DAB1F90230002BB8BF5B429342C0F294
:1041A8001481B8F80030990608D5202005F053FA94
:1041B800002384F87430012500E0002594F87C3051
:1041C800BBB90E2007F050FE3B4B012283F87C2040
:1041D8000FE0B8F8003003F03003002B9BD010201C
:1041E80005F039FA202005F036FA002384F87430F7
:1041F80001E0002D8FD0314B002003F1280503F199
:1042080050042F4A002122F810102E4A596022F833
:1042180010100432696022F8101000221A609A60A7
:104228002A60AA6022606160A260143314351434D5
:1042380000287FF470AF0120E3E74FF4807005F0A9
:104248000AFA214B5A79082A1C4601D00E2A02D1B3
:10425800402005F000FA33685A0540F1CC8094F804
:104268000C3223B9194B1B7813F0040F02E03B689A
:1042780013F4002F2ED0164B00221A703C200CF09D
:10428800BDF8002800F0B7800BF0F4FAF6E700BF9D
:104298007C240020B0210020402C00204012002067
:1042A80000040048481400207014002076140020F0
:1042B8004812002050140020D00F00205010002079
:1042C800C82F0020C8100020A0240020CF2F0020D5
:1042D800F822002006F068F807B0BDEC028BBDE8B4
:1042E800F04F0BF0EABF0120FFF72CB90320FFF7CE
:1042F80029B9012000E002205FFA80FA0AF1FF33B1
:1043080087F8A43705F0FAF905F0B2FA504607F035
:10431800CDFDFFF7E2BA019A12B17E2B3FF4DBAA7A
:10432800972B04D14FF4C873E385FFF7D6BAA72BB0
:1043380006D1334A137843F004031370FFF7CDBA5C
:104348000022BB2B059201D1022303E0B72B04D135
:104358004FF6FE73ADF8163009E0BE2B01D10223EB
:1043680003E0BD2B1AD14FF6FE73ADF81430DBF81D
:104378000020BDF81410B2F858300B44A2F8583099
:10438800BDF81610B2F85A300B44A2F85A3005F0AE
:104398000BFC002384F82A30FFF79FBA792B04D14D
:1043A800184AD37823F0010306E07A2B7FF495AA04
:1043B800144AD37843F00103D370FFF78EBA013360
:1043C80001469BB20220FFF7BDB8B8F800309B0643
:1043D8003FF5F4AE202005F04FF90B480B4B011DBB
:1043E8001A685B684360026002F006FB084B01250F
:1043F80083F87450E2E607B0BDEC028BBDE8F08F9D
:1044080070140020801A0020501200207814002018
:10441800D00F002010F80A3C0133DBB20A2B84BF0E
:1044280010F8131C044A00F80A3C82BF002322F843
:10443800113000F80A3C7047CC2E0020354A70B580
:10444800136C90681944344B1B78D940081A40F60D
:104458008C2398429160D060516013463BD9127802
:1044680093F945108A4210460BD1111F082908D824
:1044780093F84610182901D8013103E083F8442045
:1044880002E0002183F8461093F944402149A242F2
:1044980019D191F84740B4B10C310024944206DA9E
:1044A8001E4D51F8046F25F814600134F6E70C2806
:1044B80005D01A49002421F810400130F7E71848C0
:1044C80001780131017083F84520002201211A701A
:1044D80083F8471070BD92F84710C9B1A0F2EF24D5
:1044E80040F2DA518C4208D811780B2905D80B1DF7
:1044F8000131117042F8230070BD002283F8472073
:10450800084B03F13002002143F8041F9342FAD10B
:1045180070BD00BFA8010020A7010020CC2E0020FC
:10452800B9060020B4010020024A136C0133194473
:1045380011647047A8010020024B53F820301B6813
:1045480019607047F4180020064B53F820301A6899
:104558001B89A1F57A7159434FF47A7391FBF3F1F2
:1045680011607047F4180020054B98420CBF054AAB
:10457800054A138801339BB213800020704700BF9F
:1045880000540040DC110020DE110020F0B5046D5D
:104598008668236823F0010323608379054613F0B6
:1045A800020F40790CBF4FF0000E4FF4005E13F07D
:1045B800040F14BF4FF48067002710F0010F14BFD9
:1045C800042100218307206820F001002060626830
:1045D80022F440524EEA02026260226822F4B0538A
:1045E80023F00C0348BF41F008013B430B43236011
:1045F800A36895B023F44073A360684603F03CFCBD
:10460800284B9C4201D10C9B0EE0274B9C4201D1C8
:104618000D9B09E0254B9C4201D10E9B04E0244BE5
:104628009C420CBF0F9B109B2268A879170448BFB7
:104638005B00B3FBF6F206FB1233B3EB560F2368AD
:1046480028BF01321E0441BF4FF6F073C2F3420186
:10465800134041EA03026B7992B213F0020FA28170
:1046680000F0010114BF4FF400320022DC0748BFFC
:1046780042F480322B6D11B159680A4302E059683F
:1046880021EA02025A609A6801074CBF42F0080208
:1046980022F008029A601A6842F001021A6015B006
:1046A800F0BD00BF00380140004400400048004011
:1046B800004C00403D4B1B78012B30B514BF002443
:1046C8000324B1B9036A23F0010303628169036A11
:1046D80021F0F30123F00A0341F0010142F0010245
:1046E8001A4341EA041181610262836923F00C03D1
:1046F8001BE004291DD1016A4FF6EF730B400362DA
:104708008169056A120121F473414FF65F7342F023
:10471800100241F480712B4092B2134341EA0431F4
:1047280081610362836923F44063836183698361E0
:1047380030BD0829016A1AD14FF6FF630B400362A6
:10474800C169036A9BB289B223F4206343F480737E
:1047580021F0F30143EA022241F0010192B241EA59
:104768000411C1610262C2694FF6F37319E04EF693
:10477800FF730B400362C369056A40F6FF411940A5
:1047880045F6FF732B4043F4805343EA023241F469
:10479800807192B241EA0431C1610262C2694FF28A
:1047A800FF331340C361C369C36130BDA401002056
:1047B80038B510F80E2C50F8043C044652B90122C2
:1047C80000F80E2C20F80C1C997A18680222BDE813
:1047D80038406FE730F80C2C20F80A1C891A89B287
:1047E80020F8081C074A10F80F0C002522F81010B2
:1047F80004F80E5C1868997A2A46FFF75BFF04F8FC
:10480800065C38BDCC2E0020044B53F820301BB179
:1048180007289CBF1B681960704700BFD0020020A2
:10482800084A13689B050BD5074B002119700749E7
:1048380008684FF6FE7303400B604FF40073536033
:10484800704700BF00000240CE2F00203000024019
:104858002DE9F047664D2B6866490A78581C02F026
:10486800FF068E460AB10346F6E72B60687BAB6805
:1048780095F80C80AA7B374639B2202900F09B8036
:10488800DFF880C10CEB81033CF82110DC789B78C1
:10489800C3F1FF039BB2002B65D0C3F1FF03634351
:1048A8004FF03C0C1B12B1FBFCF9B9F1050F5DD8B8
:1048B800DFE809F0030B1A293A4AE01ADAB2414351
:1048C800B1FBFCF01044C0B251E0B1FBFCF00CFBB2
:1048D800101189B2DAB2C1F13C01E31A4B43204608
:1048E800B3FBFCFC94442CE0B1FBFCF00CFB101176
:1048F8005FFA83F8E21A89B24A43B2FBFCF24244F7
:10490800D2B2204632E0B1FBFCF90CFB191189B296
:104918005FFA83F8E01AC1F13C014843B0FBFCF0B0
:104928004044C0B2224621E0B1FBFCF80CFB181150
:10493800D8B289B2E31A01FB03F2B2FBFCFC2246AF
:1049480084445FFA8CF412E0B1FBFCF80CFB1811FC
:1049580089B2D8B2C1F13C01E31A4B43B3FBFCF274
:104968000244D2B203E02246204600E044464FEA21
:10497800042C4CEA004C4CEA020C172306F11701F0
:104988004FF0010808FA03F8C91A18EA0C0F89B29F
:10499800DFF8748014BF4FF011094FF0090913F1C3
:1049A800FF3308F80190E9D218360137B6B2BFB222
:1049B800114BA04660E7AA73AB60104AE980012357
:1049C8008EF800300E4985F80C8040F22A3368735F
:1049D800AE80536000234B620B889BB243F0010307
:1049E8000B80136843F001031360BDE8F08700BF34
:1049F800D0100020CE2F0020DC1000203000024014
:104A0800004401400A0F00204D03002073B50646FC
:104A18000D46002401232A88A34013421AD0AA78FD
:104A2800009302F003038DF80430EB78022B03D0D7
:104A3800032B0CBF032301238DF805303046C2F346
:104A480001136946C2F381028DF806308DF80720FC
:104A580003F080FB0134102CDCD102B070BD2DE9CD
:104A6800F04F734EF57B07460C4687B011469A46C1
:104A780000686B1C914622464FF0020BF3730BF053
:104A880049FF3B897868ADF8043001A98DF806B074
:104A98008DF807B0FFF7BAFF0023ADF80A30ADF87C
:104AA8001230ADF8163070230193BA7A3C68CDF80D
:104AB8000CA0012306F110082D01ADF808304FF4C1
:104AC8008073A844ADF810B0ADF814300C2A7ED825
:104AD800DFE802F0077D7D7D0F7D7D7D387D7D7D62
:104AE8005E00204601A903F089F9A36943F0080391
:104AF80026E0236A4F4823F010032362236A616883
:104B0800A26922F0807222F4E642844242F4E04232
:104B180006D000F50060844202D043F0300307E07D
:104B280023F0E00321F4406143F0300341F4806155
:104B38006160A261C4F838A02362A36943F40063EA
:104B4800A36144E0236A3B4823F480732362226A0A
:104B58006168E369844223F0730343F0700306D06D
:104B680000F50060844202D042F4407207E022F46B
:104B7800606221F4405142F4407241F48051616016
:104B8800E361C4F83CA02262E36943F008031DE036
:104B9800236A284823F480532362226A6168E36900
:104BA800844223F4E64343F4E04342F4405203D002
:104BB80000F50060844201D141F480416160E36105
:104BC800C4F840A02262E36943F40063E3613A7BDE
:104BD8003B681AB15A6C42F400425A641A8892B27D
:104BE80042F001021A80BA7A0C2A18D8DFE802F0DB
:104BF800071717170B1717170F171717130072191F
:104C080003F134010AE0721903F1380106E0721960
:104C180003F13C0102E0721903F1400111613544CE
:104C28004046A5F818906B6107B0BDE8F08F00BF4B
:104C3800D0100020002C0140F8B53A4E3A4C400004
:104C4800C7B24FF420453068C4F8D050D0F818E007
:104C58001EF4004F05D0AE46013DBEF1000FF5D160
:104C680016E0D0F804E0314D0EEA050545F490351C
:104C78003D4345604FF42045C4F8D050D0F818E0C3
:104C88001EF0020F2DD1AE46013DBEF1000FF5D149
:104C9800C4F8D0501FE02946013D0029F8D08169A9
:104CA8004906F8D5C4F8D05020494568294041F054
:104CB800007141F4105141EA0241394341604FF417
:104CC8002041A2B1306885696D071ED411F1FF310A
:104CD800F9D2C4F8D010FFF747FC003018BF012004
:104CE800F8BD4FF420458162C4F8D050D7E730684A
:104CF800C4F8D0100B46826992060CD41A46013BC0
:104D0800002AF8D1C4F8D030E5E7416A03F8011B5E
:104D1800013AD2B2D3E7C4F8D0302023C3610120CE
:104D2800F8BD00BFD8110020D0100020009800FC6A
:104D3800400070B5C5B23248324B00684FF4204489
:104D4800C3F8D0408669360404D52646013C002EB7
:104D5800F8D113E046682C4C344044F0807444F495
:104D680090342C4344604FF42044C3F8D040866903
:104D7800B60729D42646013C002EF8D1C3F8D04006
:104D88001CE02146013C0029F8D081690E06F8D5BF
:104D980044681D49214041F0007141F480312943A4
:104DA80041604FF42041C3F8D0108469A40711D49E
:104DB8000C460139002CF8D1C3F8D010FFF7D4FB0A
:104DC800003018BF012070BD4FF420448162C3F841
:104DD800D040DAE782624FF42042C3F8D0208169DC
:104DE800890606D41146013A0029F8D1C3F8D02023
:104DF800E4E7C3F8D0202023C361012070BD00BFC1
:104E0800D8110020D0100020009800FC2DE9F047B0
:104E18004D282DED028B044600F06A8600F2B98019
:104E2800302800F0E78651D8222800F0A98423D83A
:104E3800032800F0058214D8012800F0F581022823
:104E480040F0108704200AF081FD43200AF04FFD4E
:104E58004C200AF04CFD46200AF049FD4C2000F099
:104E68006EBE042800F0F581052840F0FB861A2064
:104E78000AF06CFD0024FCE1282800F0F88515D81C
:104E8800242800F0DF85262840F0EC86D94C06203F
:104E98000AF05CFDB4F85C010AF05BFDB4F85E0151
:104EA8000AF057FDB4F8600100F0C9BD2C2800F0E5
:104EB800F1852E2800F06D862A2840F0D38601203F
:104EC8000AF044FDCB4B587900F039BE3D2800F07C
:104ED800F8821ED8362800F043860BD8322800F016
:104EE8002886342840F0BE8648200AF02FFD002589
:104EF80000F068BC3A2800F0BB823B2800F03984F7
:104F0800382840F0AF8604200AF020FDB94C00F0A4
:104F18009FBD452800F0938627D8402800F01286C8
:104F2800422840F09F86B34C10200AF00FFD6079AC
:104F38000AF0DDFCA0680AF015FD94F892010AF069
:104F4800D6FCB4F85C010AF004FDB4F85E010AF07E
:104F580000FDB4F860010AF0FCFCB4F882010AF024
:104F6800F8FCB4F8840100F06ABD492800F0B48266
:104F78004B2800F0AE85462840F074860D200AF0D4
:104F8800E5FC00200AF0B3FC00200AF0EBFC00F07E
:104F980061BE702800F0F08200F2DE80692800F01F
:104FA800478200F2AF80662800F0A18100F29F805E
:104FB800642800F07781652840F054868E4C0B20D9
:104FC8000AF0C4FC20880AF0C4FC62688B4B9A4241
:104FD8000CBF2089608980B20AF0BBFC884B1B6833
:104FE800C3F3C000C3F38002800040EA4200C3F369
:104FF80040021043C3F3401240EAC20003F010031A
:1050080018430AF0A6FC7F4B1A88E36812F0010FD8
:1050180014BF4FF0020C4FF0000C12F0020F02F018
:10502800080814BF4FF0040E4FF0000E03F4475960
:1050380012F0040F14BF1027002749EA080912F0DC
:10504800400F03F4804814BF2026002649EA0809C7
:1050580012F0100F03F4004814BF4FF40075002538
:1050680049EA080912F0200F03F4803814BF4FF4FE
:105078008060002049EA080912F4807F03F40038B0
:1050880014BF4FF40061002149EA080912F4007FB7
:1050980003F480285C4A49EA080903F4002849EA2D
:1050A8000809127803F4801849EA080903F0007324
:1050B80049EA0303C2F3800243EA020343EA0C030A
:1050C80043EA0E0E4EEA070746EA070645EA0605D2
:1050D80040EA050041EA000114BF4FF400184FF000
:1050E8000008002041EA08080346217CEAE0672816
:1050F80000F02581682840F0B58510200AF026FCCC
:1051080000248CE16C2800F0A68117D86A2800F0EA
:105118001B846B2840F0A68505200AF017FC3B4B42
:1051280018880AF016FC3A4B18880AF012FC324B21
:1051380093F8720000F0010000F001BD6E282E4DBA
:1051480000F09A8100F2CE8106200AF0FFFB686E1B
:105158000AF008FC2F4B89E1782800F0FD8018D868
:10516800742800F050830AD8722800F0AD837328A1
:1051780040F0788508200AF0E9FB0124DDE3762871
:1051880000F0028400F280832F200AF0DFFB224C1B
:10519800E7E2A42800F01F8414D87B2800F0878257
:1051A800A02840F05F850C200AF0D0FB1B4B186844
:1051B8000AF0D8FB1A4B18680AF0D4FB194B186888
:1051C80000F04CBDF12800F00381FE2800F02A848D
:1051D800F02840F04785084C04200AF0B7FBA36C80
:1051E800B3F85A000AF0B5FBA36CB3F8580000F006
:1051F80026BC00BFA0240020D41100200054004089
:105208006C14002030150020CF2F0020EA14002055
:10521800EC14002040140020737F0108ACF7FF1F36
:10522800B0F7FF1FB4F7FF1F03200AF08FFB002021
:105238000AF05DFB20460AF05AFB0C2000F07FBC08
:105248000AF084FB01200AF052FB0A200AF04FFB07
:10525800BFE306200AF07AFB53200AF048FB5020EF
:105268000AF045FB4B200AF042FB59200AF03FFBAD
:10527800E4E3B04B185D01340AF039FB0B2CF8D18C
:105288000024AD4B185D01340AF031FB082CF8D12D
:105298000024AA4B185D01340AF029FB072CF8D129
:1052A80000F0DEBC07200AF051FBE7200AF01FFBE4
:1052B800A34B58790AF01BFB00200AF018FB0420C6
:1052C80000F0CCBC8B420BD29E4A9C5C012202FAB5
:1052D80004F414EA080F1CBF9A4010430133F1E7A5
:1052E8000AF040FB964B93F8A40700F028BC122064
:1052F8000AF02CFB944B1B88B3F5806F8CBF0825F4
:1053080001250024914B33F9140090FBF5F001348A
:1053180080B20AF01EFB032CF4D18D4CA08D0AF04C
:1053280018FBE08D0AF015FB208E0AF012FB608E48
:105338000AF00FFBA08E0AF00CFBE08E7FE3102032
:105348000AF004FB0024834B185D01340AF0CFFAFD
:10535800102CF8D100F084BC70200AF0F7FA00266F
:105368007B4D0E24AB6C744323440136B3F819010A
:105378000AF0EFFAAB6C2344B3F81B010AF0E9FA20
:10538800AB6C2344B3F81D010AF0E3FAAB6C234479
:1053980093F81F010AF0ABFAAB6C234493F8200191
:1053A8000AF0A5FAAB6C234493F821010AF09FFA9E
:1053B800AB6C234493F822010AF099FAAB6C1C44B5
:1053C800D4F823010AF0CEFA082EC9D100F048BC5F
:1053D80070205B4C0AF0BAFA04F1700594F8D40016
:1053E8000AF085FA94F8D5000AF081FA94F8D60004
:1053F8000AF07DFA94F8D7000AF079FA94F8D80000
:105408000AF075FA94F8D9000AF071FA073494F89A
:10541800D3000AF06CFAAC42E0D100F021BC4E4B4C
:10542800185D01340AF063FA102CF8D100F018BCAA
:105438004A4D2878400000F0FE000AF087FA002460
:105448002B789C4280F00C84454B33F814000AF00A
:1054580080FA0134F4E7434C06200AF077FA2088F2
:105468000AF077FA60880AF074FA3F4B1888E6E287
:1054780004200AF06BFAF0E307200AF067FA3B4BC6
:105488001888FF28A8BFFF20C0B20AF030FA384BAE
:10549800186880F3100080B20AF05BFAB5F868006B
:1054A8000AF057FA264B93F88721324B186822B135
:1054B8000A23584380F3100001E000F30F0080B284
:1054C800BDE21F4C02200AF041FA94F8D6010AF016
:1054D8000EFA94F8D50132E302200AF037FA184B95
:1054E8009889ACE20B200AF031FAEB6E18780AF0D2
:1054F800FEF9EB6E58780AF0FAF90026EB6E144CB8
:105508003344013618790AF0F2F9032EF6D1E36E26
:10551800D8790AF0ECF9E36E98780AF0E8F9E36EC6
:10552800D8780AF0E4F9E36E58890AF012FAE36EC3
:10553800187A04E344A2010850A2010859A20108FC
:10554800A0240020E5110020160000203A140020B5
:10555800D41100200C12002020120020382F002027
:105568007C24002036240020481400205C140020ED
:105578006814002064140020BF4C1E200AF0E6F9CD
:10558800A36C1B78022B4FF000057DD1A36C03EBB5
:10559800850393ED080AB2EE048A20EE080A10F09B
:1055A80041FCFA28A8BFFA2020EAE070C0B20AF04D
:1055B8009EF9A36CDFEDB17A03EB850393ED0B0A3B
:1055C80020EE270A10F02EFCFA28A8BFFA2020EABD
:1055D800E070C0B20AF08BF9A36CDFEDA97A03EB97
:1055E800850393ED0E0A20EE270A10F01BFC6428B1
:1055F800A8BF642020EAE070C0B201350AF077F94C
:10560800032DC3D1072DA36C2CD193ED110A20EEE5
:10561800080A10F007FCFA28A8BFFA2020EAE07070
:10562800C0B20AF064F9A36C93ED120A20EE080ADE
:1056380010F0F8FBFA28A8BFFA2020EAE070C0B200
:105648000AF055F9A36C93F84C3000EE103AB8EE16
:10565800400A10F0E7FBFA28A8BFFA2020EAE07019
:10566800C0B20BE02B4458780AF041F9A36C2B44E4
:10567800D87A0AF03CF9A36C2B44587D01350AF01E
:1056880036F90A2DBED1EBE2A36C2B4458780AF008
:105698002EF9A36C2B44D87A0AF029F9A36C2B4471
:1056A8000135587D0AF023F90A2DEDD1D8E23C20C6
:1056B8000AF04CF90024704D9FED718AAB6C03EB36
:1056C800840393ED080A20EE080A10F0ABFB80B2C1
:1056D8000AF03FF9AB6C03EB840393ED0B0A20EE61
:1056E800080A10F09FFB80B20AF033F9AB6C03EBA9
:1056F800840393ED0E0A20EE080A10F093FB0134A0
:1057080080B20AF026F9032CD5D1072CAB6C16D140
:1057180093ED110A20EE080A10F084FB80B20AF01B
:1057280018F9AB6C93ED120A20EE080A10F07AFB18
:1057380080B20AF00EF9AB6C93F84C000BE02344EE
:1057480058780AF006F9AB6C2344D87A0AF001F9C4
:10575800AB6C2344587D01340AF0FBF80A2CD4D1F1
:105768007EE214F8010F002800F07A820AF0BFF8F0
:10577800F7E701200AF0EAF83F4B9B6C1878DEE166
:1057880050200AF0E3F800253B4B9C6C3D4B04EBA2
:1057980085040C2194F8792001FB0233013593F834
:1057A80038000AF0A4F894F87A000AF0A0F894F8FF
:1057B8007B000AF09CF894F87C000AF098F8142D05
:1057C800E2D14DE22C4B9C6C062303FB05440135CA
:1057D80094F8CE000AF08BF894F8C9000AF087F81C
:1057E80094F8CA000AF083F894F8CB000AF07FF81E
:1057F80094F8CC000AF07BF894F8CD000AF077F81A
:105808000C2DDFD12CE24FF00008012600271A4B9F
:105818001A7C974227DA11330024FA5C194D0C23BD
:1058280005F130016343595C914207D12B44586B11
:1058380010F02DF982462EB9B14605E001341B2C33
:10584800ECD10EE080440CE0D1450ADA0C2303FBCE
:1058580004535B6B13F809000AF049F809F10109D0
:10586800F2E70137D3E7002E00F0FA815FFA88F0FB
:105878000AF06CF80026C9E7D41100200000C842DD
:1058880000007A44747F0108CD4D287C0AF05EF848
:1058980000242B7C9C4280F0E381CA4BE65C00210B
:1058A800C9480C2200F1300702FB01F3DA5DB2426D
:1058B80005D1034493F838000AF019F802E00131E1
:1058C8001B29EDD10134E4E7C04C16200AF03EF85C
:1058D800B4F898010AF03DF8B4F844010AF039F830
:1058E800B4F846010AF035F8B4F848010AF031F87E
:1058F800B4F8D2010AF02DF894F8E30109F0F7FFA3
:10590800002009F0F4FF94F8E40109F0F0FF94F89E
:10591800870109F0ECFF94F8940109F0E8FF0020F2
:1059280009F0E5FFA64B9B6C0A20B3F9563093FBB0
:10593800F0F080B20AF00DF88AE0E0B2013409F024
:10594800D6FF092CF9D18BE1102009F0FFFFA04BFD
:10595800A04C187800F0020009F0C9FF9E4B187897
:1059680009F0C5FF206809F0FDFF606809F0FAFF3B
:105978009A4B188809F0EDFF994B188809F0E9FF50
:105988008F4BB3F870005AE009F094FF07461220D5
:1059980009F0DCFF8A4C17B9666FA56F06E0102F77
:1059A80013BF0025E66FD4F880502E46384609F01C
:1059B8009EFF304609F0D6FF284609F0D3FFD4F8F9
:1059C800840009F0CFFF002009F0C3FF002009F090
:1059D800C0FF0020B3E07A4D95F8880080000130C0
:1059E800C0B209F0B3FF95F8880009F080FF0024E1
:1059F8002E4696F888309C4280F03281794D285D99
:105A080009F075FF05F11003185D09F070FF05F145
:105A180020033035185D09F06AFF285D09F067FF3B
:105A28000134E6E7082009F091FF002009F091FF12
:105A3800002009F08EFF002009F08BFF002009F0FC
:105A480088FF0DE1042009F081FF604B986805E1AB
:105A580094F87C0109F04BFF94F8800109F047FFA6
:105A680094F87F0109F043FF94F8810167E0574CEF
:105A7800072009F06BFFB4F8820109F06AFFB4F857
:105A8800840109F066FF94F8860109F030FFB4F844
:105A98008801D4E74D4C0C2009F058FF94F8920186
:105AA80009F025FFB4F89C0109F053FFB4F89801F8
:105AB80009F04FFFB4F89A0109F04BFF94F89301ED
:105AC80009F015FFB4F89E0109F043FFB4F8A001EE
:105AD800B5E73E4C042009F039FF94F8D00109F0ED
:105AE80006FF94F8D10109F002FFB4F8D201A6E745
:105AF8003D4C3E4D2078043800EB4000C0B209F020
:105B080025FF042623789E4205F1020580F0A8802F
:105B180015F8020C09F0EBFE15F8010C00EB8000FB
:105B280000EB800000F2EE2080B209F012FF01368F
:105B3800E8E7012009F00AFF244B93F8940109F0E3
:105B4800D6FE8DE0082009F001FF00241F4B2344F6
:105B5800013493F88A0109F0CAFE082CF6D17FE0D7
:105B6800174B1A4C93F8C900C0EBC000C0B209F03B
:105B7800EDFE04F1200594F8EA0100231C4AD25CEA
:105B8800904271D00C33302BF8D10834AC42F2D1AA
:105B980066E040200D4C09F0D9FE04F14005B4F848
:105BA8009C0209F0D6FE94F89E0209F0A0FE043487
:105BB80094F89B0209F09BFEAC42F0D150E000BF84
:105BC800D4110020E5110020747F0108A0240020D2
:105BD800701400207814002076140020741400201B
:105BE800721400205D120020382F00204226002069
:105BF80000230020E0202A4C09F0A8FE04F18005CB
:105C0800B4F81E0200F03F0009F0A3FEB4F81E022B
:105C1800C0F3861009F09DFE94F81C02000909F0F3
:105C280066FE94F81C0200F00F0009F060FE0434D0
:105C380094F8190209F05BFEAC42E1D110E01320A0
:105C480009F084FE0024174B185D013409F04FFE5B
:105C58000B2CF8D1002009F085FE002009F082FE07
:105C6800012018E0002016E009F041FEB4F8EC012C
:105C780009F06FFE94F8EE0109F039FE94F8EF018F
:105C880009F035FE94F8F10109F031FE94F8F001BD
:105C980009F02DFE79E7BDEC028BBDE8F08700BF67
:105CA800A024002044A2010882B01B4B1B4A8DF897
:105CB80007101968106860B31268052A29D1184AB4
:105CC800106810BB9DF808109DF8073043EA0123BF
:105CD80014490B80144B1968144B89B20B445B00B0
:105CE80019680121196013680B441360104A13687E
:105CF80023F4E04323F040039BB283F0300343F4E2
:105D0800004343F08003136003E01A68521A312AF3
:105D1800D5D902B0704700BF64240020B42F0020FA
:105D28005822002080610040505C00400A3000206A
:105D3800045C0040014B1868C0B270471422002070
:105D480001207047704770476D4B6E4A9FED6E7A21
:105D5800D2ED007ADFED6D4ADFED6D3A30B51C8883
:105D6800B3F90AE01D8A06EE904AB8EEE76AF8EE43
:105D7800666ADFED687AB3F9044067EEE67AB7EE53
:105D8800004AE6EE077A9FED647A67EE666A9FED51
:105D9800637AE6EE076A27EEA77A07EE904AB3F928
:105DA80002409FED5F6AF8EEE77A67EE277A07EE22
:105DB800104AB8EEC77ADC89E6EE877AB6EE007A42
:105DC800FDEEE76A87EE866AC3ED066AF8EEE66AD4
:105DD800D2ED017A9A89E6EE874A06EE90EAB3F99F
:105DE80008E09FED507A05EE90EAF8EEE66AF8EEE4
:105DF800E55A66EEA46A65EEA45A66EEA46AB3F89C
:105E080006E0E6EE875A65EE875AA5EEA34AF0EE5D
:105E1800445A04EE10EAB8EE444A25EE844AB5EE38
:105E2800404AF1EE10FA5BD02DB205EE905A24B23A
:105E380024EEA45A07EE104AF8EEE55A12B265EEBF
:105E4800255AB8EEC75A65EEA35A64EE854AB0EEF5
:105E5800007AE4EE875AB5EE007A65EE875A07EEC7
:105E6800102AB8EEC75A9FED307ADFED306AB3F9E1
:105E78001620E5EE075AF8EEE77A9FED2D7A76EED2
:105E8800E77ADFED2C6AE5EEC77A05EE902AB0EEE8
:105E9800677ADFED297AB3F91420B3F9123067EE87
:105EA800277A07EE102AC7EE847AF8EEE55AB8EE9C
:105EB800C77A65EEA75A27EE877A65EEA75A27EEC6
:105EC800237AA5EEA67AF0EE476A07EE103AB8EE06
:105ED800C77A36EE877ADFED196AE7EE267A01E0AF
:105EE800DFED177A18B1FDEEE77AC0ED007A31B12F
:105EF800FDEEC67A642217EE903A53430B6030BD2C
:105F080010030020A01200200000003700007AC70C
:105F180000000038000000390000803A0000803896
:105F28000000A045000000360000804700008049BE
:105F380000008039000000300050C3450000803D5B
:105F480000000000704770476C4B6D4A2DE9F04F18
:105F58005E8994684FEA062AB4EB0A0A9C884FEADD
:105F680004481C894FF000054FF0000B65EB0B0B44
:105F7800A4FB0A6704FB0B77F40944EA476418EBAF
:105F880004065C884FF000094FEAE7154FEAC43869
:105F9800DC8849EB050787B0CDE90467A4FB0A67ED
:105FA80004FB0B77340A44EA076418EB04064FEA4B
:105FB80027259C894FF0000949EB0507CDE90067C3
:105FC800AAFB046704FB0B77F40D44EA472414F595
:105FD800FA664FEAE75545F10007B6F5FA6F77F12B
:105FE8000003CDE90267964667DAA4FB046704FB61
:105FF80005F34FF0050C07EB4307DDE90489A6FB21
:106008000C230CFB07335F104FEA3206B8EB060887
:106018004FEA920669EB070946EA83769F10DDE9A5
:106028000023921B63EB0703DDE90267CDE9002338
:10603800344A4FF0FF33964277EB0303CDE90489E6
:1060480028DA40F6AC52A4184FF000035D4104FB77
:1060580005F3A4FB044505EB43056FF00602664211
:1060680002FB0566A4FB0223334418EB020649EB46
:106078000307CDE904670B26A4FB062306FB0533BB
:10608800DDE900455B104FEA3202A41A65EB03050F
:10609800CDE900450AFB0BF3DDE90245AAFB0AAB93
:1060A8000BEB430B4FEADA7242EA4B02A41A4FEAAF
:1060B800EB7365EB0305CDE90245DEF80C40009B68
:1060C800019DA4FB032304FB05334FEA52584FEA12
:1060D800635948EAC328DDE90423B8EB020269EBF7
:1060E80003039946D30B43EA494300B1036009B15E
:1060F800029B0B6007B0BDE8F08F00BFFE020020D6
:10610800A012002024FAFFFF07EE900AF8EEE77AC3
:10611800DFED0C6A9FED0C0AF5EEC07AF1EE10FA8D
:10612800D4BFB1EE677AC7EEA67A08B5D8BFC7EE76
:10613800267A27EE800A03F0EBF9044B83ED000A78
:1061480008BD00BF8096184B35FA8E3C74000020BD
:10615800F7B51C4B1A680AB91C6800E001241A49F3
:106168000E7C0022D0B2A04202F1010207D202AD99
:106178002F18164D3544285C07F8040CF2E71A6806
:10618800121B1A600A7C1D6822440A749DB90320F8
:10619800402101F0C7FC0E4A136823F4804323F022
:1061A80070039BB283F4405343F4004343F08003ED
:1061B8001360054B1D74002CCBD09DF8040003B070
:1061C800F0BD00BF14220020A012002018220020D9
:1061D8000C5C00407620F4213122FEF7A9BD1FB5E2
:1061E800044602210C2001220DF10703FEF724FDCD
:1061F800C8B39DF80730DB0735D50321062202AB6B
:106208000C20FEF719FD0C20092101220DF10703CE
:10621800FEF712FD38B39DF8073013F00C0F22D1AA
:106228009DF809209DF8083043EA0223C3EB833325
:106238009B009DF80B2023809DF80A3043EA022337
:10624800C3EB83339B009DF80D2063809DF80C30D1
:1062580043EA0223C3EB83339B00A3800C200A216B
:106268000122FEF765FD04B010BD07B5F7216B46A6
:1062780006227620FEF7E0FC9DF800309DF801101C
:106288000B4A1B0343EA01139DF8021043EA11135A
:1062980053609DF803309DF804101B0343EA011373
:1062A8009DF8051043EA1113136003B05DF804FB71
:1062B800A012002007B50A2100220C20FEF738FDA5
:1062C800142005F030FE0A210F220C20FEF730FDC5
:1062D8000A2005F028FE01AB102103220C20FEF74E
:1062E800ABFC0A2005F01FFE0A2100220C20FEF755
:1062F8001FFD0A2005F017FE0DF1030302210122FC
:106308000C20FEF799FC0DF10303092101220C2052
:10631800FEF792FC0A2101220C20FEF709FD03B0CA
:106328005DF804FBF8B59F4B1B680446187818B154
:10633800012800F07181EDE2242C9B4D0CD006D889
:106348000A2C00F0DD800D2C00F0DA804EE12A2CBA
:1063580006D02C2C04D049E16874A874E87457E17D
:10636800924BA97C6F7C904A002058542FBB197817
:106378001775472921D1597850291ED1997847296D
:1063880007D1D978472904D11979412901D10121A7
:1063980011759978854A522903D1D1784D2900F091
:1063A800BB829978814A472907D1D178532904D1EA
:1063B8001279562A04BF03222A752A7D7A4E022AA8
:1063C8003AD0032A4DD0012A40F08880BA1E072A05
:1063D80000F28480DFE802F004080F131A25822BEC
:1063E8000AF04CFDA86179E01B78532B76D1AB6994
:1063F8005B42AB6172E00AF041FDE8616EE01B7838
:10640800572B6BD1EB695B42EB6167E01B78302B54
:10641800674B1A788CBF42F0020222F002021A700F
:106428005CE000200AF08AFD85F8200056E0002094
:106438000AF084FD688451E0072F06D0082F4DD15B
:1064480001200AF07BFDF08448E001200AF076FD87
:1064580041F2184358434FF47A73B0FBF3F0B08419
:106468003CE0022F07D0032F0BD100200AF066FD75
:10647800504B187032E000200AF060FD86F82800C2
:106488002CE02BD93A1F921096F828300132D2B25C
:10649800013B02EB8303DBB2102B1FD8F91EC2F1BC
:1064A800010201EB8202D2B2012A0BD0042A11D1D7
:1064B80000205E1E0AF042FD3F4B98553F4B0022DC
:1064C8009A5507E05E1E3E4A002093550AF036FDB5
:1064D8003C4B98553C4A136801331360324B2A2CC5
:1064E80018BFDA7C07F101074FF000000CBF01224A
:1064F80054406F74A8740CBF83F82920DC7487E0BB
:1065080095F82900002848D0304B13F8012D304960
:106518005A708B42F9D1254A234C13785278402B74
:1065280085BF373B1B011B01DBB298BF03F0F003AB
:10653800402A8CBF373A303AD2B21344EA7CDBB2F5
:106548009A4227D121230B702249207D0B68204ACB
:10655800013301280B600AD002281DD17223137061
:106568001D4BA28C1A801D4BE28C1A8014E0672305
:1065780013700F4B1B789F070FD5194BA2691A6030
:10658800E2695A60174B94F820201A70164B628CF7
:106598001A8002E03F230B700020002385F8293081
:1065A80036E000BF4C080020A01200206C24002018
:1065B800701400205C1200208D1200207D12002033
:1065C8005D1200206D120020781700204C03002077
:1065D8003803002084170020721400204412002081
:1065E800781400207614002074140020AB7C95F8F1
:1065F80029000E2B9FBFAB4A591C9174AA4A98BF19
:10660800D454A84A18B9D37C5C40D47400E0002064
:10661800003018BF0120F8BDA24B93F82A100022C1
:10662800082900F27781DFE801F0050C101A2B3BEE
:106638005F7B8800B52C40F06D8183F82B20012208
:106648004FE0622C08BF02224BE0032283F82A2085
:1066580083F82C4083F82D4083F82E405AE1042219
:1066680083F82A2093F82D2093F82E1083F82F40D2
:106678002244D2B283F82D200A4483F82E2049E11F
:10668800052283F82A2093F82D2093F82E101C86D3
:106698002244D2B283F82D200A4483F82E2039E10F
:1066A800062283F82A2093F82D2093F82E102244EE
:1066B800D2B283F82D200A4483F82E201A8E02EBDA
:1066C8000424A4B2B4F5AC7F88BF764A1C8684BF84
:1066D800012182F82B1000225A86002C40F01A81E2
:1066E800072283F82A2015E193F82D2093F82E101D
:1066F8002244D2B283F82D200A4483F82E205A8EE1
:10670800B2F5AC7F3CBF6749891802F1010238BF76
:1067180081F83440198E92B291425A86E0D9F9E054
:10672800082283F82A2093F82D30A34200F0F28043
:106738005C4B012283F82B200FE05C4D83F82A2064
:1067480015F8012D6A705A4A9542F9D193F82E101E
:10675800544AA14206D03F232B70564A536801334E
:106768005360D7E0544801680131016092F82B006A
:1067780010B13E232B70CDE02121297092F82F1003
:10678800062941D004D8022907D0032923D0F8BD0F
:10679800122959D0302967D0F8BD502129704749AE
:1067A800946B4C60D46B0C60516C4FF47A7491FB11
:1067B800F4F1434C218092F88C11424A19B11178B6
:1067C80041F0020102E0117821F00201117001226A
:1067D80083F88D2190E05321297092F83910CE0763
:1067E80005D592F83820D51E6A426A4100E0024673
:1067F80002F0010183F88C11002A7DD131490A7811
:1068080022F002020A7077E04F21297092F83F10B7
:10681800CC0705D592F83E20D11E4A424A4100E0F5
:10682800024602F0010183F88C1122B925490A7841
:1068380022F002020A70244A93F863101170234A66
:10684800B3F86010118057E0562129702049946CE4
:106858000C8042F21074D16C91FBF4F11D4C218034
:10686800012182F88E1147E04921297092F83810E9
:10687800194A102988BF102111701849147800226C
:10688800A24235D2164D0E7A5655164D4E7A5655A9
:10689800154DCE7A5655154D11F80C6F56550132D7
:1068A800EEE700BFA01200206C2400204C0300205B
:1068B800380300202C0800208417002078140020BA
:1068C80074140020701400207614002002010020A7
:1068D80072140020441200205C120020D412002000
:1068E8005D1200206D1200207D1200208D12002004
:1068F8000D490A6801320A6093F88D310B4A93B149
:1069080092F88E317BB1002182F88D1182F88E11B8
:106918001846F8BD0020F8BD1279432A7FF441AD2E
:1069280002222A753DE5F8BD78170020A012002044
:106938000449054B0968187000225A6199611A7751
:10694800704700BF642400202C08002010B5121ADC
:1069580007EE902A5B1A2DED028BF8EEE78A07EE18
:10696800903A184B059CB8EEE78AD3ED007A28EEEA
:10697800278A28EE080AA8EEA80A0FF0F9FCDFED2E
:10698800127A049B20EE270AF0EE480ABCEEC00AF1
:1069980083ED000AB1EE680A0FF046FBDFED0B7AD3
:1069A8009FED0B7AE0EE077ABDEC028BFDEEE77AFD
:1069B80017EE903A002BBCBF03F50C43A0332360BD
:1069C80010BD00BF740000202C7D8E3F00A00C4637
:1069D800A00CB34544F25063984203DDA0F50C4087
:1069E800A0387047034B9842BCBF00F50C40A0305C
:1069F800704700BFB0B9FFFF73B51A4C0368236036
:106A08000B686360184D0068184EFFF77DFB184B44
:106A1800009395E8030094E80C000196FFF796FFB1
:106A2800144B32681A606868636813491B1A07EECA
:106A3800903A124B286893ED007A23681B1A0B6072
:106A48000F4BF8EEE77A1A600E4B67EE877A1B68F1
:106A5800FDEEE77ADA880C4BC1ED017A1A8002B0B4
:106A680070BD00BF50210020781400205C21002058
:106A78005821002098210020602100207400002067
:106A880090210020481000208C2100204279DFED61
:106A98002A5A2A4B9FED2A5A07EE902AF8EE677A6F
:106AA800C27BC7EEA57AB2EE047AC3ED007A07EE90
:106AB800902AF8EE677A234ADA60C7EEA57AC3ED22
:106AC800017A8179204B07EE901AF8EE677A017CFB
:106AD800DA60C7EE877AC3ED007A07EE901A817EF6
:106AE80006EE101AF8EE677AB8EE466AC7EEA57A8F
:106AF80086EE056AC3ED017A83ED026AC179134B0C
:106B080006EE901A417CDA60F8EE666AC6EE876A8D
:106B180007EE101AC17EC3ED006A07EE901AB8EEB0
:106B2800477AF8EE677A87EE257AC7EE857A83ED9D
:106B3800017AC3ED027A70470000C842682100203C
:106B480000007A440000FA44782100209C210020AB
:106B580010B50C4C23789B0713D50B4B1B78042BD3
:106B68000FD90A4A0A4B106852685A601860FFF732
:106B7800CBFA084B1A88084B1A80237843F0010394
:106B8800237010BD701400207614002078140020A3
:106B98004812002048140020AC2100201C4B1B6820
:106BA8001B0307B530D51B4A1B4BD2ED007A1B7867
:106BB8008DF80030B2EE047A67EE877A174B9FEDB6
:106BC800187A1B788DF80130FCEEE77A0A2017EE68
:106BD800903AD2ED017A8DF8023067EE877A6946ED
:106BE800FCEEE77A17EE903AD2ED027A8DF8033090
:106BF800FCEEE77A17EE903A8DF80430094B1B78D3
:106C08008DF8053001F01AFD03B05DF804FB00BFF4
:106C18004024002054240020302400205024002048
:106C280000007A4434240020054A137883F00103D5
:106C38001370044A00231360034A1360AEE700BFD1
:106C4800342400204C240020482400202DE9FF474C
:106C5800CA4CCB4F23780646002B00F0EA813A68ED
:106C68006368D31A7C2B40F2E481237A6260013393
:106C780023724FF0000808F12400C04DC0B203F0A1
:106C880047FB05F10A0333F9183007EE903ABD4B7C
:106C98001B88B8EEE77A07EE903AF8EEE77A08F143
:106CA8000108C7EE277A9FEDB87A67EE877AFDEE7E
:106CB800E77ACDED017ABDF9040003F017FBB8F1CE
:106CC800030FD8D1302003F023FBB5F9100003F0EF
:106CD8000DFB03F015FB2B7A9A072CD16A6841F259
:106CE80088339A4218D9102003F012FB4FF0640839
:106CF800686990FBF8F000B203F0F8FA212003F07D
:106D080007FB686990FBF8F308FB13000028B8BF7D
:106D1800404200B203F0EAFA142003F0F9FAB4F999
:106D2800180003F0E3FA1C2003F0F2FA002003F045
:106D3800DDFA03F0E5FA237ADFF840825B0740F0DA
:106D48005581022003F0E4FAD8F81C00DFF85092CD
:106D58006423323090FBF3F000B203F0C7FA03204B
:106D6800B8F9265003F0D4FA884B1B7813F0040FB7
:106D78004FF0050A95FBFAF5ADB20BD030460AF094
:106D88003AF928B9D9F8003013F0100F18BF0025C8
:106D980028B205E0D8F828309889B0FBFAF000B29C
:106DA80003F0A4FAD9F800309E0765D5DFF8F4910E
:106DB800E68D99F80030A28D704D36014FF06408C9
:106DC800B6B208FB02325B00B2FBF3F346EA0326D5
:106DD800B6B2C3F303231E43062003F099FA30B278
:106DE80003F084FAE38D99F8001001339BB293FB0A
:106DF800F1F201FB1233E385236B9B7B012B05D159
:106E0800392003F085FAB5F92C0019E0AD8D6E2311
:106E18003A205D43152603F07BFA95FBF6F5AEB2F2
:106E2800B6FBF8F528B203F061FA08FB15653B20BC
:106E380003F06EFAA8B2451D0A2095FBF0F000B2E7
:106E480003F054FA282003F063FA636B0A2093FBDB
:106E5800F0F000B203F04AFA042003F059FAA36AEA
:106E68009B8913B101F04EFA03E0444B986B80F311
:106E7800100000B203F03AFAE36B404E9D0640F171
:106E8800AA8096F8403098071DD5112003F040FAE3
:106E9800B6F842003E4B4FF4F365684390FBF3F0BD
:106EA80000B203F023FA192003F032FAB6F84200D0
:106EB8004543642095FBF0F595FBF0F300FB135078
:106EC80000B203F013FA94F84030B4F8445013F0C9
:106ED800020F08BF0025012003F01AFA28B203F0B8
:106EE80005FA092003F014FA002003F0FFF9294BF2
:106EF80094F846501A88B2F5967F0AD91F4B1B7A28
:106F080003F00F03072B04D842F20F75954228BFF0
:106F18001546052003F0FCF9236B5B7B0BB928B2FF
:106F28001CE0A5F1200307EE903A9FED1B7AF8EEDE
:106F3800E77AF6EE006AC7EE877ABEEE007AF5EEDB
:106F4800C07AF1EE10FA58BFB0EE667A77EE877A1B
:106F5800FDEEE77ACDED017ABDF9040003F0C6F93C
:106F680094F84020054B910703D493F84720012A51
:106F78001CD1012384F84730084833E0301400203E
:106F8800642400201600002000007A44CF2F00203F
:106F9800A0860100020100206666E63F7814002002
:106FA80040240020010100208096184B1B6B5FEDE8
:106FB800026A93ED017AD3ED027A27EE267A67EE1C
:106FC800A67ABDEEC77AFDEEE77A8DED027ACDEDB1
:106FD800037A02A806E0A74A92E8030002AB83E816
:106FE8000300184603F0A4F903F08AF9237A282B42
:106FF8001FD1A14B00221A723C263B684FF47A70CD
:10700800B3FBF0F8172003F083F9B8FBF6F5B5FBEE
:10701800F6F006FB1050000200B203F067F91820E2
:1070280003F076F906FB158000B203F05FF903F070
:1070380067F994F85030904D002B00F03D8104F032
:107048004DFF6B6D8D4AC31A9342064640F2C180CC
:10705800002385F85A3085F85C30AB8DDAB21B0A0C
:1070680085F8762085F8773085F86C2085F86D30BE
:10707800D5F884203B689A1AD5F88830D97B4FF424
:107088007A734B439A420ED37D4B1B68C5F8843004
:1070980095F88C30013B012B9FBF102385F85A309F
:1070A800022385F85C300A20626B92FBF0F284F8C8
:1070B8007420121284F8752094F84020A36B93FB77
:1070C800F0F384F878301B1284F87930920794F83A
:1070D8004630694984F8A73003D42D2381F8A830B5
:1070E80076E0042BD4F84890E76CDFF8A481654A71
:1070F8008CBF3323322381F8A8304FF0060C624B43
:1071080099FBF3F097FBF3F308FB009108FB037876
:1071180003EB83030CFB01F103EB830391FBF2FE0A
:10712800642502FB1E119B0091FBF5F184F8991070
:1071380009120CFB08FC84F89A109CFBF2F143FA44
:1071480081F39BB202FB11C292FBF5F284F89E20F8
:10715800121284F89C3084F89F201B0AB4F842204D
:1071680084F89D302423534393FBF5F5B4F8BA30E3
:1071780084F8A03000EB80001B0A00EB8000800040
:1071880084F8A1300A22B4F84430B3FBF2F303F5D3
:10719800FA739BB240FA8EF080B284F8A2301B0AD0
:1071A8004FEAD97984F89700FF0F000A84F89450C1
:1071B80084F8A330C5F30725B4F8BC3084F896905A
:1071C80084F8980084F89B7084F8955084F8A93066
:1071D800666594F8BE80284DB8F1000F0DD1D5F83A
:1071E800C40005F033F8012807D90228274F00F01A
:1071F800388203F06DF80123BB70D4F8C8001E4D27
:10720800002859D095F8BE703FB1D5F8D03040F677
:10721800B732F31A93420BD84EE00123D5F8C400D5
:1072280085F8BE30022105F005F885F8D47041E0F4
:1072380095F8CC305BB9D5F8C400C5F8C830012141
:1072480085F8BE3004F0F6FF03F042F832E0013B67
:10725800DBB285F8CC3095F8D41095F8D520CBB9A9
:107268004B1C013285F8D43085F8D520D5F8C400F8
:107278001EE000BFF4800108301400203F0D030019
:107288006424002040420F008096980016000020D9
:10729800806967FF0346013213F8017BC5F8C830DF
:1072A800781885F8D400D5F8C40085F8D520394673
:1072B80004F0CFFFC4F8D06094F8D6309D4DF3B1F8
:1072C800D5F8D830DBB1D5F8DC30C3B1C5F8E0303B
:1072D8001B68994AC5F8E430D5F8E8301344187AA1
:1072E800FDF794FDD5F8E030987908F000FBD5F863
:1072F800E8300133092B88BF0023C5F8E8308F4DEB
:1073080094F8EC202E688B4B002A00F0E481D3F827
:10731800F020002A00F0DF8193F8F430013B012BC4
:1073280000F2D981D4F8F000824F04F08FFFE0B169
:10733800D7F8F00004F087FF97F8F530D5F80090FB
:107348007E2B80460ED102231B2887F8F43009D102
:10735800D7F8F00004F07AFF20B90123C7F8F890B5
:1073680087F8FC3084F8F580DCE7D7F8F8202B683C
:107378009B1A41F6583293421DD9032387F8F430FB
:10738800A9E16F4A32F8130010B903464FF40360BD
:107398000133B0F5C06FDBB275D01DD9B0F5006F01
:1073A8007AD031D9B0F5036F3ED184F8FD30E36B64
:1073B800604F99063FD494F8FC1094F8FD300029EA
:1073C80000F04C812A68921B012ADAD984F8FD3032
:1073D800002384F8FC307EE1B0F5007F42D007D866
:1073E800B0F5807F47D0B0F5887F00F08580E6E76C
:1073F800B0F5806F00F0A880B0F5826F00F0ED80E6
:10740800B0F5047FDBD123E0B0F5E26F00F08480B3
:10741800B0F5E46F00F08580B0F5E06FCFD184F867
:10742800FD30B4F90A1080E0B0F5046F6DD0B0F506
:10743800026FC4D1FCE097F840309A07BBD5B7F883
:10744800421024234B431233642193FBF1F1FFE0F4
:1074580084F8FD303B4B374F1B689B07ABD5BB8D82
:107468000A21F4E084F8FD30364B324F1B681905C9
:10747800A1D5796BECE084F8FD30E36B2D4F5A070A
:1074880099D57969E4E084F8FD302E4B294F1B68C3
:107498001B0590D5B96BDBE0E16B264A84F8FD301B
:1074A8008F0688D592F84010880784D5D90711D55A
:1074B800D36C83EAE371002BA1EBE37101EB51017B
:1074C8004FF01902B1FBF2F1ACBF41F0004141F0BD
:1074D80040410EE0936C83EAE371A1EBE371002B6A
:1074E80001EB51014FF01902B1FBF2F1B8BF41F0C5
:1074F80080414FF400608AE084F8FD30E36B0D4F63
:107508005B077FF558AF3969A2E0B4F9181084F821
:10751800FD30642359437AE084F8FD30B4F90C1047
:1075280003E0B4F90E1084F8FD302C2391FBF3F13D
:107538006DE000BF30140020F480010864240020AE
:107548003CA301084024002084F8FD3094F8FE3064
:10755800624A0133DBB2032B88BF012382F8FE3075
:1075680094F8FE1042F2107359435D4B1B78D8070C
:1075780048BF01319A0748BF02315F07B4F80031AC
:1075880048BF0431D80748BF0A319A0748BF1431A9
:107598001F0648BF2831D80548BF28315A0748BFB9
:1075A80064311F0748BFC831980548BF01F5C87145
:1075B8009A0648BF01F57A71DF0648BF01F5FA61FE
:1075C800580648BF01F57A614FF4806002F04CFE1E
:1075D800424B002283F8FC20EDE6E16BDFF8FC80EB
:1075E80084F8FD3011F0200717D098F8402012F0E9
:1075F800020F14BF4FF47A71002112F0010F14BF6B
:107608004FF4FA6300230B4494F84610194402F02F
:107618002BFE002384F8FC30CDE6324B1B6819069C
:107628007FF5C9AE394602F01FFE88F8FC70C2E645
:1076380084F8FD30E36B294F9A067FF5BCAE97F8C6
:1076480040309B077FF5B7AEB7F844306421594303
:1076580002F00AFE002387F8FC30ACE684F8FD301F
:1076680039E0BB7823B1C5F8C06087F80280C4E56B
:10767800D5F8C030F31AB3F57A6FFFF4BEAD012325
:10768800D5F8C400BB7004F0DEFD0746D5F8C40089
:1076980004F0D9FD7F067FF4B0AD8A2802D08E2889
:1076A8000CD0AAE5EB6B98067FF5A7AD95F8BE3030
:1076B800002B7FF4A2AD05F18D0306E095F8BE30EE
:1076C800002B7FF49AAD05F15803C5F8C8302D2377
:1076D80085F8CC3091E504B0BDE8F087301400207F
:1076E800CF2F00204024002010B5214A18B9136874
:1076F80002221A8210BD1F481468002303802178D3
:1077080011F07F0102460DD1637A990644BF022128
:10771800017013F0400F037814BF43F0010323F006
:10772800010315E0012921D002291ED1637913F044
:10773800800F03F00F034FEA830303F1804303F53F
:10774800B8431B6806D003F03003102B07D1012380
:10775800137004E003F44053B3F5805FF6E7064B7B
:107768001B681B699847034810BD184610BD00BF29
:10777800F421002038150020D420002010B5064C34
:1077880018B9236801221A8210BD044B1B689B6834
:10779800984720680C3010BDF4210020D420002028
:1077A80010B5064C18B9236801221A8210BD044B83
:1077B8001B681B68984720680A3010BDF421002018
:1077C800D420002003788B4283BF034B03EB410195
:1077D80048880020704700BF3815002070B5002287
:1077E8001346244914180C44A47E83EA042308246D
:1077F80013F4004F4FEA430318BF83F4815304F195
:10780800FF3418BF83F0010314F0FF049BB2EFD1DB
:107818000132192AE5D100F1190200F11A050A44CA
:107828000D44967EAA7E02EB062292B29A421FD19E
:10783800104B93F83B50E2B2AA4216D2431C03EB1A
:107848004203DBB2CA1801330B44927E9B7E03EBE2
:1078580002239BB24FF4AF6253431B13064A03F54E
:10786800487322F814300134E5E7012381F83C30ED
:1078780070BD00BF381500203A15002003788B42F0
:107888000BD9074B8900194493F83D20086C02B1C5
:10789800400800F5777080B270470020704700BF3D
:1078A8003815002007299DBF034B03EB8101B1F870
:1078B80070000020704700BF38150020034B03EB11
:1078C8008101D1F89000C0F3CF007047381500202F
:1078D80070B5334C054604F001FBD4F8D030C4F839
:1078E800D000C31AB3F5FA5FC4F8D43082BF0023BE
:1078F80084F8D83084F8D93094F8D8302BB9A12D31
:1079080002BF274A012182F8D91094F8D910244AD5
:1079180029B1D118EDB201338D7682F8D83094F8B8
:10792800D85094F8DA30AB4239D11D4B93F8DB309C
:10793800052B02D0062B03D02CE00020FFF74EFFCA
:10794800E37E1E2B26D100200246C1B26B1E99424F
:1079580019DA21448B7E0821DBB283EA0206F60796
:1079680044BF83F01803C3F3460301F1FF3154BF4A
:107978005B0843F0800311F0FF01C2F34702ECD12A
:1079880001301A46E1E723449B7E9A4202D1032044
:10799800FFF724FF002384F8D93084F8D83070BD6D
:1079A8003815002010B5044604F098FA0F4BD3F8A8
:1079B800DC20C3F8DC00821A41F288318A42C3F81D
:1079C800E02084BF002283F8E42093F8E4200749EC
:1079D80013440F2AE4B218BF013283F8E54012BFFE
:1079E80081F8E420012381F8F53010BD3815002016
:1079F80010B5044604F072FA0F4BD3F8F820C3F818
:107A0800F800821A41F288318A42C3F8FC2084BF08
:107A1800002283F8002193F8002107491344142A0F
:107A280018BF013283F8014112BF81F800210123F8
:107A380081F8163110BD00BF381500202DE9F84334
:107A4800324F3D682A8A2E7AB2B9042E14D1304CAE
:107A580030482378012B0BD12F4B19682F4B89B253
:107A68000B445B0019681A6030230380227048E0D9
:107A780010230380072644E0AC8AAB69A24294BF76
:107A880004260226944228BF14461FFA84F840466A
:107A98009847214A13689BB203F1005303F54053FA
:107AA8005B0004F1010E1B689BB203F1005303F560
:107AB80040534FEA6E0E5B000021714500F1020051
:107AC80009D010F8019C10F802CC4CEA092C23F8D4
:107AD80021C00131F1E71268104B92B213445B00E8
:107AE8001A681C602B8AC8EB03032B826B8A9844A4
:107AF800084BA5F8128030221A80094B4FF44052E7
:107B08001A803B681E72BDE8F88300BFF42100208C
:107B1800D12F0020CE200020505C004002300020F1
:107B2800CC2000200E4B0F4A1B689BB203EBC00011
:107B380002443E294FEA420209D94B09C80604BF4C
:107B480003F1FF339BB29B0243F4004304E04B086C
:107B5800C90748BF01339B0211681360704700BF13
:107B6800505C00400630002010B5454B1A6810786C
:107B780010F07F0004D1537A23F02003537210BD14
:107B880002287AD15388002B78D11379002B75D12C
:107B9800537923F08000840004F1804101F5B84155
:107BA80013F0800F096814BF01F0300101F440514F
:107BB800032862D8002960D0927A002A5DD004F1A7
:107BC800804404F5B8441906226825D502F030022D
:107BD800102A4CD103F07F039B0003F1804303F587
:107BE800B8431A68510641BF196840F60F720A4037
:107BF80042F4004244BF42F0C0021A601A6822F4FC
:107C0800E04222F0400292B282F0300242F4004296
:107C180042F080021A602AE002F44052B2F5805F16
:107C280025D128B9174B93F82C10FFF77BFF11E0EB
:107C38009B0003F1804303F5B8431A68520441BF1F
:107C4800196840F60F720A4042F4404244BF42F0BD
:107C580080021A60236823F4804323F070039BB2E8
:107C680083F4405343F4004343F080032360064BFE
:107C78001B685B699847002010BD022010BD00BF3B
:107C8800F4210020B4000020D42000200023036049
:107C9800436083608381036143618361C3610362DD
:107CA8004362836270478A68036810B50C6A14439C
:107CB8000A6914434A6914438A691443CA69144314
:107CC8004A6A14438A6A23F4FF4323F07003224369
:107CD800134303608B8943600B6883604B68C36000
:107CE80010BD02684FF6FE73134003600023036063
:107CF80043608360C360294B984201D1284A27E03A
:107D0800284B984201D1264A2AE0274B984201D1B4
:107D1800234A2DE0254B984201D1214A30E0244BDB
:107D2800984201D11E4A33E0224B984204D11C4AA2
:107D3800536843F470032EE01F4B984204D1184A4D
:107D4800536843F0706326E01C4B984204D11C4AE8
:107D5800536843F00F031EE01A4B984204D1184AA7
:107D6800536843F0F00316E0174B984204D1144AC5
:107D7800536843F470630EE0144B984204D1104AE0
:107D8800536843F4704306E0114B984204D10C4AFF
:107D9800536843F470235360704700BF08000240E3
:107DA800000002401C000240300002404400024033
:107DB800580002406C000240800002400804024063
:107DC800000402401C040240300402404404024003
:107DD80058040240084BDA68D10709D4DA68D20699
:107DE80008D4DB6813F0040F14BF03200420704785
:107DF800012070470220704700200240036A23F0E8
:107E080001030362036A70B5446882690D6822F44D
:107E1800803222F0730215438A8923F00203134348
:107E28008A881343134A90420FD002F500629042A9
:107E38000BD002F54062904207D002F58062904272
:107E480003D002F5806290420DD1CA89CE8823F012
:107E5800080313430A8A24F4407414434A8A23F01B
:107E68000403334314438A684460856142630362B0
:107E780070BD00BF002C0140994A536803F00C0301
:107E8800042B2DE9F04105D0082B06D09549016057
:107E9800B3B916E0934B036012E053685468C3F318
:107EA8008343991CE30349BFD36A8F4B8D4C03F07E
:107EB8000F0344BF0133B4FBF3F34B43036000E00B
:107EC80000235168894FC1F303117D5C0168EDB24D
:107ED80021FA05F444605668C6F30226BE5D24FA0A
:107EE80006FEC0F808E05668C6F3C226BE5DF6B2C4
:107EF800F440C460D2F82C80C8F3041808F00F0CC2
:107F080007EB4C0C18F0100FBCF810C01FFA8CFCD3
:107F180007D0BCF1000F04D0B3FBFCFCC0F810C0C4
:107F280000E00161D2F82CC0CCF3442C0CF00F080F
:107F380007EB48071CF0100F3F8ABFB204D01FB1EF
:107F4800B3FBF7F7476100E04161176BFF065ABFC3
:107F5800644F87618161176BBF065ABF614FC76164
:107F6800C161176B7F065ABF5E4F07620162176BCC
:107F7800FF0506D5994204D1AE4202D14F004762AF
:107F880000E04462176BFF0406D5994204D1AE4263
:107F980002D14F00876200E08462176BBF0506D5E7
:107FA800994204D1AE4202D14F00C76200E0C462D8
:107FB800176B7F0506D5994204D1AE4202D14F0016
:107FC800476400E04464176B3F0506D5994204D125
:107FD800AE4202D14F00876400E08464176BBF048F
:107FE80006D5994204D1AE4202D14B00C36400E0E9
:107FF8008464156B3A4BAD0701D1046315E01C6B23
:1080080004F00304012C01D101630EE01C6B04F0A1
:108018000304022C02D14FF4004305E01B6B03F06C
:108028000303032B01D12F4B0363146B2C4B14F464
:10803800403F02D1C0F834E018E01C6B04F440342F
:10804800B4F5803F01D1416310E01C6B04F4403467
:10805800B4F5003F02D14FF4004306E01B6B03F474
:108068004033B3F5403F01D11E4B4363146B1C4BA7
:1080780014F4402F02D1C0F838E018E01C6B04F467
:108088004024B4F5802F01D1816310E01C6B04F407
:108098004024B4F5002F02D14FF4004306E01B6BD7
:1080A80003F44023B3F5402F01D10E4B8363146BC7
:1080B8000B4B14F4401F02D1C0F83CE020E01C6BCD
:1080C80004F44014B4F5801F01D1C16318E01C6B9F
:1080D80004F44014B4F5001F0AD14FF400430EE035
:1080E8000010024000127A0000093D001A0000202A
:1080F8001B6B03F44013B3F5401F01D1134BC3634B
:10810800126B134B12F4400F03D1C0F840E0BDE8E6
:10811800F0811A6B02F44002B2F5800F02D10164BB
:10812800BDE8F0811A6B02F44002B2F5000F02D1EB
:108138004FF4004306E01B6B03F44003B3F5400F14
:1081480001D1024B0364BDE8F08100BF00127A0040
:1081580000100240F0B500230E681C460125A5401A
:1081680005EA060EAE452BD10F797A1E012A15D8DD
:10817800856803229A4025EA020282604D79826866
:108188009D4015438560828892B222EA0E02828061
:108198008A798588A2402A4392B2828003220568A0
:1081A8009A40D2431540056005689F402F430760F9
:1081B800C7681740CA7902FA03F547EA0502C260A0
:1081C8000134102C03F10203C8D1F0BD38B52DEDF0
:1081D800048B4A4C0368C4F818318388A4F81C310E
:1081E800013A0D46072A42D8DFE802F0040A1018BF
:1081F80022292F35B4F818310B80B4F81A3113E05E
:10820800B4F81A310B80B4F8183105E0B4F8183115
:108218005B420B80B4F81A315B4205E0B4F81A31BE
:108228005B420B80B4F818316B80B4F81C311DE048
:10823800B4F818315B420B80B4F81A3112E0B4F884
:108248001A310B80B4F818310CE0B4F818310B80EF
:10825800B4F81A3105E0B4F81A315B420B80B4F86F
:1082680018315B426B80B4F81C315B42AB80244B05
:1082780093F83030002B3ED1B5F9003094ED4B0A1D
:10828800D4ED487A09EE103AB5F9023008EE103A02
:10829800B8EEC88AB5F90430B8EEC99A28EE000AD3
:1082A80008EE903AA7EE890AF8EEE88AD4ED4E7AFD
:1082B800A7EEA80A0DF0B6FD94ED4C0AD4ED497A64
:1082C800288028EE000AA7EE890AD4ED4F7AA7EE97
:1082D800A80A0DF0A7FD94ED4D0AD4ED4A7A6880FE
:1082E80028EE000AA7EE890AD4ED507AA7EEA80A6C
:1082F8000DF098FDA880BDEC048B38BD3815002022
:108308001A000020104BDFED117A1B689A89104B78
:108318001B6883F31003D31A07EE103AB8EEC77A36
:1083280027EE277A07EE902AF8EEE77AC7EE277A43
:10833800FDEEE77A17EE900A6428A8BF642020EAC9
:10834800E070C0B2704700BF581400200000C84257
:1083580068140020094B1A68137844F6FB7103EB84
:10836800431300FB03135078C0EB0030B3FBF0F36A
:108378009078B3FBF0F080B2704700BF581400202B
:1083880008B50A4890F8453100EB43030A22B3F8D0
:10839800541189B2A0F85C1100F5B07003F05CFFCD
:1083A80080B2FFF7D7FF024B188008BD38150020B0
:1083B8005C1400202E4B2F4A1B68126810B51A60F7
:1083C8002D4A1168596051689268DA602B4A9960A1
:1083D80011681961516892689A61294A596111684E
:1083E800D961516892685A62264A196211881985BA
:1083F800518859859188D288DA85234A99851188C8
:1084080019865188598692889A86204A1188D98671
:10841800518819871946928821F83A2F1C4A1078F2
:108428000022824206DA1B4C34F8124021F8024F2F
:108438000132F6E7184A1288A3F86420174A12880E
:10844800A3F86620164A1188A3F86C105188928800
:10845800A3F87020134AA3F86E1012689A66124A9D
:108468001288A3F87220114A5289A3F85E2010BD21
:10847800F42C0020B02F0020FC1700200818002042
:108488001418002050140020001200203A14002074
:10849800241900202012002094160020B40F002078
:1084A80006120020441400203C1200200C12002068
:1084B8002DE9F8430E4B93E8800305460E46002449
:1084C800B44213DA7B1933F9140008EB050333F9C6
:1084D800142009EB050333F914301344022293FBEB
:1084E800F2F3C01A09F0B1F80134E9E7BDE8F883FE
:1084F800F42C002070B5472009F086F8174B1B684C
:108508001B0307D5164B174A5B6810681B68C01A0F
:1085180009F08CF8144E154C154D307809F086F892
:1085280023682868C01A09F090F863686868C01A58
:1085380009F08BF80F4B188809F078F80E4B18885B
:1085480009F074F80D4B188809F070F83378237423
:108558002B68A3606B68E36070BD00BF602E0020CD
:10856800F42C0020B02F002076140020E02C0020EE
:108578007814002074140020721400204412002083
:1085880037B51A4B1A4C1B491B4A20B11B480088A7
:10859800B0F5805F21D2164D09881278ADF8041025
:1085A8008DF806209B798DF8073001A8294604220A
:1085B8000DF00EFAC0B101982860532009F024F894
:1085C800208809F033F8A07809F030F8E07809F04D
:1085D8002DF80A4B00221A8006E0098812789B7948
:1085E8002180A270E370E8E703B030BDC82C0020FA
:1085F800201700203015002070140020802E002045
:108608000A4A138801331380094A13680133136037
:10861800084A138801339BB2202B01BF0023138023
:10862800054A138808BF013313807047802E002045
:10863800682E00206C2E00206E2E002038B53A4B94
:108648001B78083B012B05460C466BD8452008F0E3
:10865800DBFF284608F0D8FF0C2D23D004D80A2DBC
:108668000AD014D835B138BD0E2D4BD02ED3FF2DDE
:1086780050D038BD206849E0207808F0C5FF6279FD
:108688006378002A14BF80200020184300E0207877
:1086980008F0BAFFA07808F0B7FFE07808F0B4FF58
:1086A80020793BE0B4F9000008F0B6FFA07808F0A4
:1086B800ABFFE07808F0A8FFB4F9040008F0ACFFBD
:1086C800B4F90600BDE8384008F0A6BF6378207802
:1086D8008BB180F0800008F097FFA468E0B208F042
:1086E80093FFC4F3072008F08FFFC4F3074008F096
:1086F8008BFF200E12E008F087FF6068BDE8384065
:1087080008F0A3BF206808F091FF6068BDE8384012
:1087180008F08CBF054808F055FF0020BDE8384038
:1087280008F072BF38BD00BFD02C00205CA3010840
:108738002DE9F04FBC4B8BB018880193002840F00E
:108748009D80BA4EFFF71CFFFFF734FE34684920BE
:1087580008F05AFFB64B2546186808F067FF55F829
:10876800040B08F063FF284607F09AFD04F1100097
:1087780007F096FD04F11C081027AE4D01232A6866
:10878800BB40134203D0D8F8000008F05EFF013761
:10879800132F08F10408F0D1A74F04F1280007F0BF
:1087A8006FFDB7F84431B4F92E00C01A08F03EFF47
:1087B8002B6813F4805FB84608D0A04BB4F8640067
:1087C8001B88181AC0F30D0008F030FF2B689904B5
:1087D80003D5B4F8660008F029FF2B685A0503D5BD
:1087E80004F16C0007F04CFD2B681B0502D5A06E48
:1087F80008F02BFF2B681F0403D5B4F8720008F0AB
:1088080015FF04F13000274607F03AFD04F1360061
:1088180007F036FDB8F8443137F93C0FC01A08F0B4
:1088280005FF4FF00108864B1B78984509DA37F9A0
:10883800020FB4F93C30C01A08F007FF08F101082C
:10884800F1E72B689D0505D5B4F95E00A0F2DC5070
:1088580008F0FBFE32687B487260B260121A911011
:10886800794A4A43531C032293FBF2F202EB420279
:108878009A1A742303FB020333605DE2734B744A54
:108888001B6811688B4206D00AA9002041F8203DD8
:108898001360FFF7D3FE684A019B92F8CA171B883A
:1088A80092F8CB070B44013BB3FBF0F200FB123309
:1088B8008B4280F00C825D4F0120FFF761FEFFF7CD
:1088C80079FD50203E687D6808F09EFEBA683B68D6
:1088D80010681B687A6803441068A3EB400008F02E
:1088E800B4FE6A6873689B1A0293AA68B3689B1AF5
:1088F8000393EA68F36802A89B1A049307F0D0FC74
:108908002A6933699B1A02936A6973699B1A0393EC
:10891800B369AA699B1A04930023194602AA52F85C
:10892800212002F120003F2842D802F108000F2838
:1089380006D80232032A04D9002B08BF012300E01D
:10894800022301310329E9D1012B02980ED0022B11
:1089580021D0039B03F003039B0000F0030043EACC
:108968000010049B03F0030318430CE000F00F0011
:1089780040F0400008F048FE0498039B00F00F0008
:1089880040EA0310C0B208F03FFE06F11C0B05F1E7
:108998001C0810246FE000F03F0040F0800008F051
:1089A80033FE9DF80C0008F02FFE9DF81000EAE752
:1089B80002224FF0000802AB4FEA880853F8223031
:1089C80003F18001FF2910D903F50041B1F5803F7B
:1089D80002D248F0010808E003F50003B3F1807FF4
:1089E80034BF48F0020848F0030812F1FF32E2D21F
:1089F80068F03F00C0B208F007FE02AC0DF1140A9F
:108A080008F00303022B207807D0032B22D0012B78
:108A180029D108F0F9FD607825E008F0F5FD6078C7
:108A280008F0F2FDA0781EE06C2E0020F42C002047
:108A3800682E0020602E0020A02400205C2E00203C
:108A480024190020002D002035C2724F742E0020FA
:108A5800702E002008F0D8FD607808F0D5FDA078C9
:108A680008F0D2FDE078043408F0CEFD54454FEA12
:108A7800A808C5D189E7B34901220B68A2401A4268
:108A88008A4606D0DBF80000D8F80030C01A08F093
:108A9800DCFD0134132C0BF1040B08F10408EAD1B6
:108AA80006F1260005F12601002331F9024F30F9BD
:108AB800022F121B02AC44F823200133042BF4D1FB
:108AC80003214FF000094FEA89035FFA83F902ABEB
:108AD80053F821206AB102F108000F2802D849F0A2
:108AE800010906E08032FF2A94BF49F0020949F0E3
:108AF800030911F1FF31E6D2484608F085FD00244C
:108B08000DF1080BA04609F00302022A16D0032A29
:108B18001DD0012A38D1B8F1000F05D1DBF800408B
:108B28002401E4B290462FE0DBF8000000F00F00CB
:108B3800204308F069FD4FF0000825E0B8F1000F68
:108B48000CD0DBF80000C0F30310204316E0B8F1A6
:108B5800000F08D19BF8010008F056FD9BF80000B3
:108B680008F052FD10E0DBF80000C0F303302043AA
:108B780008F04AFDDBF80000C0F3071008F044FDD8
:108B8800DBF800402401E4B20BF1040B06AB9B4573
:108B98004FEA9909B7D1B8F1010F02D1204608F080
:108BA80033FDDAF8003013F480541FBFB6F86420A0
:108BB800B5F86410521A029218BF012498040AD515
:108BC8000AAA02EB8401B5F86600B6F86620121A04
:108BD80041F8202C0134590513D502AA02EB840C64
:108BE80006F16A0E05F16A0000223EF9021F30F90B
:108BF800028FC8EB01014CF822100132032AF4D18C
:108C080003341A0508D50AAA02EB8400A96EB26ECD
:108C1800521A40F8202C013418040BD50AAB03EB88
:108C28008402B5F87210B6F872305B1A42F8203C2C
:108C3800013400E0FCB1012C03D1029808F005FDD5
:108C480019E0631E002002AA400052F82320C0B297
:108C58000AB140F00100013BF5D508F0D5FC4FF012
:108C6800000802AB53F8280008B108F0EEFC08F140
:108C78000108A045F5DB30200321FFF719FC362059
:108C88000321FFF715FC304B3C201978FFF710FC47
:108C9800DAF80030990506D5B6F95E00B5F95E3008
:108CA800C01A08F0D2FC3A6828487B687A60121A21
:108CB8009110274ABB604A43531C032293FBF2F2EC
:108CC80002EB42029A1A742303FB02033B60214B16
:108CD8001B681A0630D5204C204D22682B689A4212
:108CE8000BD162686B689A4207D1019B1B88102BD5
:108CF80011D11B4B1B885B060DD1482008F084FC62
:108D0800206808F0A2FC606808F09FFC23682B60CC
:108D180063686B600EE0134A104B11782A7C91420D
:108D280008D1114A99681068884203D15268DB68F3
:108D38009A4201D0FFF7DEFB08F036FC0BB0BDE825
:108D4800F08F00BF602E002024190020002D002085
:108D580035C2724F4024002048120020E02C002029
:108D68006E2E002076140020781400202DE9F84F8C
:108D78000C9E3A4CC2EB030B0B9BF61A6368002956
:108D880014BF4FF0060A4FF0040A01330546904617
:108D980013D1236853455ED2314A324852F8232012
:108DA800032B98BF294608F01DFC636801336360F4
:108DB8002D4B002205461A7113E0002511E02B4ABD
:108DC8001278954240DA0B9BE3B109FB06F2995CF5
:108DD80001228A40264909680A4213D1636801338F
:108DE8006360D4F804900A9B1C4F9945E7DB2BD1AC
:108DF8000A2008F009FC3B6801333B604FF0FF3361
:108E08007B6021E0184A117921B12C2008F0FCFB85
:108E1800013501E001211171226809FB0BF308EB10
:108E2800030752B958F8030008F0CCFB97F904106F
:108E38004B1C0544D2D00F4802E03A440E48117941
:108E480008F0D0FB0544C9E7206850452CBF002036
:108E58000120BDE8F88F0020BDE8F88F782E0020AB
:108E68000881010867A30108201700200C010020D1
:108E7800602E002076A30108AAA40108F0B50124F9
:108E8800B0FBF4F58D4201D34C43F9E70026D4B189
:108E9800B0FBF4F504FB1500B4FBF1F41EB9002D8A
:108EA80001DC002CF3D1092D03F1010EEFB204DD32
:108EB800002A14BF3725572500E030253D441D7092
:108EC80001367346E3E71C70F0BDF0B50124B0FB32
:108ED800F4F58D4201D34C43F9E70026D4B1B0FB39
:108EE800F4F504FB1500B4FBF1F41EB9002D01DC08
:108EF800002CF3D1092D03F1010EEFB204DD002A95
:108F080014BF3725572500E030253D441D70013634
:108F18007346E3E71C70F0BD03685A1C02601970C1
:108F280070472DE9F843089E002B074688461446EB
:108F380014BF4FF030094FF02009334613F8012BC6
:108F48000AB9254603E0002CFBDD013CF6E7002DBD
:108F580004DD38464946C047013DF8E724EAE47491
:108F68003546A01B284415F8011B11B13846C047E7
:108F7800F7E7BDE8F883024B186803F06AB900BF49
:108F8800C00F002090ED017A07EE901AB5EE407AF6
:108F9800F1EE10FA01BFF8EEE77A9FED0E7A67EE70
:108FA800877AB7EE007A04BFC7EE277AC0ED017A58
:108FB80090ED017AD0ED007A30EE877A30EE670ACC
:108FC800C0EE870AE0EE807AB0EE670AC0ED007A5C
:108FD800704700BFDB0FC94010B50278202A03464E
:108FE80000F10100F9D0092AF7D02D2A03D1034650
:108FF800BFEE000A04E02B2A08BF0346B7EE000ABA
:10900800DFED387A1A46134612F8010BA0F1300149
:10901800CCB2092C0AD807EE101AB8EEC77AF2EECD
:10902800046AA7EEA67AF0EE477AECE72E2816D166
:10903800F2EE046A1146B0EE666A0B4611F8012B8F
:10904800303AD0B209280AD807EE102AB8EEC77A03
:1090580087EE267A66EE866A77EE877AEDE71A78E3
:1090680002F0DF02452A35D15A782D2A02D102337F
:10907800012004E02B2A14BF013302330020013BF6
:10908800002213F8011F3039CCB2092C03D80A2466
:1090980004FB0212F5E7B2F59A7F28BF4FF49A72E3
:1090A8001346B7EE007A072B05D9DFED0F6A083BA8
:1090B80027EE267AF7E702F007032BB1F2EE046AEF
:1090C80027EE267A013BF8E7F0EE476A20B1C7EEB3
:1090D800877A03E0F7EE006A67EEA67A20EE270AA1
:1090E80010BD00BF0000000020BCBE4C30B52DED07
:1090F800028B87B0B0EE408A0C220021054603A8F7
:109108000CF081FCB5EEC08ADFED2A7AF1EE10FA98
:10911800CCBF38EE278A38EE678ADFED277A28EE4B
:10912800278A6946FDEEC87A17EE904A84EAE47009
:10913800A0EBE47007F04EFF002CACBF20232D23DA
:1091480068468DF80C300CF0A2FC012807D13023BA
:109158008DF80D308DF80E308DF80F300CE00228A8
:1091680005D130238DF80D308DF80E3004E003283A
:1091780004BF30238DF80D30694603A80CF06AFC53
:1091880003A80CF084FC0338C4B2224603A928467D
:109198000CF0AAFC00232B55284608490CF05AFC71
:1091A80003AB284619190CF055FC284607B0BDEC4E
:1091B800028B30BD6F12033A00007A449AA301086B
:1091C80070B5064615460846B6FBF2F414B12046BB
:1091D800FFF7F6FF05FB1464024B1B5D00F8013B2B
:1091E80070BD00BF9CA301082DE9F04F814689B0EE
:1091F8008A4616461C4600253178002900F0DD8095
:10920800252902D00136484675E07278302A08BF11
:10921800B278A2F1300319BFB71C4FF0000BF71C4E
:109228004FF0010B092B4FF0000819D8A2F13003B9
:10923800D9B2092905D80A2202FB083817F8012BE8
:10924800F4E7A2F16103052B02D8A2F1570305E068
:10925800A2F14103052B03D8A2F137030A2BEADD5B
:109268006C2A31D13A78642A07F1010600F083802C
:109278000BD8252A3DD003D8002A00F09E80BBE7F2
:10928800582A0CD0632A19D0B6E7732A22D002D8FC
:109298006E2A37D0B0E7752A5CD0782AACD1271D62
:1092A8002068A2F1580462424FF01001624155E073
:1092B8002CD9582A32D0632A2AD13E4648462178EA
:1092C800271DD04701350FE0642A64D00ED9732AD0
:1092D80014D13E462368009348465146424600232F
:1092E800FFF71FFE271D05443C4685E7252ADFD1E9
:1092F8003E4648462521D04701357DE70AD86E2AE3
:1093080006D13E46236804341D6075E7002A54D010
:109318003E4671E7752A26D0782AF9D1A2F158037A
:1093280004F1040C5A422068CDF80CC04FF010012B
:109338005A4105ABFFF7A2FDDDF80CC03E46644676
:1093480005AB00934846514642465B46FFF7E9FDA8
:10935800054451E72068271D0A21002205ABFFF7C5
:10936800B4FD3C46ECE704F1040CCDF80CC02068D1
:109378000A210022DDE72068002804F1040708DA42
:109388002D238DF8143040420DF115030A210022D7
:10939800E5E705ABFAE72068002804F1040C0ADACF
:1093A8002D238DF8143040420DF11503CDF80CC073
:1093B8000A210022BEE705ABF8E7284609B0BDE858
:1093C800F08F0EB40FB505AB019053F8042B064986
:1093D800039301A8FFF708FF019B00221A7004B04D
:1093E8005DF804EB03B07047218F00080FB413B584
:1093F8000B4904AB08680B4953F8042B096801931F
:10940800FFF7F2FE0446084B186802F016FF002822
:10941800F9D0204602B0BDE8104004B0704700BF44
:109428008401002080010020C00F002080EAE07342
:10943800A3EBE0738B4206DB002801DD401A70477E
:1094480002D00844704700207047FDEEC07A17EE3E
:10945800903A2033402B43D8DFED237AB4EEE70A65
:10946800F1EE10FA04DDDFED217A30EE670AF3E75A
:10947800DFED1F7AB4EEE70AF1EE10FA04D5DFED5E
:109488001B7A30EE270AF3E7DFED1A7AB4EEE70A23
:10949800F1EE10FA04DD30EE670A37EEC00A0AE092
:1094A8009FED157AB4EEC70AF1EE10FA44BF30EE1C
:1094B800270A37EE400A60EE007ADFED106A9FED6A
:1094C800107AA7EEA67ADFED0F6AE7EE876A9FEDBE
:1094D8000E7AA7EEA67A20EE276AA6EE070A70474C
:1094E8009FED0A0A704700BFDB0F4940DB0FC940F8
:1094F800DB0F49C0DB0FC93FDB0FC9BF9A7C2E3693
:10950800FAAF4FB93587083CA4AA2ABE000000006C
:10951800DFED027A30EE270A97E700BFDB0FC93F7D
:1095280038B52DED068B90ED008AB0EE480A0C4652
:109538000546FFF7EDFFB0EE40AAB0EE480AFFF788
:1095480084FFD5ED018AB0EE409AB0EE680AFFF7C5
:10955800DFFFB0EE408AB0EE680AFFF776FFD5ED80
:1095680002AAF0EE408AB0EE6A0AFFF7D1FFF0EEE9
:10957800409AB0EE6A0AFFF768FF60EE0A6A69EE81
:10958800297AF0EE665AE7EEA85A29EE8A6A29EE99
:10959800007A69EE889A29EE489A28EE400A28EE61
:1095A8000A8AC4ED035AF0EE465AE7EE685AE6EE28
:1095B800A87AA6EE687AC4ED009AC4ED028A84ED12
:1095C800059A84ED088ABDEC068B84ED010AC4ED8A
:1095D800045A84ED067AC4ED077A38BD10B52DED2E
:1095E800048B8AB090ED009AD0ED028A90ED018A42
:1095F8000446084601A9FFF793FFDDED047A9DEDC7
:10960800017A68EE277AE9EE077A9DED077AE8EEA7
:10961800877A9DED027AC4ED007ADDED057A68EE71
:10962800277AE9EE077A9DED087AE8EE877AC4EDA5
:10963800017ADDED067A28EE278ADDED037AA9EEB8
:10964800278ADDED097AA8EEA78A84ED028A0AB096
:10965800BDEC048B10BD074B1A8822EA000090422B
:1096680010B518801C4602D0012002F01FFC20888B
:1096780010BD00BF30150020064B1A8810439042D9
:1096880010B518801C4602D0012002F00FFC20887B
:1096980010BD00BF30150020024A936823EA00007D
:1096A80090607047A024002008B5104B1A7800235A
:1096B800D9B2914207D20E4951F823100968002007
:1096C80008600133F4E7322002F02DFC094B1B68D7
:1096D8005A0309D5084B9B685B0305D440F2DC505C
:1096E800BDE8084002F01FBC08BD00BF24190020D7
:1096F800F418002040240020A0240020454A6923B3
:109708002DE9F34113704FF4FA635380BE231371AC
:10971800EF2382F8CD37002382F8CE371946164654
:10972800F25C0133B3F5FA6F81EA0201F8D1394BE3
:1097380083F8CE17384B1A69120604D5374A5A608F
:1097480002F188325A6004270020013F17F0FF0712
:109758004FD0314B3422DA60002444B1002356F84C
:109768000480019306F016FE0428EED117E006F0F7
:1097780011FE0428E9D1284D2B6943F002032B611F
:10978800274B6B612B6943F040032B6106F002FE07
:109798002B69042823F002032B61DFD0D5E71E4D87
:1097A8002B6943F001032B6104F1006303F57E3359
:1097B8001FFA88F21A8006F0EDFD042810D1194B23
:1097C80023440193019B4FEA1848A3F8008006F050
:1097D800E1FD2B69042823F001032B6105D0B4E7D0
:1097E8002B6923F001032B61AFE70434B4F5FA6F5A
:1097F800B3D1094A1369042843F08003136102D1E5
:1098080007F012FC10B90A2002F0D2FC02B0BDE841
:10981800F08100BFA02400200020024023016745FA
:1098280000F8030802F8030810B50E4C206802F08F
:109838008FFA2068047A002202FB02F3193B634383
:1098480003F6C4135343192193FBF1F3064921F896
:1098580012300132072AEFD10449BDE8104002F066
:109868002DBA00BF40120020900F0020E4250020F0
:109878002DE9F04107F0D8FB10B90A2002F098FC56
:10988800A44CA549A54D4FF4FA6220460CF0B0F857
:1098980094F8A437022B84BF002384F8A43794F8E3
:1098A800A4274FF4CC7101FB02F3E018234400F520
:1098B8003770286093F8300303F54A73022801FBD8
:1098C800024284BF0020187292F83033944A137011
:1098D8000C2202FB0343934A03F2A6731360A368A6
:1098E80046F209021A401AB98A4A43F400539360AF
:1098F800A368D80703D54FF40050FFF7CDFEA3683F
:10990800590409D50820FFF7C7FE4FF40050FFF7A8
:10991800C3FE0120FFF7C0FEA3681A0706D54FF45F
:109928000050FFF7B9FE0120FFF7B6FEA3689B04BD
:1099380002D54020FFF7B0FE94F8D421754B2AB128
:1099480093F8D82112B1002283F8D821764B774EAC
:109958001E604FF0000C674604EB0C03B3F8ECE113
:109968004FEA5E0101F077314FEA9E0303F033338B
:10997800C1EB0E00C11A4FEADE0303F01133CB1A14
:1099880003EB23131EF0010803F00F324FF0FF031F
:1099980092FBF3F3C3EB032318BF0137A2EB0303D6
:1099A80018BFFFB2012B0ADD022B40F0B080B8F1DE
:1099B800000F00F0AC801EF0BC0F00F0A8800CF186
:1099C800080CBCF1200FC7D1013F012F00F29F8086
:1099D800FFF72AFF302200215548564F0CF013F8A4
:1099E800554BD5F800801F60544B002108F17900D1
:1099F800C3F8008002F0ECF9514B80F001001870B8
:109A0800504B07F126021A604F4B07F1C8021A6043
:109A180098F8000002F058FE28684C4B00F5C57213
:109A28001A60FDF733F84A4BDFED4A6A07F18C02FA
:109A38001A60494B00221A809A71484B07F12C0290
:109A48001A602B68464A93ED187A03F219111160CF
:109A5800444A03F289111160434A07F10801116071
:109A6800424A1760424A07F194011160414A07F1DE
:109A78009E0111604049536167EE266A0E60B6EE9A
:109A8800007AB4F8661187EE267A101D07EE901A50
:109A9800B4F86811F8EE677AC2ED027A07EE901A08
:109AA80093F85C10117193F87810517194F8D711EC
:109AB8001174F8EE677AB3F81611C2ED037A07EE5F
:109AC800901A2E492E4A086003F1640111602D4A4C
:109AD8002D4982ED007AF8EEE77A9FED2C7A2C4A30
:109AE8000B60C7EE277A2B499FED2B7A67EE877AB2
:109AF800C2ED007A03F168020A60284903F21113E3
:109B08000B60274B1F60274B1A60BDE8F08106F0F9
:109B180015FC5DE7A024002000F803081C120020B3
:109B2800B021002040120020E42E00202A26002028
:109B380004100020E4250020381000203C100020EC
:109B48001400002054080020780600204810002047
:109B5800F00F0020DB0F4940C82C0020AC08002083
:109B6800C41A0020C00A0020F0190020F4190020AF
:109B7800D409002028170020980A0020DC080020BB
:109B88001409002010090020280800200000614462
:109B9800D00900201C0800204C3D0F44C0090020BB
:109BA800C80900201807002008B5FFF7A7FDFFF730
:109BB8005FFE0120BDE8084002F078B908B5084802
:109BC8000BF065FFC0B209280246054B04DC0130E2
:109BD8002021C0B29954F6E700221A5408BD00BFEC
:109BE8006117002008B507480BF051FFC0B21428D0
:109BF800044B04D8421C20211954D0B2F7E70022A4
:109C08001A5408BD611700202DE9F74FA74C02F040
:109C180065F926686568A768861BF643451BC71B58
:109C2800ED43FF43F60F8046ED0FFF0F2EB93FB906
:109C3800002D00F08682B9462CE04FF0000929E09B
:109C4800B14627E003EB8A0BBBF802301A050ED4A5
:109C580013F4805F1DBF964A9BF801101268954A5D
:109C6800954B14BF52F82120126843F82A20BBF8FC
:109C78000230D80516D499050AD5904B1B7813F0F5
:109C8800040F0CBF8E4A8F4A8B4B126843F82A2068
:109C980009F10109207B8C495FFA89FA82450B6832
:109CA800D0D326E0894A5046594604F0F5FE884B41
:109CB8001B885A0603D550465946864A16E0580767
:109CC80003D550465946844A10E0190703D5504633
:109CD8005946824A0AE09A0703D550465946804AAF
:109CE80004E0DB07D4D57F4A5046594604F0D4FE39
:109CF800CEE7DFF808E20093BEF906307822A3F534
:109D08007A7353434FF47A7293FBF2F303F22B13F3
:109D180001930022F3465FFA82FE864517D2009B24
:109D280003EB820EBEF802E01EF4806F0DD0DFF860
:109D38008891019B39F822E040F2671A9E449EFB05
:109D4800FAFC0AFB1CEE29F822E00132E3E74DB3E6
:109D580008F5C333A0336360637B544A13BB937322
:109D6800614B1B6813F0020F0AD0DFF894E19EF8EC
:109D780000E0BEF1000F03D04FF0010E82F80EE0B4
:109D8800DA0506D5594B5B791BB1A37B43F0020377
:109D9800A3734A4B1B7813F0050F02BFA37B43F054
:109DA8000403A37394F80EE0BEF1000F03D13F4BF8
:109DB8005B7B002B4FD094F80DC01CF0010FACF169
:109DC8000C031DD1BCF1030F07D8DFF8E8903C4A1B
:109DD8001EF0040F08BF4A4600E0364AACF1040CF6
:109DE800BCF1070F05D8DFF81CC11EF0010F18BF22
:109DF8006246DBB2032B0ED81EF0020F3C4B06E086
:109E0800DBB2032B06D82F4B2A4A1EF0020F18BFCD
:109E18001A4600E0274A4FF0000C5FFA8CF38342A1
:109E28000DD20B6803EB8C035B881B0642BF224BE9
:109E3800D2F8009043F82C900CF1010CEDE785B1B5
:109E4800BEF1000F08D0637B184A0133DBB2142B34
:109E580006D1002304E025B1637B002BF3D100E099
:109E68005373002E52D0234AB2F90250B2F900209F
:109E7800002DB8BF6D42002A4FF03203B8BF5242DE
:109E880095FBF3F592FBF3F2EDB2D3B2AB4238BFD8
:109E98002B46194A13B192FBF3F300E013464344EF
:109EA8002360E37B014A7BBB01232EE0401700209F
:109EB800C01A0020D8A001080A0F0020CF2F0020C8
:109EC80014A0010804A00108C81A00202081010874
:109ED80030150020268101082C81010832810108F3
:109EE800388101083E81010840240020C82C002048
:109EF8001CA0010850140020400D03007C24002001
:109F0800BC14002024A001080023D3738E4D8F4B6E
:109F18002D78E27BADB9002F00F00E818C4B267BAB
:109F28001A788C4B8C4D93F800C08C4BD3F800E01A
:109F38000B6802F004020021D2B203EB86060F463A
:109F4800B5E01AB9864A1A61002508E0854AFAE799
:109F58000A68AB00D6187688760604D40135EBB2C9
:109F68008342F5D3D7E7804EB6F90060192E25DD78
:109F780012F803E094F814C026690EF00F09E145C1
:109F88000CDCDFF8C8C19CF815C0BCEB1E1FDEBF97
:109F9800DFF8D8E1D6F800C043F80EC012F803E0A5
:109FA80094F816C00EF00F09E14533DBDFF89CC1C9
:109FB8009CF815C0BCEB1E1F2CDC26E0193629DAEC
:109FC80012F803E094F814C026690EF00F09E14571
:109FD8000CDCDFF878C19CF817C0BCEB1E1FA2BFD1
:109FE800DFF888E1D6F800C043F80EC012F803E0A5
:109FF80094F816C00EF00F09E1450BDBDFF84CC1F1
:10A008009CF817C0BCEB1E1F04DBD6F800E0574EC7
:10A0180043F806E0544EB6F90260192E1BDD12F81B
:10A0280003C094F814E026690CF00F09F1450CDC24
:10A03800DFF8189199F81590B9EB1C1FDEBFDFF80F
:10A048002CC1D6F8009043F80C90D25C02F00F0CAB
:10A05800F4451EDD82E7193680DA12F803C094F859
:10A0680016E026690CF00F09F1450CDBDFF8DC90EF
:10A0780099F81590B9EB1C1FDEBFDFF8F0C0D6F8D1
:10A08800009043F80C90D25C02F00F0CF445FFF6F8
:10A0980065AF94F817E0BEEB121FA2BF334A3668CB
:10A0A8009E505BE75888000504D404330435B34256
:10A0B800F8D122E04AB101EB0C0A06209AFBF0F92C
:10A0C80000FB19A001280DDC01E057B9012793F81E
:10A0D80001900EEB89003EF829A090F80290C07814
:10A0E80003E01746002081468246013125F802AC7C
:10A0F80085F800906870C9B2D7E7164A1378013B13
:10A1080013F0FF0308BF06231370114B1B785B077E
:10A1180041BFBBF90630A3F57A7303EBC3034FF4D1
:10A128007A7243BF93FBF2F30133DBB20123104A87
:10A1380092FBF3F34344A36003B0BDE8F04FFAF792
:10A1480087BB03B0BDE8F08F3A2F002040170020EE
:10A15800CF2F00204C0000200C0F0020C01A002038
:10A1680020A00108D8A00108501400200A0F0020E0
:10A17800400D030030B50028104C114AB8BF4042CA
:10A188003C2590FBF2F304FB030068430D4D90FB64
:10A19800F2F22D682D7B25B903EB830303EB8303D0
:10A1A80001E0C3EB031302EB83030B8004FB020201
:10A1B8004FF47A7392FBF3F24A8030BD806967FFEF
:10A1C8008096980060140020022803D0431E58424D
:10A1D80058417047064B1B681B7823B1054B18681C
:10A1E800C0F3C0407047044B1878C0F38000704734
:10A1F80078060020E0110020CF2F0020A0F17D0379
:10A20800012B70B504460D460A4E05D830687D21ED
:10A2180002F01FF884F020043068214602F019F893
:10A2280035B12B881C4404EB142404F0FF042C8063
:10A2380070BD00BF2015002010B50A4C5E280146ED
:10A24800206805D15D2102F004F820683E2105E070
:10A258005D2903D101F0FDFF20683D21BDE81040D4
:10A2680001F0F7BF5817002030B585B004AC0025C1
:10A2780024F8025D0091ADF8060021461020FFF792
:10A28800BDFF9DF806002146FFF7B8FF9DF80700BF
:10A298002146FFF7B3FF9DF800002146FFF7AEFF08
:10A2A8009DF801002146FFF7A9FF9DF8020021460D
:10A2B800FFF7A4FF9DF803002146FFF79FFF9DF8D5
:10A2C8000E00C043C0B22946FFF798FF05B030BD65
:10A2D80010B5054C206801F0B9FF18B1206801F0ED
:10A2E800B2FFF6E710BD00BFF414002010B5044615
:10A2F800C0B2FFF7A1FFC4F30720BDE810409BE7F9
:10A30800024B5E21186801F0A4BF00BF5817002057
:10A3180038B5064C05465E21206801F09AFF206892
:10A328002946BDE8384001F094BF00BF5817002007
:10A3380013B5044601A90068FFF71CFF1320FFF7B7
:10A34800E7FFBDF90400FFF7D1FF1B20FFF7E0FF8F
:10A35800BDF90600FFF7CAFF2320FFF7D9FF2368DE
:10A36800002BB4BF53204E20FFF7C0FF01A960683F
:10A37800FFF700FF1220FFF7CBFFBDF90400FFF73E
:10A38800B5FF1A20FFF7C4FFBDF90600FFF7AEFFBF
:10A398002220FFF7BDFF6368002BB4BF572045207C
:10A3A800FFF7A4FF02B010BD674B73B51878674D6F
:10A3B800FFF70AFF2B788342044620D0C8B1644BCC
:10A3C8001B68E3B193F9000002230093614B1B68FB
:10A3D8005B78003318BF0123019304214FF416530F
:10A3E800002201F0AAFD5C4B186040B101232B70DC
:10A3F80005E0594E306803F072FC34602C70574BFE
:10A40800574D1878FFF7E0FE2B788342044618D0A2
:10A4180088B1544B1B68A3B10022012493F90000B2
:10A4280000944FF496430192082101F086FD4E4BAB
:10A43800186028B905E04C4E306803F050FC3460D1
:10A448002C704A4B4A4D1878FFF7BEFE2B78834292
:10A4580004462E4642D0002837D0464B1A68002AB8
:10A468003CD0D37992F90000434C002B08BF02235B
:10A4780002220092002254F823300192102101F0A8
:10A488005CFD3E4B0546186040B33D4C94F84A309D
:10A49800022B0BD094F89620022A01D14C3405E007
:10A4A80023B1002A04F14C0418BF0024354B1C606A
:10A4B80044B1204600214C220BF0A5FA0223256066
:10A4C80084F84A300123337008E02C4E306805F0D8
:10A4D800D1F9306803F003FC34602C702A4B2B4D03
:10A4E8001878FFF771FE2B788342044629D000B311
:10A4F800274B1B682BB3274A93F900001268527840
:10A50800002A0CBF082209220323009301924FF46A
:10A5180061432021002201F010FD1F4B186080B11B
:10A528001E4A012313702B701D4B1A681D4B1A60AD
:10A5380007E0194E306803F0D2FB184B34601C70EA
:10A548002C7002B070BD00BF8006002030140020BF
:10A558007C06002060140020581700208806002080
:10A568008014002084060020F414002094060020A3
:10A578000615002090060020E89B01080815002019
:10A58800602200200C150020A00600201C150020C9
:10A598009C06002098060020201500202415002085
:10A5A8006424002028150020642928BF6421F8B5F8
:10A5B80010FB01F56424064695FBF4F40027E4B289
:10A5C800FBB2A34204D29F2006F0BDF80137F7E79B
:10A5D800B4420BD2C4EB84101421C4EB800095FB69
:10A5E800F1F5663D2844C0B206F0ADF80134E4B296
:10A5F800B44201D29A20F7E7F8BD2DE9F743934C0E
:10A6080001F06CFC6368C31A002BC0F2618300F58B
:10A61800433303F5A07363608D4B1D78237AC5F32C
:10A628008005EB1A18BF012325724DB1002B00F0ED
:10A638004F83884B5A789A7001225A701A702BE00F
:10A64800844A2BB1D37843F00203D37093785370C4
:10A65800D67806F0020101F0FF0339B97D4989680F
:10A66800411A002903DB06F0010300E0012303F08F
:10A678000107784917707BB1F2070DD50A790132C5
:10A68800D2B20523B2FBF3F303EB8303D31ADBB295
:10A69800714A0B71D35C4B706E4EDFF808823378C9
:10A6A8007BB3F37823F00203F3706C4B0344AE20C2
:10A6B800B36006F06CF808B106F06EF888F8000090
:10A6C800002800F00583B02006F061F8402006F06D
:10A6D8005EF8002006F05BF8102006F058F84FF4FA
:10A6E8008067013F0020BFB206F028F8002FF8D19C
:10A6F800384606F0C0F87278594B53F8220006F035
:10A708003DF898F80030002B00F0E2827378062BB1
:10A7180000F2B382DFE813F00700B10218007800F6
:10A728006C018901EE014F494F4A504B5048FEF7E2
:10A7380048FE012006F09FF84D4806F01FF8022059
:10A7480006F099F84B48AEE14B4F3B689B0735D56F
:10A75800DFF85481DFF85491B8F8001044480A2310
:10A76800B1FBF3F203FB121399F80010009192B2B7
:10A7780042499BB2FEF725FEFFF734FA012006F0A6
:10A788007AF83B4805F0FAFF3D4B99F80020186825
:10A79800B8F80030067906FB123164234B43C178C0
:10A7A8008E1B56430220B3FBF6F6F6B206F063F8AA
:10A7B80031461520FFF7F8FE032600E001263B6826
:10A7C8001F0540F15A822F4B2F491F6809680091D5
:10A7D80064232E4997FBF3F2254803FB1273FEF717
:10A7E800F0FDFFF7FFF9304606F045F8204805F080
:10A7F800C5FFFDF787FD0746701C06F03CF81520DD
:10A808003946FFF7D1FE38E20120214F06F033F830
:10A81800204805F0B3FF3B68980749D51E4A1448FD
:10A82800B2F90210B2F900300091B2F904201B49C4
:10A8380001921B4AFEF7C5FDFFF7D4F9022006F086
:10A848001AF80B4805F09AFF032632E05817002043
:10A85800CF2F0020801A0020C1A30108404B4C00D4
:10A8680044810108C6A30108CFA3010859A2010821
:10A8780061170020D6A3010840240020DDA30108A9
:10A88800581400206414002068140020F5A301085F
:10A898006C1400200AA401083A14002020A401081E
:10A8A8002FA40108F10200205C14002001010020FF
:10A8B80002263B68D9071AD57C4A7D48B2F90210AE
:10A8C800B2F900300091B2F904207A4901927A4A2B
:10A8D800FEF777FDFFF786F9304605F0CCFF7448A0
:10A8E80006F1010805F04AFF5FFA88F846463B681A
:10A8F8001A0718D5714A6E48B2F90210B2F9003039
:10A908000091B2F904206B4901926D4AFEF759FD96
:10A91800FFF768F9304605F0AEFF6548771C05F08B
:10A928002DFFFFB23E46674A6249B2F90030B2F9DC
:10A9380002200092644A5E48B2F900200192634AFC
:10A94800634FFEF73EFDFFF74DF9304605F093FFE4
:10A95800574805F013FF97ED000A5548FEF7C6FB68
:10A9680053480BF094F806F101085FFA88F8C0B272
:10A97800B946092809D8431C2044DBB22022427278
:10A98800E218002191721846F3E7494F99ED010A40
:10A998003844FEF7ABFBFFF725F9404605F06BFF9F
:10A9A800384605F0EBFE99ED020A3846FEF79EFBA5
:10A9B80038460BF06CF80236F6B2C0B2092809D84E
:10A9C8002318421CD2B220215972A318002199726F
:10A9D8001046F3E73F4AB2F9003000EE103A384427
:10A9E800B8EEC00AFEF782FBFFF7FCF8304657E0E6
:10A9F8000026394F3B78B34240F23F810E2E00F0DB
:10AA08003C817008013005F036FF304606F0BCFA8C
:10AA18003B78B34206D9202005F095FE701CC0B2E1
:10AA280006F0B2FA0236F6B2E3E72C4E2C4996F855
:10AA3800A4271F48FEF7C5FC012005F01CFF1C4891
:10AA480005F09CFE274B28491F7819483A46FEF71F
:10AA5800B8FC022005F00FFF154805F08FFE0C2307
:10AA680003FB0766214996F8A72796F8A6371048EA
:10AA7800FEF7A7FCFFF7B6F8032005F0FCFE0C482C
:10AA880005F07CFE96F8AC1796F8AA2796F8AB372F
:10AA9800074800911649FEF794FCFFF7A3F8042035
:10AAA80005F0E9FE024805F069FEE6E00012002024
:10AAB8006117002020A4010833A401080612002011
:10AAC800AABB0108362400204814002037A4010836
:10AAD800EC080020F8080020382F0020A0240020CF
:10AAE8003BA40108B021002047A4010858A401088C
:10AAF80069A40108784B1B681B0640F1BA80236AD9
:10AB0800616A764A8B421FBF536292F8283001333C
:10AB180003F003034FF001014FF0000018BF82F863
:10AB2800283005F0B4FE94F828306D4AD05C05F062
:10AB38000AFE0220012105F0AAFE0026694B9B5D52
:10AB48003620C3EBC30393FBF0F0C0B2062828BF3E
:10AB580006206038C0B2013605F0F5FD102EEDD1A3
:10AB6800614B62491B78624813F0020F614B1A78F7
:10AB780014BF59234E23FEF724FCFFF733F80220B5
:10AB880005F079FE5A4805F0F9FD5B495B4B4E68C4
:10AB98000A68574892FBF3F2594996FBF3F3FEF71C
:10ABA80010FCFFF71FF8032005F065FE5048554ECE
:10ABB80005F0E4FD544B55491A884D48FEF701FC51
:10ABC800FEF7FCFF042005F056FE494805F0D6FDC7
:10ABD8004F4B50491A884648FEF7F3FBFEF7EEFF45
:10ABE80004210A2005F053FE414805F0C7FD4A49F3
:10ABF800E26A3F48FEF7E5FBFEF7E0FF052005F0B7
:10AC08003AFE3B4805F0BAFD7268B36843493848D4
:10AC1800FEF7D7FBFEF7D2FF05210A2005F037FE25
:10AC2800334805F0ABFD3369F2683D493048D21A24
:10AC3800FEF7C7FBFEF7C2FF062005F01CFE2C48F6
:10AC480005F09CFDB26837492948FEF7BAFBFEF7C4
:10AC5800B5FF06210A2005F01AFE254805F08EFDED
:10AC68003149234815220AF03FFFFEF7A7FF0720C6
:10AC780016E7F37843F00203F3704DBB2B4B9B7937
:10AC8800032B9BBF2A4A9B183F251D7F00211220BA
:10AC980005F0FDFD284605F056FD1320002105F0BE
:10ACA800F6FD244B1B78002B14BF5220212005F001
:10ACB8004AFD1420002105F0EAFD94F83050084BB5
:10ACC800585D013505F0030505F03DFD84F8305069
:10ACD80003B0BDE8F08300BF4024002058170020CF
:10ACE8007BA401088D1200207014002080A40108A4
:10ACF80061170020761400207814002080969800B0
:10AD080091A401082C080020721400209EA40108B8
:10AD180044120020A6A40108ADA40108B4A40108A7
:10AD2800BDA40108C4A4010838030020C82C0020D1
:10AD3800448101083A2F00202DE9F04F2DED028BB8
:10AD480085B007460293A04B1B889807934636D5D3
:10AD5800109B9E48DC89B0F900301B1B03F2F315E9
:10AD680040F2E632954203D8002BB8BF5B4201E0BF
:10AD78004FF4FA73B0F90220121B02F2F31440F2F6
:10AD8800E630844203D8002AB8BF524201E04FF4AB
:10AD9800FA729342B8BF1346C3F5FA73052293FBC0
:10ADA800F2F30A22643B53433A7FD210534364229E
:10ADB80093FBF2F3134423EAE373DBB200E064236A
:10ADC8000093CB1C0193B8460024019BDFF824A212
:10ADD80013F8016F0193022C4FEA440905D1BAF91F
:10ADE80004301B365E43761146E079493AF8142060
:10ADF80031F91410022012FB0011CBF1000291422C
:10AE080003DB59450A46A8BF5A467249029B31F9E5
:10AE18000950551B33F91420154406F01DFC88B160
:10AE280007EE905A6C4AB8EEE70AB2EE048A105D53
:10AE380080EE080A05F094FE20EE080AFDEEC07ABE
:10AE480017EE905A604A1288D10712D43AF909309D
:10AE58001B365E4393074FEA26160DD5BB7C5D4330
:10AE68009DF900305D43642395FBF3F506EB251649
:10AE780002E03E7A75432E11584B042533F9093008
:10AE880093FBF5F5564BE25C924698F80120751B4A
:10AE980051466A434A43642192FBF1F297F85110F4
:10AEA800D21108EE102AA9B1022CB8EEC80A08D1AE
:10AEB8004A0803D09142A8BF114600E00121494841
:10AEC80002E0181D00EBC400D3ED070AFEF75AF89C
:10AED800BDEEC08ADFF808E1434B98F80B6018888C
:10AEE8000EF1200300FB05F253F82410D21206FBE2
:10AEF8000216B6F5001F3D4AA8BF4FF40016964249
:10AF0800B8BF16460EF12C0243F8246052F82430DC
:10AF180042F82450EB1A0EF138014FF6FF7200097F
:10AF2800B2FBF0F043430EF1440051F8245050F8BE
:10AF3800242040F824509B112A4441F8243097F8E3
:10AF480050101A444FEA840C761300EE102A79B197
:10AF58000EF15000B8EEC00A00EBC400DEED070A9F
:10AF6800CDF80CC0FEF70EF8DDF80CC0BDEEC00A37
:10AF780098F8153010EE102A18EE101A5A43534656
:10AF880053431A463144642392FBF3F3184A1B12C5
:10AF9800194422F8091018EE100A02F108010134C8
:10AFA8004CF8010002F114012032032C4CF8016026
:10AFB8004CF8023008F101087FF407AF05B0BDEC8A
:10AFC800028BBDE8F08F00BF301500207C240020E4
:10AFD800C82F0020362400206481010800120020B8
:10AFE8008C170020A0170020D41100200000E0FFDB
:10AFF800F4170020501400202DE9F04F2DED028B9E
:10B0080087B000260593C54B0491B3F90280B3F9C4
:10B0180000300392B8F1000FB8BFC8F10008002B48
:10B02800B8BF5B429845B8BF9846B8F5FA7F07465F
:10B03800A8BF4FF4FA780090B1460196B34634465B
:10B04800B74D2B88990758D0B44BB64A33F814300B
:10B0580032F91420022013FB0022039B5B429A4220
:10B068004FEA440103DB039B9342A8BF1346AE4A51
:10B0780031F902A0059A32F91420CAEB030303EB55
:10B08800020A06F0E9FA88B107EE90AAA74BB8EED3
:10B09800E70AB2EE048A185D80EE080A05F060FD42
:10B0A80020EE080AFDEEC07A17EE90AA3B7A6422D9
:10B0B80003FB0AF393FBF2F33A7F6FF0040101FB01
:10B0C80002FB5B4505DB02EB82029342A8BF1346F5
:10B0D8009B46974A52F824100AEB010342F210717A
:10B0E8008B42A8BF0B4693498B42B8BF0B4642F828
:10B0F8002430BA7C53431B1301932D8805F00303B6
:10B10800012B38D0854B8C4933F91490009B51F8AA
:10B1180024E093F801C0894B33F9140080EAE07306
:10B12800A3EBE073B3F5206F4FEA840616DC09EB56
:10B1380089031A0192FBFCF3042290FBF2F0181A1F
:10B148008644BEF57A5FA8BF4FF47A5E7C4B9E4575
:10B15800ACBF41F824E041F8243002E0002341F874
:10B1680024308B597D2693FBF6F6009BDB7A7343DC
:10B17800402693FBF6F6AA0711D5019BC8F5FA728B
:10B1880008FB09F008FB06F54FF4FA7102FB0B0007
:10B1980002FB035590FBF1F095FBF1F505E0EB0799
:10B1A8004DBF019D354648465846644B33F9142037
:10B1B800042392FBF3F3634A02F19C014FEA440A29
:10B1C800615C4B436FF04F0193FBF1F397F851101B
:10B1D800C31808EE103A51B1101DB8EEC80A00EBBA
:10B1E800C400D2ED070AFDF7CDFEBDEEC08ADFF838
:10B1F80054E1524B0EF1A0013AF803003AF901303C
:10B208002AF8010002B20EF1A4010EF1AC00D31A23
:10B21800042293FBF2F2A30051F824C0029350F8E1
:10B22800243041F82420634497F8501040F824C093
:10B23800134400EE103A59B10EF15000B8EEC00AAE
:10B2480000EBC400DEED070AFDF79CFEBDEEC00A68
:10B258003C4A02F1B40110EE103A095D01FB03FE0D
:10B2680018EE101A02F1680029444FF0200C9EFBDA
:10B27800FCF3C91A2AF80010029902F1700E084668
:10B2880018EE101A40F80E1002F17C015B4245508E
:10B2980002F188014350009B013300930CB901244B
:10B2A800CEE61E4B946AB3F90410049B9B790F33C6
:10B2B8005B004B435B112149002BB1F904104FF09F
:10B2C800040091FBF0F0A3EB0000B8BF5B42322B07
:10B2D800797B0BDC1C4B01FB00418B42A8BF0B4662
:10B2E8001A498B42ACBF9362916201E000239362DA
:10B2F800F97801FB00F31649097803294FEAA313EB
:10B3080029D9B7F84E10B1F5FA7F24D248428342C2
:10B3180020DB8B42A8BF0B461DE000BF5014002065
:10B3280030150020C82F0020362400206481010831
:10B3380020180020F0D8FFFFAC17002000120020D2
:10B3480080C1FFFF8C170020FEFFFF0F020000F0F6
:10B35800241900200346916A936741F34F31B1F5F0
:10B36800807FA8BF4FF480716FF0FF008142B8BFA3
:10B37800014658180023A2F86C00C2F88410C2F8DD
:10B38800903007B0BDEC028BBDE8F08F2DE9F04F8F
:10B398002DED028B85B080460393BC4B02911C882F
:10B3A800019204F00204A4B294B1B94BB3F902407B
:10B3B800B3F90030002CB8BF6442002BB8BF5B4221
:10B3C8009C42B8BF1C46B4F5007FA8BF4FF4007478
:10B3D800C2460025AF4AAE4B32F9152033F8151096
:10B3E800AD4882EAE27EAEEBE27E0BB2BEF5206F9C
:10B3F8004FEA45094FEA43034FEA850750F82560AD
:10B4080012DC4FF0040E92FBFEF29A1A1644B6F5BF
:10B418007A5FA8BF4FF47A56A04A9642ACBF40F86C
:10B42800256040F8252002E0002240F82520C65972
:10B438009AF80B20F61156439AF801205343934A81
:10B4480012884FEAA31B93074FEAA61654D0944AD2
:10B45800019B32F90920022011FB00215A42914236
:10B4680003DB8B42A8BF0B461A468E49039B39F96A
:10B478000110511A33F915208B1808EE103A06F00E
:10B48800EBF868B1B8EEC80A874AB2EE048A80EED3
:10B49800080A505D05F064FB20EE080ABDEEC08A7C
:10B4A800824883493A5818EE103A42F2107E1A44FC
:10B4B8007245A8BF72468A42B8BF0A463A5098F801
:10B4C800081098F81C00594300EB8000C911C0F11E
:10B4D800000E714503DB8142A8BF01468E4698F8ED
:10B4E80012104A431213CEEB0B03B61A664363439A
:10B4F80002EB66260EEB632B664A39F9021004222A
:10B5080091FBF2F16B4A02F19C00405D4143ABEBC9
:10B51800A11398F8511008EE103A51B1101DB8EE69
:10B52800C80A00EBC500D2ED070AFDF72BFDBDEEFA
:10B53800C08ADFF880E1574B0EF1B80139F80300F3
:10B5480039F9012029F801000FFA80FC0EF1BC013D
:10B558000EF1C400C2EB0C023B584FF0040C92FBF6
:10B56800FCF257F801C07A50634498F8501047F835
:10B5780000C0134400EE103A59B10EF15000B8EE75
:10B58800C00A00EBC500DEED070AFDF7FBFCBDEEC7
:10B59800C00A484901F1B40210EE103A525D534313
:10B5A8005A1118EE103A01F1680E9819801A01F133
:10B5B800700329F80E0018EE100AF85001F17C0308
:10B5C8005242FE5001F188030AF1010AFA500B4673
:10B5D8000DB90125FEE62E4A9C6AB2F90410029ABA
:10B5E80092790F3252004A4352112A49002AB1F97E
:10B5F80004104FF0040091FBF0F0A2EB0000B8BF7C
:10B608005242322A98F80D100BDC2B4A01FB0041FC
:10B618008A42A8BF0A4629498A42ACBF9A629962FF
:10B6280001E000229A6298F8031001FB00F2244915
:10B63800097803294FEAA2120CD9B8F84E10B1F5CF
:10B64800FA7F07D24842824203DB8A42A8BF0A46F1
:10B6580000E00246996A9A6741F34F31B1F5807F5D
:10B66800A8BF4FF480716FF0FF008142B8BF014658
:10B6780050180022A3F86C00C3F88410C3F8902077
:10B6880005B0BDEC028BBDE8F08F00BF301500207F
:10B698005014002000120020AC17002080C1FFFFCA
:10B6A800C82F0020362400206481010820180020BB
:10B6B800F0D8FFFF8C170020FEFFFF0F020000F0FC
:10B6C800241900202DE9F04F2DED0A8B85B0834613
:10B6D800039390F85030029101921BB1322BA8BF0E
:10B6E800322300E0012307EE903AF8EEE7BADFEDE7
:10B6F800DE7ADE4B9FEDDECA1B88C7EEABBA002BA5
:10B7080008BF012307EE903AB8EEE7AAD94B2AEE14
:10B718000CCA1B887BEE8CBA9807CCEE2BBA27D5BF
:10B72800D54AB2F90030B2F9022083EAE37182EA1D
:10B73800E270A1EBE371A0EBE27088420446B8BF67
:10B748000C46B4F5E17F16DA88429FEDCCBA05DDE8
:10B75800002AD8BF524207EE902A04E0002BD8BF37
:10B768005B4207EE903AF8EEE77A87EE8BBA04E090
:10B778009FEDC3BA01E0B7EE00BAC24EDFEDC09A42
:10B78800CDF800B006F1080806F1100906F11C050D
:10B798000024F0EE69AABC49DFF8D8A231F91430C8
:10B7A800B54909EE103AB8EEC99AF5EE047A29EED1
:10B7B800279A31F91430BAF80010BDEEC99A08EE8C
:10B7C800103AF8EEC97A9FEDB19A89074FEA440713
:10B7D80027EE899AB8EEC88A00F08180AC4931F921
:10B7E800143007EE903AF8EEE77AB0EE007AE8EE19
:10B7F800077A019B5842FDEEE77A17EE901A8142CC
:10B8080003DB8B42A8BF0B461846A249039B795E0F
:10B81800401A33F91410084407EE900AF8EEE78A44
:10B8280005F01AFF48B19C49F2EE049A88EEA90A7D
:10B83800085D05F095F960EE298A9BF81C30DFED6C
:10B84800976A0AEE903A9BF8083007EE903AF8EEBD
:10B85800677AF8EE6AAA68EEA77AB1EE047A67EE1C
:10B86800A67A2AEE877AFDEEE77A17EE901AF1EEBD
:10B87800477AFDEEE7AA1AEE903A994208DBFDEE08
:10B88800C7AA1AEE903A8B42A8BF0B460AEE903A26
:10B89800D5ED007AE8EE8C7ABBEE0E7AF4EEC77A34
:10B8A800F1EE10FAF8EEEAAA09D4B3EE0E7AF4EE45
:10B8B800477AF1EE10FAC8BFF0EE477A01E0F0EEF1
:10B8C800477AC5ED007A9BF8123009EE903AF8EE07
:10B8D800699A67EEA97ADFED729A67EEA99ABAF8C3
:10B8E8000010CA0753D46848385E0028B8BF4042E1
:10B8F800B0F5206F03DD0020C9F8000026E0009BAA
:10B908009FED687A5B7868EE077A07EE103AB8EE32
:10B91800477A87EE877AD9ED007A37EE497AE7EEEB
:10B928000C7A9FED617AF4EEC77AF1EE10FA09D439
:10B938009FED5E7AF4EE477AF1EE10FAC8BFF0EEAA
:10B94800477A01E0F0EE477AC9ED007A009BD9ED1D
:10B95800007ADB7A08EE903AF8EE688A8B0768EE90
:10B96800A77ADFED538A67EEA88A14D538EE6A8A7B
:10B97800F0EE6A7AEBEE087A78EEE98AB0EE678A3A
:10B98800F0EE697AEBEE287AF0EE678A03E0F0EEE3
:10B99800698AB0EE6A8A474B9FED477A03F19C01AA
:10B9A800625C9BF8511007EE902AF8EEE77A67EE92
:10B9B800C97AA7EE878A51B1181DB0EE480A00EB84
:10B9C800C400D3ED070AFDF7DDFAB0EE408A96ED24
:10B9D800007ADFF8E0A0D8ED007AA6EC019A39EEFB
:10B9E800477A0AF1B40187EE0C7A635C09F104091D
:10B9F800043509EE103A37EE677AB8EEC99AEBEEDD
:10BA0800877A38EE280AE8EC017A67EE897A9FEDA2
:10BA18002B9A27EE899A30EE490A0AF003FA0AF1BE
:10BA28006801BDEEC88AC85318EE103A0AF17001D1
:10BA3800FDEEE88AB1EE499A41F82430BDEEC99A84
:10BA48000AF17C0118EE903A41F8243019EE103AC8
:10BA58000AF18801574641F82430009B01330093CE
:10BA680074BB012497E600BF83F9223ED41100205D
:10BA7800BD37863530150020501400200000E14302
:10BA8800000000005818002000120020CDCC4C40C7
:10BA9800C82F002036240020648101086F12033C5F
:10BAA8000AD7A33D0000A043000040C30000404364
:10BAB8000AD7233C8C170020A69B443BF7CC92382E
:10BAC800029A584B9479B3F90430640028345C43E3
:10BAD800554BB3F9043000EE103ABAEECF0A0AF02B
:10BAE800A1F96411201A002C07EE900AB8BF64422D
:10BAF800322CF8EEE76A03DD0023CAF8283029E083
:10BB0800BDEECAAA1AEE103A23F0030307EE903AE4
:10BB1800B8EEE7AADFED457A9BF80D30CAEE277A32
:10BB280007EE103AB8EE477ADAF8283026EE877A28
:10BB380067EE277AFDEEE77A17EE902A13443C4A1F
:10BB48009342A8BF13463B4A9342ACBFCAF8283079
:10BB5800CAF82820BB6A5B13B3F5807FA8BF4FF4EF
:10BB680080736FF0FF029342B8BF134607EE903A16
:10BB7800F8EEE78AFDEEE67A9BF8032017EE903A96
:10BB880053439B1107EE903A2B4B1B78032BB8EECF
:10BB9800E78A14D9BBF84E20B2F5FA7F0FD2FDEE32
:10BBA800C87A534217EE901A994204DB914217EE75
:10BBB800903AA8BF134607EE903AB8EEE78A9BF88A
:10BBC800511079B14B0803D09942A8BF194600E03B
:10BBD8000121B0EE480A1948D7ED070AFDF7D2F956
:10BBE800B0EE408A38EE280ABDEEC00A8DED000A94
:10BBF800BDF9003000EE103AB8EEC00A0AF012F9AA
:10BC0800BDEEC88AFDEEE88A0023A7F86C0087ED30
:10BC18001E8AC7ED218AC7F8903005B0BDEC0A8BA3
:10BC2800BDE8F08F501400200012002000803B4532
:10BC3800FEFFFF0F020000F024190020A0170020CB
:10BC480010B5084B1968002201EBC20393F90240B2
:10BC5800844201D1981C10BD0132042AF4D100207D
:10BC680010BD00BFFC22002038B1438811EA030050
:10BC780003D08B420CBF01200220704730B50A4B1D
:10BC88000A491C680A78032A0AD8134604EBC30336
:10BC9800551CEAB29D882842F5D00A70981C30BD20
:10BCA8000A70002030BD00BFFC2200207C18002054
:10BCB800014B00221A70E1E77C1800202DE9F047BB
:10BCC800877890F803C0214DBBB2C7F1640E03EB2F
:10BCD80083065C42C3F178005FFA8EFE7600CCF1F1
:10BCE8006408A4B280B2A3B20FFA83F9B9F1000FC5
:10BCF80005DC002B14BFBA464FF0010A00E0F246FB
:10BD080013FB03F303FB0CF21AFB0AF392FBF3F3A6
:10BD1800434403FB09F30A2293FBF2F333449BB237
:10BD280025F8023FB1F800904A880A34C9EB020AA4
:10BD3800A4B21AB202FB0AF24FF47A73844292FB5D
:10BD4800F3F34B442B80CED1BDE8F0877C1800205C
:10BD580010B544780078002202FB02F3193B6343D4
:10BD680003F6C413534340F6C411434393FBF1F362
:10BD7800034921F812300132072AEDD110BD00BF66
:10BD8800961800200430114B33F91000B0F5617F8C
:10BD980010B506DB40F6330398420246A8BF1A46A0
:10BDA80001E04FF461720C78192340F2833013FBE1
:10BDB8000404944207DA497813FB01039342B4BFA1
:10BDC8000020012010BD002010BD00BF7C240020F1
:10BDD80010B500F1500302788A4203D18478C27802
:10BDE800944204D304309842F5D1002010BD0120BC
:10BDF80010BD1FB5084B1B681B030AD58DF804003E
:10BE080001230D2001A98DED030A8DF80530FCF7FB
:10BE180015FC05B05DF804FB402400201FB5084B55
:10BE28001B681B0309D58DF80400029100230D201F
:10BE380001A98DF80530FCF701FC05B05DF804FB9D
:10BE48004024002010B5064B00241C7006F0E6FACA
:10BE5800044B83F82840DC621C865C6310BD00BF7D
:10BE68009E2F00207C18002010B510B9BDE81040A6
:10BE7800E8E700230C225A430A4C1119125D82424A
:10BE880003D00133102BF5D110BD074B586B18B1F7
:10BE98004A784078824203D2002259631A86DA62CD
:10BEA80010BD00BFEC8C01087C18002010B54000C4
:10BEB8001428A8BF14200023074A022199540B44D0
:10BEC80099181424834201F8014CF5DBFF21D15461
:10BED8000F20BDE81040C7E7DC21002010B5094A53
:10BEE800094B11689B6812689142F8D1074A946B14
:10BEF8004FF47A7000FB04F2D31AB3FBF4F300FB9F
:10BF0800013010BD6424002010E000E07C180020FF
:10BF180038B50446FFF7E2FF0546FFF7DFFF401B91
:10BF2800A042FAD338BD10B504462CB14FF47A704C
:10BF3800FFF7EEFF013CF8E710BD2DE9F04F87B0A1
:10BF480088469DF8444011461A469DF8403081467F
:10BF580000250C206843814E87198057484505D134
:10BF680097F808A0BAF1000F04D0F3E00135042DCA
:10BF7800EFD1EFE0B9F1010F00F0DA8006DCB9F19A
:10BF8800000F40F0E78000947548D6E0B9F1020F41
:10BF980000F0D180B9F1140F40F0DC80714FBB691B
:10BFA80043F00103BB617B694FF0904443F40033D5
:10BFB8007B61012603224FF4805B04A94FF0904077
:10BFC8008DF815200392CDF810B08DF814608DF817
:10BFD80016608DF817A0FCF7BDF8A4F828B0C820A3
:10BFE800FFF7A1FFC4F818B07B69039A43F4003344
:10BFF8007B6120464FF4C0534FF0020B04A9049311
:10C008008DF815208DF814B08DF816A08DF817A0AE
:10C01800FCF7A0F8636A23F470436362636A43F42D
:10C0280060436362636A23F470236362636A43F460
:10C03800602363624C4B4D4C4FF480221A6002F12E
:10C048008042A2F53F321223E366082384F8713058
:10C05800136884F8726023F480231360536823F410
:10C068008023536094F8703003F1804303F58233E2
:10C078001A6842F480221A60E26E3D4B22F01F00DB
:10C0880002F01F02C15806FA02F221EA0202C25067
:10C09800E26E384922F01F0002F01F0250F801E05A
:10C0A80006FA02F22EEA02024250E26E22F01F0164
:10C0B80002F01F02C85806FA02F20243CA502E4B79
:10C0C8002E4AC3F800A0FB6943F40003FB612C4B24
:10C0D80004A8DA608DF810908DF811B08DF812A0D0
:10C0E8008DF8136004F0F2FC2A238DF810309DF8C7
:10C0F80013308DF811608DF812A01BB104A804F05C
:10C10800E5FC04E01F4B4FF48062C3F884201E4A0C
:10C118001E4B136002221A721D4A1E4B13601E4AE0
:10C128001E491B68116098471D4BE3631D4807E0D3
:10C1380000941D4801E01D48009401F0A3FE48B199
:10C14800064B80F804900C2202FB053585F8088020
:10C15800686000E0002007B0BDE8F08F00230020F1
:10C168000038014000100240140401407C180020EF
:10C17800080401400C040140D80042420005FA05B9
:10C1880000ED00E000E100E0F4210020F8210020AB
:10C19800D8200020B4000020D42000205000002027
:10C1A80068810108B8180020004400400048004099
:10C1B80038B5134B202240F2DB151A85684310224C
:10C1C8009A61851E0B24013C14F0FF0411D00C4A1F
:10C1D800938A9BB283F020039382938A9BB283F065
:10C1E800100328469382FFF79EFE1920FFF79BFE57
:10C1F800E9E7044B044A1A60044B054ADA6038BD83
:10C2080000040048FC9F0020EFBEADDE00ED00E01A
:10C218000400FA05024A136801331360704700BF2F
:10C2280064240020024B5B6F03B11847704700BFBE
:10C238007C18002003685B69184703681B69184766
:10C248000368DB68184703689B68184703685B68DE
:10C25800184703681B6818472DE9F84FB0F90230F2
:10C26800934218BF00232DED028B18BF0370057889
:10C2780004460E469146002D40F08B8007EE902A2A
:10C288009FED770AF8EEE77AB6EE008A27EE800A85
:10C29800DFED747A20EE270AA04620EE080A09F09E
:10C2A80037FEDFED716A60EE266AB7EE006AB0EE1F
:10C2B800667AA0EE007A40F2DC536365D0EE006A3D
:10C2C8001023A4F8523037EE067A76EE866AC6EE68
:10C2D800077A1823A4F85030274684ED046A27EE1D
:10C2E800807A27EE007A77EE075A84ED017AC4ED5A
:10C2F800025A70EE005A84ED037AB8EE007AA5EE81
:10C30800807A27EE877A67EEA67A84ED057AC4EDFF
:10C31800067ADFED567A98ED047A27EE277AF0EE62
:10C32800678AB5EEC07AF1EE10FA4CBF77EE487A1C
:10C3380077EE087A013517EE900A06F0CBF8D8EDBB
:10C34800017A67EEA87AC7E90E01F5EEC07AF1EE38
:10C3580010FA4CBF77EEC87A77EE887A08F10408AD
:10C3680017EE900A06F0B6F8032DC7E9080107F1A1
:10C378000807CED1A6F2DC531B042367E367636783
:10C38800C4F88030A367C4F884300123A4F802906D
:10C398002370D4F85490B4F95280636A276A206FE6
:10C3A800E26FD4F840C0D4F88010C4F88020C9EBFC
:10C3B800060606FA08F64FEAE67B734307FB0B33DB
:10C3C8002667A7FB06671F44636C656F60674FEAC3
:10C3D800E27B53430CFB0B3EACFB02237344B61ABF
:10C3E80067EB0307E36AA26AC4F884104FEAE07BAC
:10C3F800434302FB0B3EA2FB00237344B6185F4184
:10C40800E36CA06CB4F95020A5674FEAE17B4B437D
:10C4180000FB0B33A0FB01011944636B361A206B38
:10C428004FEAE57B05FB03F300FB0B3367EB0107E2
:10C43800A0FB050119448019794106F021F808F19B
:10C44800FF3201239340E067C01841EBE371424695
:10C4580006F016F8BDEC028B4844BDE8F88F00BF23
:10C468006F12833ADB0F4940F404B53F0000804B5C
:10C478002DE9F8430024234B93F8A860E0B2B042BA
:10C488000CD203EB8003204A9B6F32F810101BB1CB
:10C498000B2801D8DB6898470134ECE71B4B1B6875
:10C4A8005B032DD500242346E2B2B24228D2DFF83E
:10C4B800549009F178074FEA840857F82420556802
:10C4C8009D4215D0284604F073FAEFF312835022E8
:10C4D80082F3128828216A6A01FB00900132C0F8B1
:10C4E800D0206A6942F001026A61DBB283F31188E5
:10C4F80057F808301B6800221A6001342B46D3E72E
:10C50800BDE8F8837C180020201200204024002079
:10C5180008B50E4B1B6813F4805F0D4B14BFD3F89E
:10C528007421D3F8782193F8A81092880023D8B200
:10C53800884204D2074820F813200133F7E7FFF7B1
:10C5480097FF3220BDE80840EDE400BF40240020FA
:10C558007C180020201200200A4B1A680A4B30B5BC
:10C5680002F48052D3F87441D3F8785100230AB109
:10C57800A18800E0A988054820F8131001330C2B86
:10C58800F5D130BD402400207C180020B2210020C5
:10C5980070B5124D0024214605F27D10702285F8F1
:10C5A8007C4109F030FA2146D5F8F0310B4A0B44AA
:10C5B80093F9020080B102F27D141E680E51081929
:10C5C8009C8884809B79837192F87C310731013390
:10C5D800702982F87C31E7D170BD00BF7C1800203B
:10C5E800094B1A680E2303FB0020437AFF2B07D060
:10C5F800064A12789A4203D9054A32F8130000E035
:10C60800808800B2704700BFC41A0020382F00206D
:10C618007C24002038B5294C2DED048B94ED7D8ABF
:10C62800B0EE480A0546FCF773FFF0EE408AB0EE1C
:10C63800480AFCF70AFF94ED7E9AB0EE408AB0EE05
:10C64800490AFCF765FFF0EE409AB0EE490AFCF79C
:10C65800FCFE95ED017AD5ED027A95ED006A68EE5B
:10C66800676A27EE088AE7EE286A68EE000A67EE2E
:10C67800807AE6EE290AB0EE660AE7EEA80A09F023
:10C68800D3FCDFED0F7A20EE270ADFED0E7A80EE7D
:10C69800270AD4ED7F7A30EE270AF2EE047A80EE8C
:10C6A800270A09F0BFFBBDEC048B83B21A0444BF10
:10C6B80000F5B47083B218B238BD00BF7C180020F2
:10C6C8000000E144DB0F494001380A4B042804D834
:10C6D800DFE800F00507090B0D00074A08E0074AE4
:10C6E80006E0074A04E0074A02E0074A00E0074A72
:10C6F8001A607047040100208516010841AD000842
:10C70800B119010895B3000801B00008CDB60008BA
:10C7180038B500240B4D6059254403F09FF969682A
:10C7280011B10948FCF762FEA96811B10748FCF786
:10C738005DFE0748103403F091F9B4F5D87FE9D1CC
:10C7480038BD00BF80810108FDA4010803A50108C8
:10C7580094B00108F0B585B0044609F098F90828A6
:10C7680026D1621EE01D1F4912F8013F09681944CD
:10C77800497801F00301022908BF203B8242137067
:10C78800F1D1254604F1080715F8016B1648314622
:10C7980009F06FF920B12846314609F06AF910B15D
:10C7A80000F042FE1CE0BD42EED1204603F004FE3C
:10C7B8000E4803F053F900230D4A1A4404A992F8CD
:10C7C8008A210A440849595C02F80C1C0133082BD9
:10C7D800F2D1002307488DF80C3001A9FCF706FEBA
:10C7E80005B0F0BD10010020C4BB010809A501086F
:10C7F800A0240020D6AF01082A4B2B4C1E682068C5
:10C8080080B501F061FA304601F05EFA206841799E
:10C818008D0703D441F00201FFF70CFD234B244D93
:10C8280010229A6120229A612B689A0341BF06233D
:10C838006371E37923F0010344BF43F00203E3711A
:10C848002068FFF703FD90B1184F10233B85164B66
:10C858001868FFF7F8FC8046F9F764FD08B102F0A4
:10C86800E5F930464146FFF7F4FC1023BB6130463A
:10C87800FFF7ECFC78B10D4FD4F800904FF020088A
:10C88800A7F828803046FFF7DEFC01464846FFF748
:10C89800E0FCC7F818802B689B03D1D5FDF7ADFEE7
:10C8A800CEE700BFCC2100207C1A002000040048FD
:10C8B800402400202DE9F047054609F0E8F8314EFC
:10C8C8000446D6F8088090B92F4803F0C7F82F4BD4
:10C8D80053F8241049B10123A34013EA080F02D0EA
:10C8E8002B48FCF783FD0134F1E72A4822E028466B
:10C8F8002949224609F0D4F858B92848284C03F0A9
:10C90800ADF854F8041F0029EFD02148FCF76EFD5C
:10C91800F7E72B782D2B03BF013504F1FF344FF0D7
:10C92800010A4FF0000A4FF00009184B53F829701C
:10C9380027B91C48BDE8F04703F090B828463946A7
:10C94800224609F0ADF8C8B9012000FA09F08305BC
:10C9580001D51548EEE7BAF1000F03D0FCF79CFEAD
:10C96800124803E040EA0800B060114803F076F886
:10C9780039461048BDE8F047FCF738BD09F1010910
:10C98800D3E700BFA02400200FA5010830830108C9
:10C9980019A5010894B001081DA5010822A50108E0
:10C9A8002C8301082EA501083DA501084BA5010807
:10C9B80054A50108D5AF010810B5084803F04EF892
:10C9C800074B00241C741C64064B1C70FFF7C4FD45
:10C9D80003F028FA044B1C6010BD00BF5CA50108D9
:10C9E8007C1A0020D02F0020CC21002070B50646EC
:10C9F80000240B4BE518AA8816420AD0E1580948CA
:10CA0800FCF7F4FC2846002102F0B5FF064803F0C5
:10CA180025F8143440F694439C42EAD170BD00BF17
:10CA28008C8E010888A5010894B00108F0B5047837
:10CA38008BB005460CB1002436E04A4B19680E232A
:10CA480003FB041101F58C70B1F91D51B1F91921DD
:10CA5800B1F91B31009591F82051019591F82151B8
:10CA6800029590F90700039001F590713E4891F9FD
:10CA78000210049121460134FCF7B8FC082CDCD1E3
:10CA88006DE02D2B14D1072C1BDC284609F056F835
:10CA98000AAB661C03EB440424F8100C15F8013F9C
:10CAA800303B092BFAD934462B78002BE9D104E026
:10CAB800A3F13002092A09D8E5E7082CBDF81820A7
:10CAC80009D00BB0BDE8F04000F0AEBC202BF8D187
:10CAD80001352646E7E7072AF3D8BDF81A00214BA7
:10CAE800A0F2EE2189B240F2DC55A9421B68E8D8D1
:10CAF800BDF81C10A1F2EE24A4B2AC42E1D8BDF8F6
:10CB08001E7004B23EB2A642DBDB0DB2AE42D8DCE8
:10CB1800A542D6DBBDF92440642CD2D1BDF82660ED
:10CB280034B2112CCDDCBDF82050B42DC9D8BDF8D5
:10CB38002240B42CC5D812B24FF00E0E0EFB0233B1
:10CB4800A3F81B116421A3F81901A3F81D7183F838
:10CB5800205183F8214183F81F1183F822610BB01B
:10CB6800F0BD00BF1C12002092A50108F0B50446D4
:10CB78008FB0204608F08BFFC5B225BBAC48AD4C42
:10CB880002F06CFF94F8D61009B9AB4854E049B2EA
:10CB980094F8D42094F8D530009194F8D7100191E6
:10CBA80094F9D810029194F9D910039194F8DA10F5
:10CBB8000491A24829460135FCF718FC102D04F110
:10CBC8000704DFD1E1E720469D49052208F068FF08
:10CBD8000546B8B929469B48702208F014FF9A4BBD
:10CBE800196828460E2303FB001301300022082889
:10CBF80083F8232183F8242183F8252183F826212B
:10CC0800F0D113E120469149042208F049FF054676
:10CC18002046002D4AD1202108F02BFF002800F0E3
:10CC28000581461C304608F032FF2C460746884BE3
:10CC380053F824502DB987480FB0BDE8F040FCF7F1
:10CC4800D5BB30462946FAB208F02AFF013400283D
:10CC5800EDD1784A02F170011646002382F8DA30E5
:10CC680082F8D63082F8D53082F8D43007328A423A
:10CC7800F3D1794901EBC40191F80822934210DA03
:10CC8800D1F80C72C3EBC302B0183A4400F1D401D6
:10CC98001768C0F8D4709088888092798A710133B7
:10CCA800E7E729466D48FCF7A1FB90E06C490722AD
:10CCB80008F0F6FE05462046002D4AD1202108F04E
:10CCC800D8FE064608F0E3FEC4B274BB6548FCF71C
:10CCD8008DFB214664480134FCF788FB0E2CF8D103
:10CCE8005548FCF783FB002460482146FCF77EFB8F
:10CCF8000025554A5E4811680E2202FB04120123E2
:10CD0800D2F823215B49AB4013425B4B05F1010587
:10CD180008BF1946FCF76AFB0E2DEAD146480134D4
:10CD2800FCF764FB082CDFD180E03046534908F05B
:10CD380009FF2C4600284CD0022C4FD008F0FEFEEC
:10CD480006AB4E4943F82400002008F0FBFE0134EE
:10CD5800F0E74A4908F0F6FE002460B1082C38D004
:10CD680008F0ECFE06AB454943F82400002008F023
:10CD7800E9FE0134F1E7082C2BD1069B0F2B28D8AC
:10CD8800DDF81CE0BEF1070F23D8089F0D2F20D82F
:10CD9800099E06F16402C82A1BD80A9DFF2D18D8DF
:10CDA8000B98642815D80C99642912D8884210DA8F
:10CDB8000D9C032C0DD8324AC3EBC303134483F8EC
:10CDC80004E05F719E71DD71187259729C722D4C6E
:10CDD800CFE60FB0BDE8F04000F026BB069B072B5E
:10CDE80020D807990D291DD80278722A0DD06E2AED
:10CDF80018D1154A12680E2000FB032301228A402D
:10CE0800D3F8231121EA020209E00F4A12680E2022
:10CE180000FB032301228A40D3F823110A43C3F8F5
:10CE2800232101E000F000FB0D4CA2E60FB0F0BD9D
:10CE3800BAA50108A024002094B00108E5A50108BE
:10CE480001A60108742500201C12002007A601086D
:10CE5800209B01082EA50108808101080CA6010865
:10CE6800B2A5010807A5010818A60108AAA4010887
:10CE78001DA60108EFB30108A9B4010821A60108FD
:10CE8800702500200BA201082DE9F7430478054618
:10CE98008CB9324D95F89F12B5F89C2295F89E32C0
:10CEA8002F48009121460134FCF7A0FA102C05F117
:10CEB8000405EFD14FE008F041FE0F28044636DCA8
:10CEC8002846202108F0D5FD264EE4B2D6F8448045
:10CED800451CA4000027284608F030FE5FFA87F9B1
:10CEE800B9F1010F83B208D0B9F1020F0BD0B3F535
:10CEF800B47F25D2726C13530AE0FF2B20D8736CD1
:10CF08002344987004E0FF2B1AD8736C2344D8701C
:10CF180028462C2108F0ADFD054608B1013502E090
:10CF2800B9F1020F0CD10137032FD4D113E00E4809
:10CF38000E4900220F2303B0BDE8F043FCF756BAB0
:10CF480008EB04000021042208F05DFD03B0BDE8F1
:10CF5800F04300F069BA03B0BDE8F083A0240020D4
:10CF680023A601087C1A002037A6010856A6010846
:10CF78002DE9F0412DED048BB2498AB0044608F042
:10CF88004BFDB149002820460CBF0126072608F0B2
:10CF980043FDAE490028204608BF022608F03CFDA4
:10CFA800002808BF0426F10740F10581A848A94CCC
:10CFB80002F054FD002002F059FBA74802F04EFD94
:10CFC800A64802F04BFD6379A54AA648013B2546D1
:10CFD80052F82310FCF70AFAA348FCF707FA4FF0B7
:10CFE8000008274695ED058AB5EE408AF1EE10FA5D
:10CFF80004D19E48FCF7FAF9002570E09C48D5ED6D
:10D00800069A95ED079AD5ED088A4146FCF7EEF9A0
:10D01800B5EEC08AF1EE10FA02D5202002F016FD16
:10D02800B0EE480A06A8FCF761F801469148FCF7FB
:10D03800DDF9F5EEC09AF1EE10FA02D5202002F0E3
:10D0480005FDB0EE690A06A8FCF750F801468948C4
:10D05800FCF7CCF9B5EEC09AF1EE10FA02D5202013
:10D0680002F0F4FCB0EE490A06A8FCF73FF80146C6
:10D078008048FCF7BBF9F5EEC08AF1EE10FA02D54C
:10D08800202002F0E3FCB0EE680A06A8FCF72EF8B0
:10D0980008F1010801467848FCF7A8F9B8F10C0F27
:10D0A80005F110059ED1A4E749B294F8D42094F86C
:10D0B800D530009194F8D710019194F9D8100291C5
:10D0C80094F9D910039194F8DA1004916B48294621
:10D0D8000135FCF78BF9102D04F1070403D094F8FF
:10D0E800D6100029E0D100254FF00E0808FB05F8FE
:10D0F8000024634A926C42440123D2F80A20A340D8
:10D10800134240F0948001340E2CF2D10135082DE1
:10D11800EAD15C485C4C02F0A1FCD7F8088054F8CE
:10D12800041F19B15948FCF761F9F8E70D46584B47
:10D1380053F8254054B10123AB4013EA080F03D03C
:10D1480054482146FCF752F90135F0E7524802F0FD
:10D1580085FC21467B180AAA93F88A3113444F4A62
:10D168008A5C03F8102C01310829F3D1002306A9A1
:10D178004B488DF82030FCF739F94A4802F06EFC2C
:10D18800494800F099FC494802F068FC464800F01C
:10D1980051F9474802F062FC4348FFF775FE4548DD
:10D1A800FCF724F94020FFF721FC434802F056FC25
:10D1B8003D4800F023FDB20726D5404802F04EFC5A
:10D1C8003F4802F04BFC384802F090FA3D4802F024
:10D1D80045FC354800F0AFF83B4802F03FFC3248C8
:10D1E80000F0B8FB3948FCF701F92F4800F030FA95
:10D1F800374802F033FC2C48FFF718FC2D48FCF7A1
:10D20800F5F88020FFF7F2FB730716D5314802F0D6
:10D2180025FC314802F022FC234802F041FA254857
:10D22800FCF7E4F84FF48070FFF7E0FB05E02946CF
:10D2380022462A48FCF7DAF865E70AB0BDEC048B09
:10D24800BDE8F0815CA6010868AA010863A6010888
:10D2580069A60108A024002077A6010889A601086C
:10D26800209B010895A60108A0A60108ADA6010803
:10D27800BAA6010806A50108D6AF0108C2A601088A
:10D288007C1A0020E1A601082C830108F1A60108F8
:10D2980030830108FFA601080CA70108C4BB0108D8
:10D2A80018A7010821A701080BA2010830A7010847
:10D2B8003CA7010894B001084AA7010857A701082C
:10D2C8006AA7010878A7010882A7010891A70108A1
:10D2D8009FA70108ABA70108BCA70108CEA70108B2
:10D2E800F8B504460E46174600252046202108F0CA
:10D2F800C0FB0446D0B10134204608F01FFCB0F54D
:10D30800617F05DB40F634039842A8BF184601E068
:10D318004FF46170A0F56170192390FBF3F00DB91B
:10D32800307000E070703B7801333B700DB9012517
:10D33800DBE72046F8BD7FB504780646E4B9364BEE
:10D348001B6803EB8403192193F87B0093F87C6036
:10D3580093F8792093F87A304FF4617511FB0050F7
:10D3680011FB0651009001912C4821460134FCF72D
:10D378003DF8142CE3D14CE008F0E0FB13280546F7
:10D3880041DC254B701C1C68202100238DF80F30D0
:10D3980008F06FFB1E35064670B10136304608F0BE
:10D3A800CDFB19289FBF04EB850358709DF80F30FB
:10D3B800013398BF8DF80F303046202108F059FB13
:10D3C800064670B10136304608F0B8FB0D289FBFFD
:10D3D80004EB850398709DF80F30013398BF8DF8E2
:10D3E8000F3004EB85043046E11C0DF10F02FFF706
:10D3F80077FF9DF80F30042B0BD0601C002104220E
:10D4080008F001FB05E00648064900221323FBF754
:10D41800EDFF04B070BD00BF1C120020ACAC0108C9
:10D4280037A6010856A60108014802F017BB00BF3D
:10D43800C1AC01082DE9F04304788FB00546002CF3
:10D4480059D17B4B0021142209A807AED3F80080DC
:10D4580008F0D9FA07223046002108F0D4FA05A8C6
:10D468000023A700059308EB070583801A46714936
:10D47800B5F802E031F813C01CEA0E0F0AD00DF11E
:10D48800380C0E3102F1010E6244595C02F81C1C82
:10D498005FFA8EF20133072BE9D100210B46664A69
:10D4A800B5F802E011F802C01CEA0E0F0AD00DF11F
:10D4B800380C063203F1010E63448A5C03F8242C0D
:10D4C8005FFA8EF301310629E9D118F807305B4974
:10D4D8008DE841006A78029209A81A0903F00F033F
:10D4E800FBF76FFF2146564809AA0134FBF77EFF78
:10D4F800202CA6D199E008F021FB1F28044600F350
:10D50800868028462021E4B208F0B3FA1F2C02D9FD
:10D51800FFF78AFF89E0464B1B6803EB8404451C30
:10D5280000212046042208F06EFA0027454B09AE78
:10D53800304600210A2217F803905FFA87F808F0AE
:10D5480062FA002315F8012B32B10A2B04D04A45A0
:10D5580002D0F2540133F5E74A455FD108F1FF33B1
:10D56800032B09D8DFE803F01005023F0DF1230172
:10D5780034E00DF123011EE0304608F0DFFA23788D
:10D58800C0B243EA001006E0304608F0D7FA237824
:10D5980000F00F001843207031E00133062B0AD049
:10D5A800244800F11B069E5D9642F6D103445A7D3D
:10D5B80063881343638011F8012F02B30023EFE758
:10D5C8000133072B0AD01B4800F10E069E5D9642D8
:10D5D800F6D130F8132063881343638011F8012FC4
:10D5E8006AB10023EFE7304608F0A8FA0F2804DCF8
:10D5F800304608F0A3FA607001E000236370013739
:10D60800052F93D1012401F0B7FA74B980E70E49C8
:10D618000E4800221F23FBF7E9FE06E02046002102
:10D62800042208F0F0F90024EDE70FB0BDE8F0831C
:10D63800C81A0020188501082D850108CFAC0108FB
:10D64800DEAC01083985010856A6010837A601088D
:10D658002DE9F041047807467CB9344DB5F8BE2170
:10D66800B5F8C031324821460134FBF7BFFE042C1F
:10D6780005F10405F2D1BDE8F0812E4908F0CCF996
:10D68800B0B92A4B4FF47A714FF4FA62A3F8BE117D
:10D69800A3F8C021A3F8C211A3F8C421A3F8C611A6
:10D6A800A3F8C821A3F8CA11A3F8CC21BDE8F081DA
:10D6B800384608F043FA032805462ED83846202174
:10D6C80008F0D7F9044630B10134204608F036FA9C
:10D6D8000127064600E007462046202108F0C9F940
:10D6E80010B9BDE8F0419FE6013008F027FA012F94
:10D6F800F7D1A6F2EE2240F2DC539A42F1D8A0F21A
:10D70800EE229A42EDD88642EBDA084B6E3503EBEF
:10D718008503DE801881BDE8F081074807490022AB
:10D728000323BDE8F041FBF761BE00BFA024002041
:10D73800EAAC010801A6010837A60108BCB2010835
:10D748002DE9FF4104780546002C39D17348744D02
:10D7580002F084F9D5ED057AF5EE407AF1EE10FA8B
:10D7680000F0D98021466F48FBF740FE95ED050A89
:10D778006846FBF7BBFC01466B48FBF737FE95EDA7
:10D78800060A6846FBF7B2FC01466748FBF72EFE1F
:10D7980095ED070A6846FBF7A9FC01466248FBF7C6
:10D7A80025FE95ED080A6846FBF7A0FC0134014602
:10D7B8005E48FBF71BFE0C2C05F11005CAD1AAE048
:10D7C8005B49052208F06CF940B9554B03F1C002DA
:10D7D8000021596110339342FAD19CE028465549FB
:10D7E800042208F05DF904462846002C40D1202187
:10D7F80008F03FF9002800F08E80451C284608F004
:10D8080046F907464C4B53F824601EB94B4802F0C2
:10D8180025F980E028463146FAB208F041F901348A
:10D828000028EFD13E4B03F1C0029E46002159610A
:10D8380010339342FAD1424B03EBC4029846D2F814
:10D8480004C0BCF1000F04D131463E48FBF7CEFDC1
:10D8580057E0002718F834309F42F5DA3B010EEB09
:10D86800030563440FCB143585E80F000137F1E752
:10D8780008F064F90B28064647DC2846202108F002
:10D88800F8F8054650B101352846FBF7A5FB244BAF
:10D8980003EB061383ED050A012400E0044628463D
:10D8A800202108F0E6F8054648B101352846FBF77F
:10D8B80093FB1B4B03EB061383ED060A0134284642
:10D8C800202108F0D6F8054648B101352846FBF76F
:10D8D80083FB134B03EB061383ED070A0134284639
:10D8E800202108F0C6F810B9FFF79EFD13E00130BB
:10D8F800FBF772FB0A4B032C03EB061686ED080AAE
:10D90800F2D11148FFF71CFF05E010481049012229
:10D918000C23FBF76BFD04B0BDE8F081FDAC0108FA
:10D92800A024002018AD01081EAD0108D6AF0108DB
:10D9380001A6010807A60108209B01082EA50108D9
:10D94800DCAB01080CA601080BA2010837A60108E8
:10D9580056A60108F0B5047887B006461CBB524BA2
:10D968001968062303FB0411192091F8CA5091F88D
:10D97800CB7091F8CE2091F8C9304FF4617610FB46
:10D98800056510FB07600095019091F8CC000290A6
:10D99800C83146484979039121460134FBF726FDF1
:10D9A8000C2CDCD17DE008F0C9F80B28044672DCA9
:10D9B8003D4B701C1D68202100238DF8173008F09E
:10D9C80058F8064680B10136304608F0B7F8032803
:10D9D8009FBF062303FB045383F8CE009DF817303E
:10D9E8009CBF01338DF817303046202108F041F8EC
:10D9F800074680B10137384608F0A0F80D289FBFC8
:10DA0800062303FB045383F8C9009DF817309CBF15
:10DA180001338DF8173006266643A9193846CA31EE
:10DA28000DF11702FFF75CFC202108F022F80746E9
:10DA380070B10137384608F081F814289FBF9DF867
:10DA480017307619013386F8CC0098BF8DF8173057
:10DA58003846202108F00DF878B1013008F06EF84A
:10DA68000D289FBF062303FB045383F8CD009DF8C0
:10DA780017309CBF01338DF817309DF81730062BEF
:10DA88000FD0062202FB04500021C93007F0BBFF6B
:10DA9800FFF7CAFC05E00648064900220B23FBF7FE
:10DAA800A5FC07B0F0BD00BF1C12002022AD010884
:10DAB80037A6010856A60108F0B5027887B08AB9DA
:10DAC8004A4C04F1200694F8EA21002348495956A3
:10DAD80050B281426DD00C33302BF7D10834B442A8
:10DAE800F1D180E0002204920592451C08F026F846
:10DAF800C4B260B2FEF7A4F8074618B18DF810401A
:10DB0800012400E004462846202107F0B2FF05461C
:10DB180038B10135284608F011F80134ADF8120083
:10DB2800E4B200262846202107F0A3FFB0B3451C25
:10DB3800284608F003F800222E4951F82230834283
:10DB48005FFA82FE04D00132082AF5D1002300E0F2
:10DB5800734651F82320824220D1022E0FD0032E83
:10DB680012D05A1E012ED2B204D0042A13D88DF82E
:10DB780014300EE0042A0ED88DF8153009E0052B74
:10DB880009D88DF8173004E09A1E052A03D88DF8B5
:10DB980016300134E4B20136042EC3D1052C03D863
:10DBA80007B0BDE8F0403FE404AB03CB38607960D0
:10DBB80019E094F8EF010F4B94F8EE5153F8200058
:10DBC800B4F8EC21009094F8F10153F8200001908A
:10DBD80094F8F00153F82000029053F825300648D5
:10DBE800FBF704FC7AE707B0F0BD00BFA0240020D3
:10DBF80000230020E89B010842AD0108F7B504782E
:10DC080006464CB9204601A903F0E4F90134FFF7B0
:10DC1800F5FF0E2CF6D14FE007F090FFC5B20D2DA1
:10DC280046D8701C202107F024FF034658B15B78C2
:10DC3800682B00F1010007D0732B01D1012704E004
:10DC4800FFF7F2FB38E000E00027202107F011FF82
:10DC58001A4C05F1D006C0B1013007F06FFF40F251
:10DC6800ED2380B2984205DD40F6CA039842A8BF6A
:10DC7800184601E040F2EE2004EB4603A0F2EE2045
:10DC880019229F7090FBF2F0D87004EB46042946E5
:10DC9800A3780B48012BE3784FF0190540F2EE24E6
:10DCA8000CBF7322682205FB0343FBF79FFB03E0CD
:10DCB80004480E21FBF79AFB03B0F0BDA024002016
:10DCC80061AD010873AD010810B504462046FEF7A2
:10DCD800B4FA18B90A20FEF726F9F7E710BD0022B2
:10DCE80007490C2303FB02135968814204D100221F
:10DCF800C2621A725A6070470132042AF0D1704722
:10DD080000230020026BC168034610B5406942B188
:10DD18001A6C8C1A013A005D08BF0A46C0B21A6430
:10DD280010BD1A6A805C01328A4228BF0022C0B244
:10DD38001A6210BD436B13B190F844007047836AB0
:10DD4800406A1B1A584258417047036B13B15B680D
:10DD5800016C01E0C369016A8B423CBFC2689B1831
:10DD6800581AC0B27047836A8169426B1944D160FE
:10DD7800416A99429DBF0169CB1A5360CB1A96BF7D
:10DD88000023536083624FF0000380F84430136827
:10DD980088BF816243F0010313607047436A826958
:10DDA800D154436A02690133934228BF0023436276
:10DDB800436B1BB11B68DB0705D4D4E7026D1368FE
:10DDC80043F08003136070474171F6F7DFBB816051
:10DDD800F6F7DCBB026D036B70B50446D5699BB9D9
:10DDE800A90611D5C36A1BB1908C80B298470BE085
:10DDF800E169928C40694E1CD2B2E6614254E169F5
:10DE0800E268914228BFE361616BA1B92A0612D585
:10DE1800636AA26A9A42236D09D0501CA669A0625F
:10DE2800B25C1A852369984205D3A16203E01A6897
:10DE380022F080021A602B0742BF236D08221A6263
:10DE480070BD0D4B0D484FF400525A600C4A1168D2
:10DE58004FF6FE730B401360426B11684FF6FE736A
:10DE68000B401360426A836A9A4200D07BE7012321
:10DE780080F84430704700BF00000240DC230020D7
:10DE8800440002402DE9F0471E46A14B8CB0984251
:10DE9800894690469DF850507ED19E4B9E4A1A6006
:10DEA8009E4A5A6102F580729A614FF48072DA6074
:10DEB8001A619B4A1A63143A5A63A2F54842203AF7
:10DEC800DA6404329A64C3F808801865954B9A6935
:10DED80042F480429A615A6942F001025A6102236F
:10DEE8008DF80830032315F0010A8DF809304FF03A
:10DEF80000038DF80A3014BF022301232C078DF884
:10DF08000B3017D5884C402701978AF001038DF80C
:10DF18000A30236A23F070632362236A43F0E063C4
:10DF28002362204601A9FAF715F9BAF1000F23D1A7
:10DF3800A76121E0B0070ED50CA9402341F82C3D7C
:10DF48007948036A23F070630362036A43F0E0636D
:10DF58000362FAF7FFF8F1070ED50CA9802341F800
:10DF68002C3D7148036A23F070430362036A43F04F
:10DF7800E0430362FAF7EEF80E238DF80030002232
:10DF8800012368468DF801308DF802208DF80330A2
:10DF9800604C02F09BFD08E1644B984274D1644BDD
:10DFA8005D4A1A604FF48072DA601A61614A5A61F8
:10DFB80002F580729A615B4AC3F808801865D369D4
:10DFC80043F40033D36102238DF80830032315F09E
:10DFD800010A8DF809304FF000038DF80A3014BF9C
:10DFE800022301232A078DF80B3019D54FF09044EE
:10DFF800042701978AF001038DF80A30236A23F475
:10E0080070632362236A43F4E063236220460DEBC6
:10E018000701FAF79FF8BAF1000F25D1A76123E0AD
:10E02800B3070FD50CA9042341F82C3D4FF09040BD
:10E03800036A23F470630362036A43F4E0630362D0
:10E04800FAF788F8F7070FD50CA9082341F82C3DF3
:10E058004FF09040036A23F470430362036A43F469
:10E06800E0430362FAF776F826238DF800300022A1
:10E07800012368468DF801308DF802208DF80330B1
:10E088002B4C02F023FD90E02B4B984240F00E8180
:10E098002A4B214A1A604FF48072DA601A61284AC2
:10E0A8005A6102F580729A611E4AC3F808801865A1
:10E0B800D36943F48023D36102238DF80830032306
:10E0C80015F0010A8DF809304FF000038DF80A3079
:10E0D80014BF022301232C078DF80B3032D5124CC4
:10E0E8004FF4806701978AF001038DF80A30636A5C
:10E0F80023F470636362636A43F4E06363622046F7
:10E1080001A9FAF727F8BAF1000F3FD1A7613DE05E
:10E1180000380140DC230020008A0108CC1A0020C6
:10E12800580002400010024000040048004400402B
:10E1380088230020CC1C0020004800403423002005
:10E14800CC1E0020B0070FD50CA94FF4806341F80E
:10E158002C3D5848436A23F470634362436A43F48E
:10E16800E0634362F9F7F6FFF1070FD50CA94FF406
:10E17800006341F82C3D4F48436A23F470434362DF
:10E18800436A43F4E0434362F9F7E4FF27238DF839
:10E1980000300022012368468DF801308DF80220F6
:10E1A8008DF8033002F092FC434CC4F82C90002701
:10E1B800012384F844302762E761A76267626671C9
:10E1C800C4F80880A5712046F6F7E0F9F20734D5BF
:10E1D800236B002B2AD001A8F9F758FDE36C0193B3
:10E1E8004FF480530A9380230693E368ADF8103008
:10E1F80020230993206B636902930B970597079770
:10E2080008970397F9F76DFD01A9206BF9F74BFD06
:10E21800236B216D1A6842F001021A608A6842F085
:10E2280040028A605B689BB2236406E0236D20226B
:10E238001A621A6842F020021A60B3072FD5636B7E
:10E2480043B301A8F9F722FDA36C01934FF480535F
:10E258000A93802306932369ADF810300025102314
:10E26800606B03930B950595079508950995F9F744
:10E2780038FD606B01A9F9F716FD636B1A6842F067
:10E2880002021A60226D5D605D60936843F080034E
:10E29800936004E0226D136843F080031360226DDD
:10E2A800136843F001031360204600E000200CB01F
:10E2B800BDE8F0870004004834230020704708B503
:10E2C8000B4B002093F82C10F9F72CFC094B1B681A
:10E2D800187A082801BF084B4FF480521A80102280
:10E2E80008BF5A80A0F109035842584108BD00BF31
:10E2F800B4000020F4210020CC2000207047704793
:10E308007047FEE7FEE7FEE7704730B50024E3B24A
:10E3180093420DD2030F092B94BF3033373301F8E2
:10E32800143001EB4403002500015D700134EEE771
:10E3380030BD30B5002202F1805303F5B8539B007D
:10E3480042F400441D6840F60F7144F080042940EF
:10E3580001322143042A1960EDD1024B40F08000BC
:10E36800186030BD4C5C00402DE9F347884D894C5E
:10E378002B68894E9BB2A380A28831880A409705F2
:10E3880007D54FF6FF53854A2B6013780133DBB26C
:10E398001370A3880B40180440F100830023ADF8E4
:10E3A80002302B687B4F9AB21804A28040F1F682A3
:10E3B800BB8803F00F03BB71002B40F0C182784A81
:10E3C80013689BB23B803B8803F030037B803B881B
:10E3D80003F440533B8011684BF6BF730B4083F442
:10E3E800005383F0200343F4004343F08003136099
:10E3F800BB88D90621D4116848F60F730B406949C8
:10E4080013600B681A7A022A884601D0042A02D1BE
:10E41800F9F714FB5AE2062A40F06B825A78052A6B
:10E4280008D11A78520605D1D878FFF782FFBB6861
:10E438001B6A9847E3689B685AE213689BB2ADF879
:10E448000230BDF802301F0540F1D0811168554FE8
:10E4580040F68F730B40544913600A68534B92B2CD
:10E4680013445B0088461A683B68187A092817D055
:10E4780092B2520002F1804202F5C042117819703E
:10E48800517859709188C8B2090A41EA0021598027
:10E498001189C8B2090A41EA002199809289DA8073
:10E4A80001221A72DA8893F80190002A40F0DC8081
:10E4B8001A7812F07F024AD1B9F1090F0FD1DA7830
:10E4C800012A00F2B8809978002940F0B480998830
:10E4D800002940F0B0809A72A3685B68A9E0B9F19E
:10E4E800050F10D193F90320002A01DA0823B9E0B7
:10E4F8009A78002AFAD19A88002AF7D19B7A002BB9
:10E5080000F0A280F2E7B9F1030F0ED1DA78012A00
:10E5180040F091809A88002A40F08D805A7A42F023
:10E5280020025A72A368DB6983E0B9F1010F40F059
:10E538008280DA78012A7ED19A88002A7BD15B7A98
:10E54800980678D5F9F710FB00287DD073E0012AEA
:10E558002ED1B9F10B0F6ED1E26858799269D9784A
:10E5680090473B689A7A002A65D0002863D11A79C7
:10E57800002A60D19B78002B5DD1064B9B68DB6835
:10E588009847084B1B685A79DA72DA781A735BE095
:10E59800445C0040CC2000205C220020D22F0020C8
:10E5A800005C0040F4210020505C00400430002052
:10E5B800022A40D1B9F1010FC4D0B9F1030F3AD101
:10E5C800587920F0800E4FEA8E0202F1804101F561
:10E5D800B84110F0800F096814BF01F0300101F450
:10E5E8004051BEF1030F26D8B3F802E0BEF1000F88
:10E5F80021D101B39B7AF3B102F1804202F5B8420E
:10E60800010613684BBF23F4E04323F4804323F04F
:10E61800400323F070034BBF9BB29BB283F01003FF
:10E6280083F4805343F4004343F080031360A368EA
:10E638009B69984708E0E36848465B699847032860
:10E648000FD000287FF452AFD8F80020A14B92B227
:10E6580013445B001A6800221A6030236380062383
:10E6680000E009233A6847E1B9F1060F12D11A7898
:10E67800520678D19B78012B02D1E368DB6967E009
:10E68800022B02D1E3681B6A62E0032B6BD1E368BB
:10E698005B6A5DE0B9F1000F38D15988002962D171
:10E6A8005A6822F47F42B2F5003F5CD11A7812F022
:10E6B8007F0204D19B88002B00F0D58153E0012A0A
:10E6C80008D1E26858799269904700284BD13B6895
:10E6D8009B7A17E0022A46D15A7902F00F010BB251
:10E6E8009B0003F1804303F5B84312F0800F1B68C9
:10E6F80014BF03F0300303F44053032933D812F056
:10E70800700F30D1002B40F0AE812CE0B9F1080F2A
:10E7180004D11B785B0600F0A88124E0B9F10A0F48
:10E7280021D11A7802F07F02012A1CD19A7AD2B13B
:10E738005988C1B95A6822F47F42B2F5803F12D194
:10E74800E268587992699047002800F090810AE0C1
:10E758004BB13A684FF00008A2F812809361404626
:10E76800984740460BE0E3683A681B695078984739
:10E77800032804D1584B1B6809221A72BDE03A6875
:10E78800138A4FF6FF718B4201D10923B4E00228A6
:10E7980000D00BB90823AFE092F9001000291FDA66
:10E7A800D18801910198834202D9019B138210E01C
:10E7B8008B420ED2E16891F82C00834201D20021ED
:10E7C80005E093FBF0F100FB113313B90121434B32
:10E7D8001970E36893F82C309382F9F72FF98CE0DD
:10E7E800032313724FF44053238086E0BDF80230B0
:10E7F8001BB2002BBFF6D5AD116840F68F730B40E6
:10E808001360354A17683B7A022B904671D0042B67
:10E818006FD0032B01D0052B66D1BB693A8A8BB91F
:10E82800398A00293BD04FF4405323802C4B1A6877
:10E83800284B92B213445B001A6800221A603023F6
:10E8480063802CE0002AEBD0B7F81490914528BFDC
:10E8580091461FFA89FA504698473B8ACAEB030348
:10E868003B827B8A53447B821D4B1A681D4B92B2B4
:10E8780013445B0009F101021B689BB203F10053CA
:10E8880003F5405352105B004FF0000E9645C7D079
:10E8980053F82E1020F81E100EF1010EF6E7BB8A71
:10E8A8008B42D8F8003001D8032201E011B10522CB
:10E8B8001A720BE006221A72094B1A68054B92B2BB
:10E8C80013445B001A68196030236380D8F800305D
:10E8D8001B7A0FE002300020F4210020D12F002005
:10E8E800505C004004300020072B02D1E368DB684D
:10E8F80098470823D8F800201372FFF7E0FC5E4B16
:10E908001A684BF6BF7313402288D704228848BF81
:10E9180083F480539004628848BF83F40053D1067F
:10E92800628848BF83F01003920648BF83F0200333
:10E9380043F4004343F080034F4A9BB213602DE039
:10E948009A0002F1804202F5B842116889B2ADF826
:10E958000210BDF8021009B2002909DA106840F661
:10E968008F7101401160013B444A52F823309847A7
:10E97800BDF802301F067FF514ADA1798B0003F1B5
:10E98800804303F5B84348F60F72186802401A60CE
:10E998003A4B03EB81039B69984702E5A2883388C9
:10E9A8001340590505D54FF6FF332B60344B5B6890
:10E9B8009847A28831880A40920444BF4DF6FF73F5
:10E9C8002B60A3882F4A0B40DB0452D54EF6FF7309
:10E9D8002B6000231374137C052B41D8DFE803F068
:10E9E800030D1418222D6369264D1BB901F042FD51
:10E9F800062300E005232B743BE001F03BFD0423D4
:10EA080023740123636134E002236374032328E041
:10EA1800637C013BDBB26374637C53BB194B0422F8
:10EA28001A7426E0184A13689BB243F01003136067
:10EA3800052323740A2363741BE0637C114A013B9A
:10EA4800DBB26374637C03F0FF0093B90E490C6872
:10EA58004FF6EF7323400B6006231374506108E0F0
:10EA68000623237405E0094B73E6094B71E6094B4D
:10EA78006FE602B0BDE8F087005C0040188A010824
:10EA8800B4000020CC200020405C0040F176000853
:10EA9800A97700088577000810B54B88DC0641BFC8
:10EAA8002F4B14791B6853F8244044BF2D4B43F86F
:10EAB80020404B889B0641BF294B54791B6853F86B
:10EAC800244044BF274B43F820404B881C070ED5F1
:10EAD800254B0C781B78B3EB141FA1BF204BD478BF
:10EAE8001B6853F82440A4BF1E4B43F820404B88B2
:10EAF8009B070ED51D4B0C781B78B3EB141FDFBF9B
:10EB0800174B54781B6853F82440DCBF154B43F867
:10EB180020404B88DC070FD5154C0B78247803F080
:10EB28000F03A342DFBF0E4B14781B6853F8244031
:10EB3800DCBF0C4B43F820404B885B070FD50B78A4
:10EB48000C49097803F00F038B42A1BF044B92785C
:10EB58001B6853F82220A4BF024B43F8202010BDA5
:10EB6800C01A00200A0F0020571700205517002050
:10EB78005417002056170020254A26482649002306
:10EB8800F0B5156803700B701C461A462E19768866
:10EB98004EB92F5D3FB9037000230A704B70077898
:10EBA8001C461A460CE0360548BF013204F104043D
:10EBB80003F1010348BFD2B2802CDBB2E6D1EAE709
:10EBC800E0B2B8420CD215F8240006099E4200F0C3
:10EBD8000F00A8BF731C9042A8BF421C0134EFE786
:10EBE8008A704B70C2F3470102F001020A444C1EBE
:10EBF8000A490B480A70C3F3470203F001031344A0
:10EC080004700849501E084A08701370F0BD00BF10
:10EC1800C81A00204C170020E420002056170020B6
:10EC28005417002057170020551700202DE9F04FE2
:10EC3800C24BDA682DED028B1A61C14A1168D9609E
:10EC4800C0490B6843F020030B60BF4B19780129BA
:10EC580090460CBF002201221A70BC4B1A7891070B
:10EC680089B040F13D83BA490978042940F23883D4
:10EC7800B849097801F0040101F0FF0011B922F048
:10EC880001021A701B78DB0702D408B1F7F760FF9E
:10EC9800B149CA78531C052293FBF2F202EB8202B7
:10ECA8009A1AAE4BCA701B78039392000023AC4C9F
:10ECB800DFF8CCC2DFF8D8925CF8231091FBF9F5A5
:10ECC80004F1080004F1100640F82350A54844F860
:10ECD800231000FB051142F2107091FBF0F080B296
:10ECE80026F813004FF0140E04F1140604F13C0A40
:10ECF8000EFB036E5AF823605EF802704EF802109D
:10ED0800F61B314444344AF82310052691FBF6F1EA
:10ED180009FB051144F82310039C012C4FEA830BCF
:10ED2800E24605D10238B0F5797F98BF4BF80C1050
:10ED38000BB90123BBE7884CD8F80030226D9FED52
:10ED48008A7A8A4E8A4D9B1A07EE903AF8EE677ACD
:10ED5800D8F800302365C7EE877A7C4B1B78B7EE6E
:10ED6800008AF4EEC87AF1EE10FA58BFF0EE487A4D
:10ED780013F00103C4ED157A12D005AA00927D4B59
:10ED880006AA01920CCB9AE80300F7F7DFFD64218D
:10ED9800059A069BB2FBF1F293FBF1F3328000E097
:10EDA80033802B8094F858306B48002B3BD0D0ED43
:10EDB800157AC26DDAF80030C8EE276A9B1A026E1F
:10EDC800022507EE103AB8EEC77ADAF8043027EED3
:10EDD800267A9B1AFDEEC77AB0F9662017EE901ACC
:10EDE80007EE903A644BB8EEE77AD3ED007A67EE17
:10EDF800277A67EEA67AFDEEE77A17EE903A02FADE
:10EE080083F3B0F9642093FBF5F302FA81F29BB225
:10EE180092FBF5F292B2A0F86A30A0F86820A0F848
:10EE28006630A0F86420012384F85830534BDAF890
:10EE380004101B88DAF80000474D514E216603F094
:10EE48003003E065002B00F04B8205F1740300935A
:10EE580005F178030193EA6E2B6FF7F777FD726877
:10EE68002B6F9B1A07EE903A434B326893ED007A6A
:10EE7800EB6EF8EEE77A9B1AEB67384B67EE877A0A
:10EE88001B78FDEEE77A012BC5ED207A03D0022B23
:10EE980000F0DF8024E2D5ED287A3A4BD5ED215AEF
:10EEA80095ED255A95ED156A95ED264AD5ED274A33
:10EEB80035491D68B1EE677ABDEEC77AFDEEE77A8F
:10EEC80017EE10EA17EE90CA0020304A91ED007A4A
:10EED80052F8207007EE907AF8EEE77AA2F1140360
:10EEE80067EEA57A33F81060FDEEE77A283217EE60
:10EEF800903A9B1B9BB222F810301BB207EE903A57
:10EF0800F8EEE77A3B4467EE857A4400FDEEE77A4F
:10EF1800CDED037A07EE903AF8EEE77ABDF80C806B
:10EF280067EE847AA7EE867AFDEEC77A17EE902A06
:10EF3800724531DB6245A8BF62462EE02C080020EE
:10EF4800642400206C140020461200207014002055
:10EF580076140020CF2F0020E42000204410002049
:10EF6800E8200020806967FF00007A44EA14002046
:10EF7800EC140020481200207400002030150020F6
:10EF8800781400204810002078100020602100200C
:10EF980080969800DB0FC940724607EE902AF8EE7B
:10EFA800E77A5FED046AC1ED007AFDEEE77A313663
:10EFB80017EE903A43449AB2AB78D1ED027A07EE55
:10EFC800103AB8EE477A4B684F6027EE267AFB1A5C
:10EFD80088EE077AB6B2622E06EE903AF8EEE66A46
:10EFE80037EE067AC6EE866A86EE077A76EEE76A26
:10EFF800E7EE267AC1ED047AC1ED027A0FD964EE04
:10F00800A77ABA4EFDEEE77A17EE903AB3F5FA6FA3
:10F01800A8BF4FF4FA63B342B8BF334600E00023F9
:10F0280013441BB240F6B8329342A8BF1346B04A05
:10F038009342B8BF1346AF4AA352AF4A142303FB07
:10F04800002351F8142B1A60002840F04981012050
:10F058003BE7AA4BD5F874801F68D4F878903E89AE
:10F06800DFEDA78A4FEA58039E4228BF1E46B5F82F
:10F07800A8301AB29642C3BFD5ED157A9FEDA17A92
:10F0880067EE877AB6B2C1BFFDEEE77A17EE906AEF
:10F09800F618B6B2C8BFA5F8A860D4F8AC50C5EB4E
:10F0A80009052846F7F796FC0028D8BF404241F2E8
:10F0B80093129042CCBF0020012088B307EE905AEB
:10F0C800B8EEE70A20EE280AFAF7BFF907EE908AA9
:10F0D800F8EE677A40F6B83320EE270AFDEEC07ADC
:10F0E800CDED037ABDF80C20A4F8B02012B29A42F4
:10F0F800A8BF1A467E4B9A42ACBF09EB02034B44A9
:10F1080048F6A042934203DDA3F50C43A03B04E07C
:10F11800002BBCBF03F50C43A033C4F8B43001E0A6
:10F12800C4F8B490D4F8B450C5F50C53283307EE9E
:10F13800903AF8EEE77A67EEA88AB0EE680AFAF72E
:10F14800E7F98DED070AB0EE680AFAF77EF9D4ED13
:10F15800317AD4ED2E4AD4ED155A94ED2F4A94ED18
:10F16800305A65498DED060AB1EE677ABDEEC77A69
:10F17800FDEEE77A0DF1180E17EE10AA17EE90BA09
:10F188000020614AFEEC016A32F91030DFF88C91F8
:10F1980007EE903A07EE106AF8EEE77AB8EEC77A0B
:10F1A8003C32D6EE877A4FEA400CFDEEE77ACDED99
:10F1B800037ABDF90C30B3F57A7FA8BF4FF47A73A0
:10F1C8004B45B8BF4B461FFA83F922F810900FFA47
:10F1D80089F207EE902AF8EEE77A27EEA47ABDEED8
:10F1E800C77A8DED037A27EE847AD1ED007ABDF8DF
:10F1F8000C90E7EE257AFDEEE77A17EE902A524555
:10F2080003DB5A45A8BF5A4600E0524607EE902A4B
:10F21800F8EEE77A9FED3D6AC1ED007ABA7891ED94
:10F22800027A06EE902AF8EE666A4A684B6066EE45
:10F23800866A9A1AC8EE266A143106EE102AB8EEC3
:10F24800C66A76EEA56A86EE256AC5EEA66A36EE29
:10F25800476AA6EE867A01ED017A01ED037A25EE7A
:10F26800077ABDEEC77A17EE103ABDEEE77A4B443F
:10F2780017EE102A13441BB240F6B8329342A8BFC7
:10F2880013461B4A9342B8BF13461A4A2CF8023059
:10F298001F4A142303FB0023C3ED007A08B9012099
:10F2A8006FE73B7923B1642395FBF3F5194B1D8078
:10F2B8003B8898450DD9D4F8AC30A06FC01AF7F741
:10F2C80089FB80EAE072A2EBE07242F210739A4284
:10F2D80006DD114B01221A700E4BB4F8C8201A80B3
:10F2E80009B0BDEC028BBDE8F08F00BF30F8FFFF1E
:10F2F80048F4FFFFCC100020A01000204810002088
:10F30800D30237390000C8424C210020DB0FC94026
:10F3180078100020401000204410002018FCFFFF47
:10F32800F0B5974D2B78023B87B0082B00F29181FE
:10F33800DFE813F009002E004E0063007B008D000B
:10F3480009016E0179018F4B8F4C1A686368643329
:10F358009A4240F27E8100268C4B8D4A1B789E4251
:10F368000ADA2368884FD05C30B102F04DF93B6867
:10F37800013301363B60EFE72168834B525C002A7A
:10F3880040F067811A604FF0FF325A6003235FE153
:10F39800252300937F4B019303F10C02029249202D
:10F3A800A3F10A0250210233F9F7E0FC002840F0EB
:10F3B8005081794B1B6813F080024FF0FF31724B7C
:10F3C80003D083E80300042342E11A6059602AE06D
:10F3D800724A02230021009301910291482002F110
:10F3E8000803F9F7C3FC002840F03381664B4FF05F
:10F3F800FF3218605A6005232AE107230093684BFF
:10F40800019303F10C0202924720A3F108020021A4
:10F418000433F9F7ABFC002840F01B815A4B4FF03E
:10F42800FF3218605A60062312E15E4A0323002166
:10F43800009301910291532002F10803F9F796FC19
:10F44800002840F00681504B1860072300E14E4C1D
:10F45800236813B96360012323604C4B1A786368EF
:10F468001344402BA8BF4023132B636040F3F18063
:10F47800454B1B680D2B00F2E680DFE803F06007C0
:10F488000B0E121923282D3134404B51464802F0F7
:10F4980099F851E0454846493FE046484649474AB9
:10F4A80048E0474B474893F8CA1793F8CB2741E001
:10F4B800434B454893F8A4270C2101FB023393F8EA
:10F4C800A6172AE03E4B4148B3F8441125E03C4BCF
:10F4D8003F48B3F8461120E03E4B3F4819691CE00D
:10F4E8003E483F4B18E03F4B1B68D80404D5344BCB
:10F4F8003D4893F87C1110E00C2323601FE0304B4B
:10F508003A4893F8801193F8812193F87F3102F0FB
:10F5180069F811E03648374B198802F063F80BE0B8
:10F528001D4B1B6819050AD5254B3348B3F88411C0
:10F53800B3F9822102F056F86368181A60602368EC
:10F548000133236085E02D4B1B689A0114D52C4BA1
:10F558001B888BB92B4B1B6804932B4B0E201B6805
:10F56800059304A9F9F76AF8284B4FF480521A80DA
:10F5780009232B70F9F7DCF8F9F742F869E000BFC6
:10F58800D02C002064240020782E00200C010020BC
:10F59800548A0108BE8A010840240020708C0108A2
:10F5A800888C0108D48C01088AAD0108A7AD010830
:10F5B80059A20108BFAD010844A2010850A20108E0
:10F5C800A0240020D6AD0108EAAD0108F7AD010876
:10F5D80009AE0108902C00201BAE01082EAE0108D0
:10F5E80016000020602E00203BAE01084BAE01083B
:10F5F80067AE01085C2E002075AE0108E0110020FE
:10F608006C2E0020682E0020B02F0020802E0020B5
:10F61800114B1B78002BADD0104B1B689B01A9D454
:10F6280008232B70A8E70E4B1A680E4B5B68C8338B
:10F638009A4203D901F09EFF012309E001F0B4FFCB
:10F648000028F7D105E0084B4FF480521A800923AF
:10F658002B7007B0F0BD00BF642E0020E011002021
:10F6680064240020782E0020802E002007B5064B49
:10F678000093064B01930649064A074B0748F9F7DA
:10F68800B5FE03B05DF804FB50A2010859A20108B9
:10F69800D6A30108CFA3010844A2010865AF010859
:10F6A80008B5037833B90C4B0C481978BDE8084005
:10F6B800F9F79CBE06F042FA02280CD8064B1870DF
:10F6C800074B0C2202FB0030064B06301860FAF795
:10F6D800ABF80548E5E708BDB021002085AF010873
:10F6E800402C0020401200200BA2010808B5037826
:10F6F8003BB90B4B0B4893F8A417BDE80840F9F742
:10F7080075BE06F01BFA022808D8054B83F8A40733
:10F71800F9F7F4FFFAF7ACF80348E8E708BD00BFCB
:10F72800A024002089AF01080BA2010838B503788E
:10F7380003BB214B1B6801330F2B07D81F490C2231
:10F7480002FB03121C4695682DBB00E01C460134E1
:10F758000F2C01DD002400E005D818490C2202FB1B
:10F7680004129568BDB99C42F1D11548BDE83840EE
:10F77800F9F73CBE06F0E2F90F28044605D80F4A0F
:10F788000C2303FB00239D682DB921460D48BDE8D5
:10F798003840F9F72BBE084B1C60FCF753FB214699
:10F7A8002A460948F9F722FE0C235C43034B185DEF
:10F7B800BDE83840FCF758BB78000020EC8C010805
:10F7C80096AF0108ACAF0108C4AF010873B5037860
:10F7D80013B9FDF729FE3FE001AA204906F00FFA08
:10F7E80000240246264625469AB134B1012C08D198
:10F7F800104606F0A3F9064603E0104606F09EF907
:10F80800054601AA0020154906F0F9F90134024617
:10F81800EAE70B2D03D9124812490C230CE0022CFD
:10F8280011D1A6F57A73B3F57A7F08D90C480E4939
:10F838004FF47A724FF4FA63F9F7D8FD0CE00B4BEA
:10F8480003EB45035E80094B094803EB4503294652
:10F85800B3F90220F9F7CAFD02B070BD21A601086C
:10F8680037A6010856A601088AA90108B021002078
:10F87800DBAF010838B50D4C23688342054606D135
:10F88800FEF72DFA204600214C2206F0BCF8E36C66
:10F89800AB4209D12846FEF722FA054800214C223E
:10F8A800BDE8384006F0AFB838BD00BF6022002080
:10F8B800AC220020034B1A68D379591C1344D17128
:10F8C800187A70471015002010B5FFF7F3FF84B2BF
:10F8D800FFF7F0FF04EB002080B210BD10B5FFF772
:10F8E800F3FF0446FFF7F0FF04EB004010BD064BA2
:10F8F80010B5044621461868FCF7ABFC034B1B689F
:10F9080098796040987110BD1415002010150020DA
:10F9180038B5044624200D46FFF7E9FF4D20FFF7D0
:10F92800E6FF002C084C14BF21203E20FFF7DFFF24
:10F938002368002228469A71FFF7D9FF236893F8B5
:10F948004900BDE83840D2E71015002001460020E4
:10F95800DEE710B50446C0B2FFF7C9FF200ABDE8CC
:10F968001040C4E710B5044680B2FFF7F2FF200C40
:10F97800BDE81040EDE737B5828883680446100675
:10F988000D4641BF2B4991F8A4174FF4CC7000FBEA
:10F998000133D10544BF2849097802F03F0244BF2A
:10F9A80001EB410103EB8103042A12D006D8012A96
:10F9B8000DD0022A32D193F9001030E0102A0AD073
:10F9C800202A0AD0082A29D1B3F9001027E019788B
:10F9D80025E0198823E0196821E093ED000A6846BC
:10F9E800F9F784FB01461548F9F700FD05B3D4ED96
:10F9F800037A6846B8EEE70AF9F778FB014610483B
:10FA0800F9F7F4FC94ED040A6846B8EEC00AF9F771
:10FA18006DFB01460A48F9F7E9FC09E000210948AD
:10FA2800F9F7E4FC25B10848E1682269F9F7DEFC3A
:10FA380003B030BDA0240020B021002006A5010895
:10FA4800FFA40108AAA40108EAAF0108024B014675
:10FA5800D869FCF7FEBB00BFB021002010B5441EDA
:10FA680014F8011F21B1034BD869FCF7F2FBF7E743
:10FA780010BD00BFB0210020F7B52B492B4B0878EB
:10FA88002B4D1C682B4B05EB80001A882A4BD0F8AD
:10FA9800C0101B78294800914FF47A71B4FBF1F13A
:10FAA800F9F7A4FC26484821F9F7A0FC254B1F6864
:10FAB8000026F3B205EB8302D2F8D010E9B1012495
:10FAC8009C403C4217D0220715D01F4AD25C0B201D
:10FAD80000FB0323164A1D4802EB8303D3F8F020EA
:10FAE800F9F784FC022C06D1194B93F8281011B1B0
:10FAF8001848F9F77BFC0136DBE71748FFF7AEFF3C
:10FB0800164B17481A68174B9A420CBF164B174BDF
:10FB18001A88174B198892B24FF4FA6303B0BDE8FC
:10FB2800F040F9F763BC00BFBC1400206424002037
:10FB3800EC8C01085C14002001010020F1AF0108E1
:10FB480034B001086C1400200801002044B00108FA
:10FB5800B02100204CB0010894B00108D811002051
:10FB680050B0010800540040DC110020DE110020D4
:10FB7800D41100202DE9F0410024804625460F4E7F
:10FB8800A7594146384605F0C1FF58B139460C48D7
:10FB9800F9F72CFC30190021FFF7EDFE0948FFF7B3
:10FBA8005DFF0135143440F694439C42E7D11DB9FA
:10FBB8000548BDE8F04151E7BDE8F0818C8E0108A9
:10FBC8008CA5010894B001082EA501082DE9F04F75
:10FBD8002DED028B83B0054605F059FF064620B18E
:10FBE800012818D12B782A2B15D15C48FFF736FF4E
:10FBF80000245B4D5B486159F9F7F8FB2819314639
:10FC0800FFF7B9FE5848FFF729FF143440F694432C
:10FC18009C42EED19CE028463D2105F02AFF0028B1
:10FC280000F08F800346994613F8012D202AFAD058
:10FC3800441C204605F082FF80462046F9F7CCF99F
:10FC4800C5EB0909B0EE408A0026DFF834A114227A
:10FC580002FB06F40AF5D07B54F80B70384605F021
:10FC680016FF03461A4628463946019305F018FF41
:10FC7800019B00285BD15FFA89F29A4257D10AEBBF
:10FC88000402D2ED6B7AF8EEE77A0BEB0405B4EEDA
:10FC9800E78AF1EE10FA48DBD2ED6C7AF8EEE77AF3
:10FCA800B4EEE78AF1EE10FA3FD8B2F8A431D2F8F0
:10FCB800A82113F0200F08BF08EE108A1C0641BFC8
:10FCC8002A4991F8A4174FF4CC7404FB0122D905F2
:10FCD80044BF2749097803F03F0344BF01EB4101C2
:10FCE80002EB8102042B18EE100A0BD004D8013B5A
:10FCF800012B0ED810700CE0102B05D0202B06D04D
:10FD0800082B06D1108004E082ED008A01E082ED24
:10FD1800008A39461748F9F769FB2846002103B0DD
:10FD2800BDEC028BBDE8F04F25E6134803E0013631
:10FD3800A12E8AD1114803B0BDEC028BBDE8F04F6B
:10FD48008CE6284603B0BDEC028BBDE8F04F11E706
:10FD580003B0BDEC028BBDE8F08F00BF82B0010894
:10FD68008C8E01088CA5010894B00108A0240020FD
:10FD7800B021002097B00108A2B001082EA5010803
:10FD8800EC8C010870B50546284605F080FE06464D
:10FD980058B9194B19485A79194B03EB8203BDE836
:10FDA8007040D3F8301EF9F721BB28461549324672
:10FDB80005F076FE60B91448144CFFF74FFE54F86E
:10FDC800041F19B11248F9F711FBF8E7114805E0CB
:10FDD8000024114B53F8241019B91048BDE870409D
:10FDE8003CE62846324605F05BFE01340028F0D197
:10FDF800014B0B4D5C71C7E7A0240020C2B001087D
:10FE0800EC8C01081DA50108CEB001081C9B010857
:10FE180019A5010894B00108209B01082EA5010826
:10FE28000BA2010808B50748FFF718FE064BD8696A
:10FE3800FDF74AFFFCF76CFBF9F736FC034B044A65
:10FE4800DA6008BDE1B00108B021002000ED00E053
:10FE58000400FA0508B50548FFF700FE01F006F9A9
:10FE6800F9F74CFCBDE80840DCE700BFEDB001083D
:10FE780008B50448FFF7F2FDF9F740FCBDE8084073
:10FE8800D0E700BF03B1010820B9034B1B68082263
:10FE98001A82704701487047F42100207C00002036
:10FEA80020B9034B1B6808221A8270470148704723
:10FEB800F42100207C00002021B901288CBF0220F9
:10FEC800002070470220704710B5094B1A68D37894
:10FED800042B0BD8074C518ADB00234418B99B89A3
:10FEE8005B1A138210BD9B68581810BD002010BD06
:10FEF800F42100207C000020054B1968054B4A8A34
:10FF080018B99B8D9B1A0B827047986A10447047EA
:10FF1800F42100207C000020054B1968054B4A8A13
:10FF280018B99B8E9B1A0B827047186B1044704748
:10FF3800F42100207C000020074B1B681B7803F08D
:10FF48007F03212B06D100F0DF00022814BF022016
:10FF58000020704702207047F4210020212810B5A6
:10FF680008D1114B1B681B7803F07F03212B10D09D
:10FF7800022010BD2028FBD10B4B0C4A1B681070C7
:10FF88001B7803F07F03212B094B18BF00230BB903
:10FF9800EEE7084B044A1268002493615482204615
:10FFA8009847204610BD00BFF4210020D32F002021
:10FFB80091FE0008A9FE00087047034B1A78202A12
:10FFC80004BF00221A707047D32F0020014B04226F
:10FFD8001A607047B42F0020034B9B7B13B1034B6F
:10FFE80005221A60704700BFF4210020B42F0020BA
:08FFF8000D4B0E491A680E4B77
:020000040801F1
:1000000092B213445B000D4A1B68C3F3090310B599
:100010001362136A9BB201335B1000229A4206D02E
:10002000074851F8044B20F812400132F6E710BDA2
:10003000505C0040206200401E300020F42100206F
:1000400018220020014B00225A667047F42100203C
:100050002DE9F843664B674E1B68DFF8B881664AA6
:1000600000254FF0C0099D7283F80990DD7235605C
:10007000D8F8003023F4EC4323F0700343F400730A
:100080009BB2C8F80030D8F8003023F4E04323F0E6
:1000900040039BB248F2800483F010032343C8F866
:1000A0000030336812FA83F35B0040271A681F6040
:1000B00033689BB203F1005303F540535B002846BD
:1000C0001A6880221A60D8F8003023F4F8731B05F0
:1000D0001B0D2343C8F80030484B93F86410F7F722
:1000E00025FDD8F80030464A464923F4804323F0E2
:1000F00070039BB283F440532343C8F80030136865
:1001000023F4EC4323F070039BB21360336811FABD
:1001100083F35B0003201968C3F8009013683A4921
:1001200023F4E04323F040039BB283F020032343F6
:100130001360136823F4804323F0700323439BB2BE
:100140001360536823F4EC4323F0700343F4C0635B
:100150009BB25360336811FA83F35B0019684FF464
:1001600080711960536823F4804323F070032343A4
:100170009BB25360536823F4E04323F040039BB2E7
:1001800083F0200323435360D8F80C301F4A23F434
:10019000EC4323F070039BB2C8F80C30336812FABA
:1001A00083F35B0039461A684FF488721A60F7F7D8
:1001B000BDFCD8F80C3023F4804323F070039BB2CD
:1001C00083F440532343C8F80C30D8F80C3023F4A0
:1001D000E04323F040031C43A4B2C8F80C40284677
:1001E000FEF7ABF80A4B01221A60BDE8F88300BFA6
:1001F000F4210020505C0040043000207C000020EE
:10020000045C004008300020103000201C3000202A
:10021000B42F0020005C0040134A144B50681B6848
:10022000181810B5146808D011490822FEF771F8A3
:10023000204610490422FEF76CF80F48026800239C
:1002400093720E4A012111600D4913604FF4E0547E
:100250000B6014600B604FF43641A0F86810116019
:10026000084A136010BD00BFB0F7FF1FACF7FF1FB7
:10027000E6000020F6000020F4210020405C004051
:10028000445C0040B42F002010B50446B0F90000D3
:1002900001F0DFF9B4F9020001F0DBF9B4F9040070
:1002A000BDE8104001F0D5B910B50446006801F072
:1002B000D0F9606801F0CDF9A068BDE8104001F008
:1002C000C8B92DE9F74F0120FBF7F6FC002488B3ED
:1002D000012C2FD8194E4FF04C0909FB04FA06EBFC
:1002E0000A0808F1B407BD7815B10134E4B2EEE7AD
:1002F00090F9003090F804E01846114B03228DE885
:10030000240001212A4653F82E30FBF71AFE8346BB
:1003100060B106F16C00504429464A4605F077FB6F
:1003200001231C44C8F86CB0BB70E4B20120FBF799
:10033000A9FCCCE703B0BDE8F08F00BFF42100209A
:10034000E89B01080021222210B5114805F05FFB4F
:10035000104B0022194610480424105C83F8EA016F
:100360000132052083F8EF41042A4FF0000483F89E
:10037000EE0183F8F14183F8F00103F10803EAD1BB
:100380000123A1F8EC31522381F8E83110BD00BF00
:1003900088260020A0240020C0BB010810B5F7F774
:1003A0001DFD4FF43024012806D11CB1F7F716FDCE
:1003B000013CF8E7052010BD002C08BF052010BD4A
:1003C00070B50646441E14F8011F89B1094D284630
:1003D00005F053FB0028F6D005F1080398423FBF13
:1003E000054B401BC018A31B38BF80F88A31EAE7D1
:1003F00070BD00BFC4BB0108A02400200120002163
:10040000FFF78ABAF0B5184A92F80431D2F80871A9
:100410001546032B11D807EBC3025E1C941CF6B2E1
:1004200009D013469288D10705D5104203D008E0C1
:100430000131042908D13346EBE785F80431002067
:10044000F0BD93F802E00021074C0C2204F5867CF5
:1004500002FB01F31CF803209645E9D1234484F8FC
:100460000461D3F81001F0BDF4210020024B4FF4D9
:1004700080221A60704700BF140401400A4B10B577
:1004800019684FF6FB720A401A60084A927B1C46B4
:10049000074B0AB1052200E001221A6001F03AF888
:1004A0004FF43643236010BD405C0040F42100202F
:1004B000B42F0020772048210122F4F73DBC77209B
:1004C00058210122F4F738BC07B5002101AB032203
:1004D0007720F4F7B5FB9DF805309DF804001B026A
:1004E00043EA00439DF80600184303B05DF804FB9F
:1004F00008B5FFF7E9FF014B186008BDAC120020FA
:1005000008B5FFF7E1FF014B186008BDA8120020F5
:1005100013B501220DF1070304463A216820F4F7D0
:100520008FFB9DF8073003B10123237002B010BD8B
:1005300013B506220446432168206B46F4F780FB7E
:10054000A0B19DF800209DF8013043EA02232380EA
:100550009DF802209DF8033043EA022363809DF852
:1005600004209DF8053043EA0223A38002B010BDA9
:1005700013B5062204463B2168206B46F4F760FB66
:10058000A0B19DF800209DF8013043EA02232380AA
:100590009DF802209DF8033043EA022363809DF812
:1005A00004209DF8053043EA0223A38002B010BD69
:1005B0000F4B1A7813B51C46BAB90E4B1B68A3B182
:1005C0001A681AB10C49486902434A619A88ADF821
:1005D000042002228DF807209868002201A98DF8D6
:1005E0000620F4F717FA0123237002B010BD00BFF4
:1005F00030230020F80200200010024008B5FFF769
:10060000D7FF6B2180226820F4F796FB6420FBF76C
:100610008EFC6B2103226820F4F78EFB0F20FBF782
:1006200086FC104B19211A786820F4F785FB0F20FF
:10063000FBF77DFC0C4B1A211A786820F4F77CFB41
:100640001B2118226820F4F777FB1C211022682058
:10065000F4F772FB682037210222BDE80840F4F766
:100660006BBB00BF2C0300200000002008B5FFF783
:100670009FFF074B1B7813B1012B03D008BD4FF42C
:10068000006201E04FF48052024B1A8008BD00BFA7
:10069000FC020020160000202DE9F0410369C76824
:1006A00005460E461F40002F35D0B7FA87F24FF0AF
:1006B0000043D340DB432B611F40A2F11B03042BFB
:1006C000F1D8DFE803F0221F1C190300746A24B17B
:1006D000013C0023A4B2736201E0EC6AA4B2D6F834
:1006E0002080B8F1000FDED0D8F800304046214617
:1006F0009847D8F80480F4E73068696B07E07068C1
:10070000A96B04E0B068E96B01E0F068296C03684C
:1007100089B29847C7E7BDE8F08107B52320FBF70A
:1007200006FC6820752101220DF10703F4F788FA11
:1007300028B19DF80700A0F168035842584103B062
:100740005DF804FB024640213C20F4F7F5BA70B591
:1007500000EB8000094CA0F1A1059C38254404441D
:10076000074B15F8010F1E787040FFF7EBFFA5420D
:10077000F6D13046BDE87040E4E700BFA89C010810
:10078000D42F002010B5441E14F8010F10B1FFF74C
:10079000DEFFF9E710BD024680213C20F4F7CCBA19
:1007A00010B5D420FFF7F7FF8020FFF7F4FFA82053
:1007B000FFF7F1FF3F20FFF7EEFFD320FFF7EBFF3E
:1007C0000020FFF7E8FF4020FFF7E5FF8D20FFF74F
:1007D000E2FF1420FFF7DFFFA120FFF7DCFFC820B6
:1007E000FFF7D9FFDA20FFF7D6FF1220FFF7D3FF7C
:1007F0008120FFF7D0FFCF20FFF7CDFFD920FFF7F3
:10080000CAFFF120FFF7C7FFDB20FFF7C4FF40203E
:10081000FFF7C1FFA420FFF7BEFFA620FFF7BBFF35
:10082000AF20FFF7B8FFA620FFF7B5FFAE20FFF718
:10083000B2FF2020FFF7AFFF0020FFF7ACFFB02092
:10084000FFF7A9FF4020FFF7A6FF0020FFF7A3FF57
:100850001020FFF7A0FF4FF48064013C0020A4B2F9
:10086000FFF770FF002CF8D18120FFF794FFC8201C
:10087000FFF791FFAF20FFF78EFF012010BD08B5F5
:100880005038C0B2FFF787FF0020FFF784FF102029
:10089000BDE808407FE7503910B50446C8B2FFF7FD
:1008A0007AFF04EB4400400004EB440400F00E0027
:1008B000FFF771FFC4F3C3001030BDE810406AE7D2
:1008C00001480249E8E600BF00480140C81900207D
:1008D00001480249E0E600BF00400140A0190020A5
:1008E00001480249D8E600BF000400407819002002
:1008F0004FF080400049CFE65019002001480249DE
:10090000CAE600BF002C0140281900200148024916
:10091000C2E600BF002C014028190020224B10B570
:10092000224C5A43224BB3FBF2F203880139013ABD
:10093000A04289B292B29BB20ED004F50064A042EC
:100940000AD0B0F1804F07D0A4F59834A04203D06C
:1009500004F58064A04202D123F070039BB2154CD1
:10096000A04206D004F58064A0421CBF23F440736B
:100970009BB203800D4BC162984202850FD003F5F4
:10098000006398420BD003F54063984207D003F50B
:100990008063984203D003F58063984201D100231D
:1009A00003860123436110BD40420F00002C01402B
:1009B00000A24A04001000400E4B800A984216D054
:1009C00007D8B0F5801F0CD04A3B98420DD10220C9
:1009D0007047094B984206D00233984205D1042053
:1009E00070470120704703207047FE2070470020A9
:1009F000704700BF4B00100050001000F8B50468AD
:100A0000064620460F461546FFF7D6FF04284BD86A
:100A1000B27A910847B902238B40D4F80CE0DB434B
:100A20009BB203EA0E03E3600A23204A03FB001390
:100A300042F82370043342F8235015463FB1B17A8F
:100A4000E268890802238B409BB21343E3602822AB
:100A500002FB00522032EFF31286502383F31288F8
:100A600003B203EB8303DB0003F10C011C332944C5
:100A70002B4451F8047F17B117600A680432994279
:100A8000F7D100231360F3B283F31188282303FB0B
:100A90000050036A1BB1E36843F0010303E0E2681E
:100AA0004FF6FE731340E360F8BD00BF2819002025
:100AB0000148FDF793B900BF342300200148FDF73A
:100AC0008DB900BF882300200148FDF787B900BF1A
:100AD000DC2300200C4B0D49DA684378D243C2F383
:100AE0000222C2F10402934002781B010A44DBB2E5
:100AF00082F8003303780122580903F01F0302FA39
:100B000003F341F82030704700ED00E000E100E021
:100B100073B50546002100680122FFF7FFFE2A6831
:100B200013889BB243F001031380EB7A8DF80430F5
:100B30000124002601A88DF805408DF806608DF887
:100B40000740FFF7C7FFEB7A1B2B0BD1192301A836
:100B50008DF804308DF805408DF806608DF807405B
:100B6000FFF7B8FF02B070BDF0B5BE4C23782DED95
:100B7000028B013B012B85B000F26F8165788542C5
:100B800040F06B81A378022B00F06781B64B5B5D70
:100B9000E37023796D00F2EE048A1BB16319B3F997
:100BA000063009E06319D4ED037AB3F90630F1EEAB
:100BB000677AC4ED037A5B4208EE103A2369A94EC6
:100BC000B8EEC88A1A0388EE288A35D5D6ED037A9E
:100BD000FDEEE77A28EE280A17EE903AD6ED057A70
:100BE0008DF80A30FDEEE77A17EE903A8DF80B306B
:100BF00005F062F9FCEEC07A96ED060A17EE903A1F
:100C000020EE280AADF8083005F056F9FCEEC07A5F
:100C100096ED070A17EE903A20EE280AADF80C3050
:100C200005F04AF9FCEEC07A0C2017EE903A02A9C2
:100C3000ADF80E30F7F706FDD4ED077A894BF5EEE7
:100C4000407AF1EE10FA60D1D3ED067AB4EEE78A7D
:100C5000F1EE10FA04DDDA6883ED068A5A61E8E005
:100C6000F5EEC07AF1EE10FA40F3E38093F820201D
:100C700042B1022A00F2DD805A6B83ED078AFA3214
:100C80009A63D6E0D3ED037A38EE678AF7EE007AFE
:100C9000B4EEE78AF1EE10FAACBF01210021D3EDEA
:100CA0000A7A69B19FED717A27EE877ADFED707A63
:100CB000B4EEE77AF1EE10FA58BFF0EE477A03E0AF
:100CC0009FED6C7A67EE877AC3ED0A7A2369654AED
:100CD0001B0311D58DF80810D378116B0B440B2032
:100CE0005A788DF80920DA7A8DF80A205B7D8DF824
:100CF0000B3002A9F7F7A6FC0123226B84F8203001
:100D0000E37813440022DA7291E0B4EEE78AF1EE60
:100D100010FA48BF83ED078AA16B636B94ED067AE6
:100D2000D4ED076A591AC943C90F77EE667A59B9E3
:100D3000B7EE006AF4EEC67AF1EE10FA79DDB4EEA1
:100D4000E68AF1EE10FA74DDD4ED056A454BB4EE97
:100D5000E67AF1EE10FACCBF0126002666B1D3ED9B
:100D6000097A9FED427A67EE877A9FED427AC3ED6A
:100D7000097AD3ED0B7A0AE0B0EE007AF4EEC77A86
:100D8000F1EE10FA08DDD3ED0B7A9FED387A67EEBD
:100D9000877AC3ED0B7A07E0D3ED097A9FED357AB8
:100DA00067EE877AC3ED097AD4ED097A206BE27891
:100DB00067EEA87A1044FCEEE77ACDED017A9DF853
:100DC00004304370D4ED0B7A2769FCEEE77A3F03D9
:100DD000CDED017A9DF8042042750ED546EA410119
:100DE0008DF808108DF80930C37A8DF80A300B2081
:100DF00002A98DF80B20F7F725FC94F82020194B59
:100E0000022A11D1D3ED0A7A9FED1B7A196B67EE96
:100E1000877A002283F82020FCEEE77ADA7817EE52
:100E2000903A0A44D37202E0022283F82020F5F7B8
:100E3000FFFE22790B4B0AB1104A00E0104ADA603B
:100E40002544D4ED037AB5F9063000EE103AB8EE39
:100E5000C00A80EE280A37EEC00A05B0BDEC028B4E
:100E6000F0BD00BF302400204B9F0108EC51783FBB
:100E70006F12833A0AD7833F00007A440000A041F2
:100E80000000A0C12B4BF0B52B4D1E6805F11000E2
:100E90002F78F3192C46597801F00401013501F03F
:100EA000FF0219B18542F3D10020F0BD224D631B32
:100EB000022B0ADD1AB102EB82025200D2B215F8FF
:100EC000013B303B1A44D2B2F1E70021AC420AD9CF
:100ED00019B101EB81014900C9B215F8013B303B62
:100EE0001944C9B2F2E72E2F16D101340420002391
:100EF0002578771903EB83037F785B007F079BB22C
:100F000044BF303D5B1900F1FF3044BF01349BB258
:100F100010F0FF00ECD100E00023084841436420BA
:100F200000FB03130620B3FBF0F3054800FB02307F
:100F3000F0BD00BF100100206C24002040420F00D3
:100F40008096980030B500231A4610498C1894F802
:100F50003C40BCB12E2C06D1013298B18C1804440F
:100F6000002584F83C5011440A2491F83C10634356
:100F7000A1F13004092C9CBF303B5B180E2A03D82A
:100F80000132E2E7184630BD002030BD3024002099
:100F9000104B10B50446185CFFF7D9FB0E4800EB68
:100FA0004400B0F94C10B1F57A7F05DBB1F5FA6F6A
:100FB000A8BF4FF4FA6101E04FF47A71A1F57A719C
:100FC0000A23092091FBF3F1BDE81040C9B2F9F7FB
:100FD000EFBA00BFC4BB010830240020031EB8BF15
:100FE0002D2210B5B8BF58420C46B8BF01F8012BEE
:100FF0000A22F8F7E9F800230370204610BD0B4AD7
:10100000136913F4805FB2F9523006D0B2F80822A7
:10101000111A8B4208DD104401E0B2F80A02834243
:10102000B4BF002001207047012070473024002009
:101030000E4B1A78692A16D15A88B2F5FA6F12D176
:101040001A79BE2A0FD193F8CD27EF2A4FF000006E
:101050000BD113F8012B5040054A9342F9D1B0FA55
:1010600080F04009704700207047704700F803087F
:10107000D0FF03082DE9F04FEF4C00214FF4FA6246
:1010800085B0204604F0C3FCEC4B04F537721A60BF
:10109000EB4B00221A70EB4B04F2A6711960692326
:1010A00023700323637140F20113A3604FF416739E
:1010B000A4F86631FA23A4F86831BC23A4F864319B
:1010C0004FF4FA732021A4F86E31012384F86231C1
:1010D00084F86A1184F87E316E2184F88631052304
:1010E00084F87C1184F81B320A2140F2DC5384F826
:1010F0007D11A4F898312B2140F24C4384F87F11E4
:10110000A4F89A31212140F26C7384F88011A4F87C
:101110009C31232140F2753384F88111A4F89E316B
:101120004FF4C87140F64303A4F8A031A4F882112B
:1011300023469918023200254FF01E091C2ABE4C86
:1011400081F8A25181F8A391F3D14FF4FA6340F2F0
:101150007E4040F27E57DFF8E4B2A4F8C031A4F834
:10116000C431A4F8C831A4F8CC31A4F84401052353
:1011700040F23A70A4F84C7140F2EA5701264FF45D
:101180007A78C82219214FF0320A84F8D631A4F8AF
:1011900046014FF4C87340F2DC50A4F84E7140F29F
:1011A000B457A4F8DA21039284F8959184F8D561B4
:1011B00084F8D711019184F8D86184F8D96184F852
:1011C000DC61A4F8DE3184F8E261A4F84A010290FF
:1011D000A4F85071A4F8543184F8E561A4F8BE81F4
:1011E000A4F8C281A4F8C681A4F8CA81A4F84881F1
:1011F000A4F852A1A4F856A1FFF7A4F8DBF8003038
:1012000026744FF0170E83F815E083F816E04FF0C0
:10121000550EE673A573A58183F803E04FF00F0E1A
:1012200083F805E00199D9714FF0220E83F806E0AA
:1012300021214FF00E0E83F80B9083F80C9083F869
:1012400010E059744FF0350E53214FF064092827F0
:101250004FF02D0C83F81AE0D9764FF05A0E0A2180
:1012600083F81C904FF0780983F80DC083F808E0EC
:10127000997483F80A901D705F709F70DD7583F814
:1012800004A09D731D76DD735D765F7283F814C0D4
:101290004FF4FA7CA3F84EC0DFF8C0C1C3F838C0E1
:1012A000C3F83CC0DFF8B8C1C3F828C04FF07E5C7B
:1012B000C3F834C0F7EE087ADFF8A891DFF8A8C1C8
:1012C000C3ED087AC3F82C90C3ED097AC3F83090C7
:1012D000C3F848C0F1EE047A02989E774FF04B0CA9
:1012E0004FF0000983F8501083F8525083F8517082
:1012F000C3F84090C3ED117A83F84CC084F8A6E798
:10130000A4F8B0074FF0410E042084F8A7E784F852
:10131000A8A784F8A95784F8AD5784F8AE5784F885
:10132000AA5784F8AB5784F8AC5783F85C001520B3
:101330000191A3F85850A3F85A50A3F85650C3EDA2
:10134000187A83F868004048D866404818674048D3
:10135000586783F878603F4883F8647083F8657055
:10136000FFF72EF8DBF800300199039A83F8146137
:101370004FF4487083F8115183F8125183F81371B8
:1013800083F81851A3F816015E4684F8D01184F84A
:10139000D121A4F8D28119460E2202FB05326FF04A
:1013A000170082F81901032082F81A016FF02F004C
:1013B00082F81B01072082F81C016FF0230082F8DD
:1013C0001D01052082F81E0101355A2081F82001F7
:1013D00081F821016422FF20082D81F81F2181F866
:1013E000220101F10E01D7D1002183F88911C82112
:1013F000A3F88A11142183F88C11A3F890211E21DF
:101400004FF4967283F88D11A3F8922101212822BE
:10141000A3F8942183F88E11074B03F1C0021F46F5
:10142000C3F8149010339342FAD10B4800214022A4
:1014300004F0EDFA1AE000BFA02400201C120020E6
:10144000B0210020401200209A99193FF6287C3FD5
:101450003D0A773FD9BB01083C2700208FC2F53CED
:1014600000002040CDCCCC3E000040400023264D63
:10147000264C5959FA1804330868C2F89C02382BD4
:10148000F5D104F507700021802204F0C0FA05F1BF
:101490003801702204F5077004F0AEFAFDF770FB16
:1014A000366800230125314604F274404FF4CC72B3
:1014B00084F8CC3784F8CA5784F8CB5704F09CFAE8
:1014C00004F20C6031464FF4CC7204F095FA104BE4
:1014D0001B681A68C4F8B2275A68C4F8B6279A6815
:1014E000C4F8BA271A68C4F8BE275A68C4F8C227D5
:1014F0009A68C4F8C627022384F8C85484F8603672
:1015000005B0BDE8F08F00BF509F0108A024002067
:10151000401200201549D1F8883043F47003C1F817
:101520008830134B1A6842F001021A605868114A59
:1015300002405A601A6822F0847222F480321A60E3
:101540001A6822F480221A605A6822F4FE025A6055
:10155000DA6A22F00F02DA62186B074A02401A6355
:1015600000229A604FF000638B60704700ED00E04E
:10157000001002400CC07FF8CCFC00FF38B5094BCE
:1015800093F8CC5765B9084C2068FCF7ACFB074BC7
:1015900025601B78022B03D1BDE83840FEF791BED1
:1015A00038BD00BFA0240020DC2C0020D82C002057
:1015B000044B93F8CC371BB9034B1868FAF741BEBC
:1015C00000207047A0240020DC2C002038B5054600
:1015D0000446204614F8011B21B1034B1868FAF7A2
:1015E0003CFEF6E7401B38BDDC2C00200FB407B5ED
:1015F00004AB064953F8042B01930020F7F7F8FDDC
:1016000003B05DF804EB04B0704700BF5B1601083F
:10161000024B01461868FAF720BE00BFDC2C002000
:1016200010B50446C0B2FFF7F3FFC4F30720BDE8CE
:101630001040EDE710B504467F2C06D964F07F001A
:10164000C0B2FFF7E5FFE409F6E7E0B2BDE81040FD
:10165000DEE7430083EAE070ECE70846D8E700BF26
:10166000064B1B7803F0040303F0FF001BB1044B8F
:101670001888C0F3C01000F001007047CF2F002081
:10168000301500202DE9F04F2DED028B87B000269C
:101690000493B24B0392B3F90270B3F90030019096
:1016A000002FB8BF7F42002BB8BF5B429F42B8BF3C
:1016B0001F46B7F5FA7F8146A8BF4FF4FA77B046C8
:1016C0000296B3463446A64D2B8813F0030F4FEA1B
:1016D000440A58D0022C56D0A04BA24A33F80A3004
:1016E00032F90A20022113FB0122039B5B429A423A
:1016F00003DB039B9342A8BF13469B4A32F90A209F
:101700009B1A049A32F91420134408EE103AFFF79A
:10171000A7FF68B1B8EEC80A944BB2EE048A80EE17
:10172000080A185DFFF720FA20EE080ABDEEC08A0D
:1017300018EE102A99F808305343642293FBF2F311
:1017400099F81C206FF0040B0BFB02FB5B4504DBDC
:1017500002EB820B9B45A8BF9B46854918EE103AC9
:1017600051F82420134442F210729342A8BF13464A
:10177000804A9342B8BF134699F8122041F82430AA
:1017800053431B1302932B8803F00302012A01D158
:10179000022C3FD17848714A30F90A0032F90A80A8
:1017A0007649019A51F82460557880EAE07EAEEBE4
:1017B000E07EBEF5206F4FEA84021EDC022C15D0BD
:1017C00008EB8801090191FBF5F5042190FBF1F08C
:1017D0002D1A2E44B6F57A5F68496948A8BF4FF4C0
:1017E0007A568642ACBF5650505008E088EAE87EF0
:1017F000AEEBE87EBEF1640FE2DD002088505F4969
:101800007D26525892FBF6F6019AD27A7243402610
:1018100092FBF6F69A0713D5022C11D00298C7F561
:10182000FA7307FB06F507FB08F203FB0B224FF4E4
:10183000FA7103FB005392FBF1F293FBF1F508E020
:10184000DB0704D5022C02D0029D5A4601E0354642
:101850004246494B33F91410042391FBF3F34949F1
:10186000615C4B436FF04F0193FBF1F399F851101A
:10187000D3184FEA440A08EE103AB1B1022CB8EE80
:10188000C80A414B08D14A0803D09142A8BF11466B
:1018900000E001213D4802E03D4800EBC400D3EDEB
:1018A000000AF7F773FBBDEEC08A334B394A3AF8AA
:1018B00003003AF902302AF8020001B202F10800EE
:1018C0001432CB1A50F824E0042193FBF1F152F8C2
:1018D000243040F8241073440B4499F8501042F817
:1018E00024E04FEA840C00EE103A79B1264B2A48E6
:1018F000D3ED000ACDF814C0B8EEC00A00EBC40066
:10190000F7F744FBDDF814C0BDEEC00A234A2449B2
:10191000125D10EE103A5343202293FBF2F318EEBF
:10192000102A2A44D21A2AF801201E4A18EE101A48
:101930004CF802101C4A4CF802501C4A5B424CF80E
:101940000230019B01340133032C01937FF4BBAEC1
:1019500007B0BDEC028BBDE8F08F00BF5014002033
:1019600030150020C82F0020362400206481010893
:1019700020180020F0D8FFFF00120020AC17002034
:1019800080C1FFFF28180020A8170020A017002002
:1019900090170020702C0020DC1700204018002039
:1019A000F4170020FC17002008180020141800204D
:1019B0002DE9F04F2DED088B83B092460093CF4B6D
:1019C00001931A8812F0020F0446F7EE009A4CD0E9
:1019D000149BCB48DD89B0F900305B1B03F2F31692
:1019E00040F2E632964203D8002BB8BF5B4201E0DA
:1019F0004FF4FA73B0F90220521B02F2F31540F2D1
:101A0000E630854203D8002AB8BF524201E04FF4C5
:101A1000FA7294F84C0058B39342B8BF1346C3F51A
:101A2000FA7307EE903A9FEDB77AF8EEE77A6423FF
:101A3000C7EE877A93FBF0F307EE103A77EEE97A78
:101A4000B8EEC77AB0EE699AA7EE879AF7EE006A09
:101A5000B5EEC09AF1EE10FA0AD4B4EE669AF1EE41
:101A600010FAC8BFB0EE669A04E0B0EE699A01E0E1
:101A70009FEDA59A01F1030826464FF00009B9F140
:101A8000020F18F8015FDFF8E0B24FEA4907B2EE43
:101A900004BA0DD1BBF904209FED9C7A0A3502FBF4
:101AA00005F307EE903AF8EEE77AC7EE877A44E05E
:101AB000974A3BF9190032F919201044CAF1000283
:101AC000904203DB50450246A8BF52469148009B16
:101AD000C05F101A33F91920831808EE103AB8EED7
:101AE000C88A88EE0B8AFFF7BBFD40B18A4A12F81C
:101AF0000900B0EE480AFFF737F8B0EE408A019BC4
:101B00001888C20704D5D4ED117A68EE277A14E05C
:101B10003BF907209FED7D7A143502FB05F307EEB4
:101B2000903AF8EEE77A8307C7EE877A42BF94EDE2
:101B3000127A28EE078AE8EE097A784A94F851106A
:101B4000D35F774A96ED08AAD2ED0C6A9FED758AAD
:101B5000754D07EE103AB8EEC77A744BE7EE667A29
:101B600019F80330F0EE48BAF0EE678A67EE8A7A29
:101B70000AEE103AB8EECAAA27EE8AAA8AEE08AA96
:101B8000C1B1B9F1020F0AD1480803D08142A8BF00
:101B9000014600E00121B0EE4A0A654804E06548CC
:101BA000B0EE4A0A00EBC900D5ED000AF7F7EEF9EE
:101BB000B0EE40AAD5ED000A5F4996ED0B7A4FEAE8
:101BC000890B68EEA07A594467EE877AD1ED00AAB6
:101BD000E7EE8BAADFED597AF4EEE7AAF1EE10FA00
:101BE00009D4DFED577AF4EE67AAF1EE10FAC8BF18
:101BF000F0EE67AA01E0F0EE67AA89EEA07A514AFA
